:020000040800F2
:100000000000022075BA0508AD910008E121020840
:1000100025BB050825BB050825BB05080000000019
:10002000000000000000000000000000D1AD00084A
:10003000D3AD000800000000D5AD0008790B010821
:1000400025BB050825BB050825BB050825BB0508FC
:1000500025BB050825BB050837EE00083BEE000868
:1000600025BB05083FEE000843EE0008B5990008DF
:10007000C9990008DD990008F1990008059A00085F
:10008000199A00082D9A000825BB050800000000F9
:1000900000000000000000000000000047EE000823
:1000A000ED980008159900083D990008D7980008B8
:1000B00065990008799900088D99000825BB050805
:1000C00025BB050825BB050825BB050825BB05087C
:1000D00025BB05083994000845940008000000007D
:1000E0004BEE000825BB0508D7AD00080000000056
:1000F000000000000000000000000000419A00081D
:100100000000000025BB0508A199000825BB0508D3
:1001100000000000000000000000000000000000DF
:10012000559A0008699A00087D9A0008919A00087B
:10013000A59A000800000000000000000000000078
:1001400000000000000000000000000029AE0008D0
:10015000B99A0008CD9A0008E19A000825BB050865
:1001600025BB050825BB05080000000000000000B5
:10017000000000000000000000000000000000007F
:100180000000000025BB0508000000000000000082
:0801900025BB050825BB05088D
:0801980008B60500010000009B
:1001A0002CFD00200209000008013D004CFD00204C
:1001B000010C0000000076006CFD00200110000022
:1001C000000076008CFD0020010D0100000077008A
:1001D000ACFD00200114000000001E00CCFD00203A
:1001E000011A000000000D00ECFD002001160000C7
:1001F00000000C000CFE0020011B000000000E009F
:100200002CFE0020011C000000001E004CFE0020FF
:100210000117000000000C006CFE00200118000017
:1002200000000E008CFE00200119000000000C00F0
:10023000ACFE00200128010000001800CCFE0020C8
:100240000120000000004800ECFE00200121000019
:10025000000049000CFF00200122000000004A00BD
:100260002CFF00200123000000004B004CFF002069
:100270000124000000004C006CFF0020012500005C
:1002800000004D008CFF00200126000000004E0001
:10029000ACFF00200127000000004F00CCFF002031
:1002A000012B000000002900ECFF0020012C0100C0
:1002B000000029000C000120012D01000000700049
:1002C0002C000120012E0100000052004C000120F2
:1002D000012F0100000028006C000120022901000C
:1002E00000012C008C0001200132000000003C00C5
:1002F000AC0001200135000000002000CC000120EE
:08030000013600000000290095
:10800000D0E907239A422FBFD01AC0688018C01A3F
:108010007047D0E9092300699A4238BF1218D31A71
:108020000138C01A7047D0E90902131A5842584162
:108030007047036A41690246C85CD16801338B42CC
:1080400028BF002313627047436A8269D154436A90
:1080500002690133934228BF0023426B4362D36815
:1080600043F08003D3607047436B188810F0100012
:108070001EBF1A889B8801207047436B99891A8814
:10808000890610B592B2044607D5900605D5E26A76
:1080900022B39888216B80B29047636B99891A88C4
:1080A000090692B20FD510060DD5D4E909128A42FD
:1080B00022D0A169895C998021690132B2FBF1F07B
:1080C00001FB1022A262998A1A88C90592B204D5CE
:1080D000D20744BF4FF6F7721A8010BD9B88E26941
:1080E0006169DBB28B54E369E2680133B3FBF2F1FF
:1080F00002FB1133E361D0E7DA6822F08002DA6034
:10810000E1E77047064A002352F83310814201D15B
:10811000D8B2704701330E2BF6D1FE20704700BF56
:10812000901406087047036941681F2B30B54FF063
:10813000200285BFA3F120054C680C68AA4098BFB7
:108140009A40224220D0826900201074D06884684E
:10815000206820F0010020605068046845790B48D1
:10816000A28900EB450092B2B0F870001F2B22EA02
:108170000002A28188BF203B4FF020028BBF9A40B3
:1081800002FA03F3CA608B6030BD00BF901406088A
:108190000E4BDA68D20310D4DA68D1060FD4DA684D
:1081A000D2050ED4DA6812F0E00F0CD1DB6813F0C0
:1081B000020F14BF082009207047012070470620D5
:1081C0007047022070470720704700BF003C024004
:1081D00007B509238DF80730FFF7DAFF8DF80700A0
:1081E0009DF80730012BF7D09DF8070003B05DF82C
:1081F00004FB838A028B9BB243EA024331EA030306
:108200000CBF01200020704782B00023019300932F
:10821000012300900193019B63B1009A21F07F43F9
:1082200014320092009A12681A4214BF01200020F2
:1082300002B07047009A1832F3E770477047012088
:108240007047044BD3E90003984288BF03F50063ED
:10825000181A7047F0150020054AD2E900318B4208
:10826000FDD0D1180133C3F30A03087A13607047B5
:10827000F0150020044BD3F8080820B1D3F8080803
:10828000431F584258417047F0150020012380F8E1
:108290004930704710B5D0F8E83504461B69984757
:1082A000032384F81231002010BD08B590F8123174
:1082B00080F81331042380F81231D0F8E835DB68F8
:1082C0009847002008BD08B5D0F8E435DB6903B154
:1082D0009847002008BD08B5D0F8E4351B6A9847D8
:1082E000002008BD08B5D0F8E4355B6A9847002047
:1082F00008BD10B5074C2068FF2808D00649D1F802
:108300000C2801F5016100F035F8FF2323600020FF
:1083100010BD00BF00000020F015002043230148DD
:108320000B80704704000020122301480B80704727
:1083300047000020042301480B80704759000020AB
:10834000704770477047704770477047044B002074
:108350000522C3F80828C3F81808C3F81C0870479A
:10836000F0150020024B0020C3F80808704700BF3A
:10837000F0150020212838B50C461BD022282BD020
:10838000202815D1A1B1072A12D11A4DD5F81C38D1
:1083900013B10968002098472368C5F8203823796D
:1083A00085F82438637985F82538A37985F8263847
:1083B000002038BD0029FBD0072AF9D10D4BD3F896
:1083C00020280A6093F824280A7193F825284A7116
:1083D00093F826388B71EBE70029E9D0022AE7D120
:1083E000044BD3F81838002BE2D0098800209847B6
:1083F000DEE700BFF0150020074AD2F82838D2F88F
:108400002C28934203F1FF338CBF002001209B1ADC
:1084100003EBC020704700BFF0150020ECE730B53B
:108420000F4CD4E900239A4286BF03F50065AA1ACF
:108430009A1A0A44B2F5006F10D801440022814212
:1084400003D102B16360002030BDE21810F8015B77
:1084500015720133C3F30A030122F0E70220F3E7A8
:10846000F0150020007970470079C0F34010704784
:1084700000794009704700BF704700BF704700BFD8
:10848000D0ED007AD0ED036A30EE677AE6EE877AB7
:10849000B0EE670AC0ED007A704700BFD0ED017AF8
:1084A00080ED021AF5EE407AF1EE10FA04BF9FED6E
:1084B0000C7AC7EE207A31EE277A08BFC0ED017A38
:1084C000C1EE076AD0ED007AC0ED036A30EE677A3C
:1084D000E6EE877AB0EE670AC0ED007A704700BF1B
:1084E00083F9223E9FED047AC7EE007A77EEA07AF8
:1084F00080EEA70A704700BF72C7D13D002303601A
:10850000436080ED020A704790ED017AD0ED036A76
:10851000D0ED027A30EE470AA6EE807A90ED000A9E
:1085200080ED017A37EE676AE6EE867A37EEC07A3A
:10853000C0ED027AA6EE870A80ED000A704700BF00
:10854000D0ED056AD0ED017A90ED007A90ED066AE3
:10855000D0ED025A90ED035A80ED050A66EEA77A37
:10856000C0ED066AE7EE007A90ED077AE5EE867ACE
:1085700090ED086AD0ED045A80ED087AE5EE477A6E
:10858000E5EEC67AB0EE670AC0ED077A704700BF25
:10859000D0ED057A90ED006A90ED067AD0ED035AA1
:1085A000E6EE007A90ED016AF0EE406AA6EE267AD9
:1085B000B0EE670AD0ED047A90ED026A67EEC07AF9
:1085C000A5EEC07AE6EE267A80ED057AC0ED067A51
:1085D000704703685A1C02601970704703690133C1
:1085E000012B03611CD0D0ED005AD0ED026A07EEDA
:1085F000903A30EE656AF8EEE77A86EE277A77EE03
:10860000257AB0EE667A30EE670AC0ED017AA6EE02
:10861000007AC0ED007A80ED037A80ED027A70472F
:10862000002380ED010A80ED000A83607047036833
:108630005A1C0260197070472DE9F347038A868936
:10864000B6B205460C461E404FF0004901F14C07FA
:1086500001F1340816B902B0BDE8F087B6FA86F326
:1086600029FA03F2D24391B2298216401B3B002C17
:1086700040D0042BEED8DFE803F039342E28030075
:10868000E368D5F82CA02BB19B681BB11FFA8AF1C7
:10869000201D9847636A33B19B6823B11FFA8AF1A2
:1086A00004F11C009847E36B2BB19B681BB11FFAC8
:1086B0008AF140469847636D002BCBD09B68002B16
:1086C000C8D01FFA8AF1384603E0E368696B5B683B
:1086D000201D9847BEE7636AA96B5B6804F11C0024
:1086E000F7E7E36BE96B5B684046F2E7636D296C83
:1086F0005B68E8E7042B06D8DFE803F00D0B0907F9
:108700000300EB6A0193019BA4E76B6BFAE7AB6B89
:10871000F8E7EB6BF6E72B6CF4E790F84820531C76
:108720000244DBB280F8483082F8341090F84920D7
:108730000AB1132B01D952F088B87047002280F893
:10874000492052F082B870B50F4E96F83038002BA1
:10875000FBD104464518AC4201D1002070BDD6F8CB
:108760002C3814F8011BF2180133C3F30A0382F802
:108770003118C6F82C38FFF73FFE0028EBD1012056
:108780000AF0BBFAF7E700BFF015002038B50C4639
:108790001146FFF76FFD48B1054D002A55F8C43C5E
:1087A00004DD2046FFF7CFFF55F8C43C38BD00BFBD
:1087B000E8260020F0B590F8CF5590F8CE1590F847
:1087C000D12590F8D03590F8CC7590F8CDC501EB57
:1087D00005218DB203EB022390F8D31590F8D22532
:1087E00085B002EB012207F01F06012192B29BB275
:1087F0008E4204468DF808708DF809C0ADF80A5015
:10880000ADF80C30ADF80E20C0F8402180F8111101
:1088100000F00C81022E00F01D81002E40F09B81A3
:10882000BCF1090F5ED8DFE81CF0B600F4005D0073
:10883000C8005D0057000A005D00A90076002E0AFE
:10884000022EADF806200BD0032E25D0012E49D1E3
:10885000D0F8EC351B68A0780DF10601984709E0C7
:10886000D0F8E43580789B6A0DF106019847467090
:10887000C4F8F005BDF80620002A47D0BDF80E3038
:10888000002B43D09A4228BF1A46ADF80620014675
:10889000204651F0DFFE39E0E9B2052922D8DFE8B1
:1088A00001F003070B0F1317D0F8EC355B68D2E724
:1088B000D0F8EC359B68CEE7D0F8EC35DB68CAE73A
:1088C000D0F8EC351B69C6E7D0F8EC355B69C2E738
:1088D000D0F8EC359B69BEE71A4303D190F812310A
:1088E000032B03D1204651F009FE0FE0016905F08A
:1088F0007F0680F814610B6865F30A121A430A6058
:1089000051F0BCFE2EB1022384F81231002005B0D4
:10891000F0BD0123F8E7E9B2904D012905F8C01C2C
:10892000E0D890F81231022B0FD0032BDAD1C1B965
:10893000022380F81231D0F8E43580F810115B681A
:108940009847204651F09AFEE0E70029F9D001212E
:10895000032380F8101180F81231204651F091FD68
:10896000EFE790F810110129EBD0D0F8E4355B68FF
:10897000984715F8C01C84F81011EEE7012AB1D110
:1089800090F81231022B04D0032BABD100F5887183
:108990007EE773497CE790F81231023B012BA1D8A6
:1089A0006E4B002243F8B82CD0F8182112B10222E5
:1089B00043F8B82C6B4902226AE7012D08D1C0F8B0
:1089C0001851D4F8E43502A99B6820469847B8E7C7
:1089D000022D9BD1DAB2002A98D102691B0A023B10
:1089E0005268032B03D8DFE803F00C0E10120123AA
:1089F00063F30612594B43F8B42C012384F8163163
:108A00009FE70223F4E70323F2E70423F0E70523BB
:108A1000EEE790F81231023B012B3FF663AF012DD8
:108A20007FF474AF0023C0F81831CAE790F8122120
:108A3000032A7FF457AFDBB2012B3FF653AFD0F8D8
:108A4000E43502A99B689847BDF80E30002B7FF4EF
:108A50005DAF76E707F06007202FD9B205D1D0F8D7
:108A6000E43502A99B68984750E7BCF1010F31D06B
:108A7000BCF1030F1ED0BCF1000F7FF447AF90F89C
:108A80001221022A5AD0032A7FF42CAF13F0800F50
:108A90004FF02802314B59D001F07F0102FB010158
:108AA00091F81E21002A4FD0012243F8B02C2E4904
:108AB0000222EDE690F81231022B3FD0032B7FF417
:108AC00011AF002D7FF47DAF4A063FF47AAF51F02D
:108AD000E4FC76E790F81221022A2FD0032A7FF4D3
:108AE00001AF002D7FF412AF11F07F003FF429AFEA
:108AF0005BB2002B4FF02802B5BF02FB004102FB26
:108B0000014101F58E7101F55D710022DB0F0870E6
:108B10008A704B7004EB8000C9786BB1826913686E
:108B200002396FF3555301298CBFC3F30071012142
:108B300061F31C73136044E7426DF0E74B063FF4AA
:108B4000E5AE51F0AAFCE1E60022AEE702FB01012E
:108B500091F87623A6E707F08001F2E7E8260020E7
:108B60002C260020302600203826002010B5044690
:108B700071BB90F81131032B1BD1D0F89023D0F8A2
:108B80007C339A4217D9C178012908BFD0F88013E5
:108B9000A2EB030204BFC918C0F88013934228BF98
:108BA0001346C0F890239BB2D0F88023002151F0E7
:108BB00015FE002010BDD0F8E4351B6923B190F8F4
:108BC0001221032A00D19847204651F057FDF0E7C3
:108BD000D0F8E4359B69002BEBD090F81221032AE2
:108BE000E7D19847E5E770B50A7812F060040646C9
:108BF0000D462AD0202C2FD1CC884B78FCB1120600
:108C00000CD51F4922461846FFF7B4FBEA881C49D9
:108C1000304651F01FFD0024204670BD194A1360F4
:108C2000194A0323C2F80C4880F81131C0E9E44422
:108C3000234602F50162002151F0D0FDEBE702224C
:108C400011441846FFF796FBE6E74B780A2B08D04D
:108C50000B2B0BD0062BDFD1304651F04FFC0224FA
:108C6000DAE70A49012251F0F5FCD5E78B781BB908
:108C7000074B43F8AC4CCFE751F040FCCCE700BFCA
:108C8000001E002000000020F01500203C260020DF
:108C9000E826002010B5282303FB0101074AB1F89C
:108CA0008C1304461046FFF7BAFB2046034A4023C4
:108CB000012151F093FD002010BD00BF402600208F
:108CC000002310B519460446402251F025FC4022ED
:108CD00080212046002351F01FFC012384F812312B
:108CE000D4F8E835A0785B689847002010BD38B507
:108CF000402204460223812151F00EFC204602232B
:108D00004022012151F008FC204603230822822141
:108D100051F002FC084B0222002583F84B2083F817
:108D20004C50FFF713FB01212046044A402351F029
:108D300055FD284638BD00BF000000204026002019
:108D400038B50122044640F20113A0F84431012550
:108D5000114651F061FD29462046A4F89C5300229B
:108D600051F05AFD4FF48173A4F86C3120462A4625
:108D7000022151F051FDFFF7F5FA002038BD38B55A
:108D8000254C94F83028012A034633D1234850F863
:108D9000682C1AB984F83028002038BD402AD4F84D
:108DA000281819D9403A01F1400540F8682CC4F858
:108DB000285840221A4810FA81F1C3E9541140F2B0
:108DC00001100021C3E95621A3F8440103F5A27163
:108DD000184651F06AFCDFE702EB0105C4F8285899
:108DE0004FF0000540F8685C0ABF022092B284F898
:108DF0003008DFE7022ACFD1002540F20112C0E996
:108E00005455C0E95655A0F8442100F5A27151F01F
:108E10004CFC84F83058BFE7F0150020E82600200D
:108E2000211E002038B52A4C54F8643C0F2B03F166
:108E3000010203D044F8642C002038BD254A0023E9
:108E400044F8643C92F83038002BF5D1D2F8281859
:108E5000B1F5006F08BFC2F82838D2F82818D2F848
:108E60002C38994203D1002382F83038E4E78CBFD4
:108E7000C1F500635B1A402B1BD9403B01F1400553
:108E800044F8683C012382F83038C2F8285840235F
:108E9000114A12FA81F140F20112A0F84421002295
:108EA000C0E95411C0E9563200F5A27151F0FDFB42
:108EB000C2E701EB0305C2F828584FF0000544F85B
:108EC000685C0EBF022401249BB282F83048DFE7C1
:108ED000E8260020F0150020211E002008B50248D9
:108EE0004FF009FC014808BDEDA2060888260020C5
:108EF00008B502484FF0FFFB014808BDF9A206087B
:108F00008826002008B502484FF0F5FB014808BD4F
:108F1000FEA206088826002008B502484FF0EBFBA9
:108F2000014808BD08A306088826002008B50248A5
:108F30004FF0E1FB014808BD13A306088826002076
:108F40000068F022FF2107F075BE0068B422FF21FF
:108F500007F070BECA4341EA02120068D2B2D221C1
:108F600007F068BE0A460068A52107F063BE5521D8
:108F7000F8E700689622FF2107F05CBE0A46006809
:108F8000872107F057BEC90101F0800200687821EF
:108F900007F050BEF8B504460E461546071D20687A
:108FA0003A46FF2108F0D8FB30B116B12379DB0730
:108FB000F5D40DB123792B70F8BD00220121E9E72A
:108FC00010B50446FFF7C1FF18B12046BDE81040B8
:108FD000F3E710BD10B50446FFF7C4FF18B12046F3
:108FE000BDE81040E9E710BD73B50546CDE90023A3
:108FF000FFF7E6FFA8B12846FFF7B9FF88B128467A
:10900000FFF7DBFF68B16E46082416F8011B2846FF
:10901000FFF7E0FF28B1013C14F0FF04F5D102B0E6
:1090200070BD0020FBE7CC21D4E770B506460C46A6
:109030008D18AC4201D1012006E014F8011B304626
:10904000FFF7C8FF0028F4D170BD38B505461446B7
:10905000FFF794FF2846FFF7B0FF20B11CB12B7932
:10906000C3F34013237038BD10B50446FFF7A8FFC3
:1090700038B12046FFF7D7FF18B12046BDE81040B1
:109080009BE7002010BDC90138B501F080010446FE
:109090001546FFF778FF08B9002038BD00220121EE
:1090A0002046FFF777FF0028F6D023795B092B7065
:1090B000F3E710B5021D0446FF21006808F04CFBE1
:1090C00018B12079C04300F0010010BD38B5044646
:1090D000154600680A46E12107F0ACFD30B1206872
:1090E0002A46FF21BDE8384008F036BB38BD0A46A5
:1090F000C321EBE738B5021D0D46F0210446FFF70A
:10910000E5FF08B123792B7038BD0A46E121DDE780
:1091100038B504460D46FFF72CFF40B12046FFF757
:109120004CFF20B129462046BDE83840EDE700203D
:1091300038BD70B506460C468D18AC4201D10120F1
:1091400006E021463046FFF7E3FF01340028F4D162
:1091500070BD024BD3F8A00007F017BCE826002032
:109160000E49D1F8883043F47003C1F888300C4BB5
:109170001A68002042F001021A6098601A6822F012
:10918000847222F480321A60064A5A601A6822F405
:1091900080221A60D860044B8B60704700ED00E0BD
:1091A00000380240103000240000000870472DE90C
:1091B000F041476906468846002F59D10368C3F33A
:1091C0000D0515B3D8F800803568FFF701F80928B8
:1091D00040F08780444C236923F440732361236962
:1091E00043F400732361236943F001032361C5F84D
:1091F0000080FEF7EDFF2369092823F001032361B6
:109200006FD133680433336032E0384A934229D354
:1092100002F58042934224D302F5804293422AD33E
:10922000334A934229D902F58032934227D902F575
:109230000032934225D902F50032934223D902F538
:109240000032934221D902F5003293421FD902F530
:10925000802293421DD9B3F1016F1CD305200AF07F
:1092600097F80825FEF7B4FF092816D04FF0FF370E
:109270003846BDE8F0811025F4E71825F2E72025EF
:10928000F0E72825EEE73025ECE73825EAE740252A
:10929000E8E74825E6E75825E4E7134C236923F47B
:1092A00040732361236943F400732361236923F02E
:1092B000F803236123691D4345F0020525612369F5
:1092C00043F480332361FEF783FF236923F0020315
:1092D00023612369092823F0F80323613FF472AF67
:1092E000C4E76FF00107C3E7003C024000400008FC
:1092F000FFFF0008002808DB4209012300F01F00DF
:1093000003FA00F0014B43F82200704700E100E04F
:109310000028ACBF00F16040064B4FEA0111ACBF22
:1093200000F5614000F00F00C9B2B4BF195480F8D5
:109330000013704714ED00E02DE9F04798463C4BD0
:10934000914603EB80020546946F002C45D098337C
:10935000636004F13E03A36104F59F73E3614FF47E
:109360008073C4E90433236894F83D00E160A3638B
:1093700006F08EF9064694F8440294F83CA0271DA6
:1093800008B14FF0D1FC94F8450208B14FF0CCFC85
:10939000D4F840321BB1274A116B0B43136318F00A
:1093A000080F23D00135EDB21EB14FF4E163F38015
:1093B000357218F0100F94F8462211D00221304671
:1093C00006F078F894F94702D4F84812FFF7A0FFA6
:1093D00094F94702FFF78EFF3C462046BDE8F08730
:1093E00018F0200F14BF12213221E8E719F0020F04
:1093F0000CD06B1CDBB21EB14FF4A162F280337251
:1094000094F846220221304606F054F819F0010F74
:10941000D8D0504606F03CF90135EDB218B14FF402
:10942000C163C380057294F846220221C8E700BFD9
:1094300090140608003802400148FEF71EBE00BF27
:10944000640000200148FEF718BE00BFB0020020F3
:1094500070B5002828D04C684CB942681568567918
:10946000AB8902229BB2B24023EA0203AB818A6835
:109470003AB943681D68AB8923F001031B041B0C38
:10948000AB81816044B14468216864798D8902238D
:10949000A3402B439BB28B8132B143681A689389F6
:1094A0009BB243F00103938170BD0B4B30B51A465C
:1094B00000241D79854208D1DD68294203D014209B
:1094C00000FB042030BD0029F9D001340B2C03F13E
:1094D0001403EED10020F5E7F804002038B5036846
:1094E0001B681C68254B03F2D45393ED007A07EEFA
:1094F000902AB8EE477AF8EE677A013987EE270AA4
:109500008DB2DFED1F7A30EE270A54F0FFFC1D4AC2
:1095100023880138944280B29BB212D002F5806257
:1095200094420ED0B4F1804F0BD0A2F58032944219
:1095300007D002F58062944203D002F58062944223
:1095400002D123F070039BB20F4A944206D002F579
:10955000806294421CBF23F440739BB22380094B6A
:10956000E5629C42208503D003F580639C4201D1D3
:10957000002323860123A38238BD00BF0000002002
:109580000AD7233C00000140001000402DE9F043C1
:109590004568A87910F0040300F002020BD0002007
:1095A00017468046042406466B79032B49D8DFE82A
:1095B00003F0094A89C990464FF480701F461C4643
:1095C0000126F1E72D682B8C23F001031B041B0CF3
:1095D0002B84B5F820C0B5F804902B8B23F07303CF
:1095E0001B041B0C43F0600E2CF0020C6E4B4FEA78
:1095F0000C4C4FEA1C4C48EA06069D421FFA89F9BA
:109600004CEA060C03D003F580639D420AD14FF665
:10961000F3730CEA03033B4329F4407943EA040C57
:1096200040EA0909A5F80490A5F818E06963A5F8CF
:1096300020C02B8B23F008031B041B0C43F00803F2
:109640002B83BDE8F0832D682B8C23F010031B04C3
:109650001B0C2B842A8CB5F804E0B5F818C0524BCB
:109660002CF4E64C22F020024FEA0C4C12044FEA94
:109670001C4C120C48EA06069D421FFA8EFE4CF462
:10968000C04C42EA061203D003F580639D420BD121
:1096900022F0800242EA071222F040022EF4406ECD
:1096A00042EA04124EEA800EA5F804E0A5F818C0BC
:1096B000A9632A842B8B23F400631B041B0C43F443
:1096C0000063BDE72D682B8C23F480731B041B0CF7
:1096D0002B842A8CB5F804E0B5F81CC022F4007382
:1096E0002CF0730C304A4FEA0C4C1B044FEA1C4C14
:1096F0001B0C48EA060695421FFA8EFE4CF0600CE1
:1097000043EA062303D002F5806295420BD123F48D
:10971000006343EA072323F480632EF4405E43EAA8
:1097200004234EEA001EA5F804E0A5F81CC0E96376
:109730002B84AB8B23F008031B041B0C43F00803A2
:10974000AB837EE72C68238C23F480531B041B0C13
:109750002384258CA288A38B25F400552D0448EA88
:1097600006062D0C23F4E64345EA06350E4E1B048F
:109770001B0CB44292B243F4C04303D006F580669A
:10978000B44203D122F4804242EA8012A280A38331
:1097900021642584A38B23F400631B041B0C43F476
:1097A0000063A3834DE700BF0000014043685A797E
:1097B000032A0FD8DFE802F00205080B18683430DE
:1097C000704718683830704718683C307047186820
:1097D000403070470020704710B543681A685879C8
:1097E000084B0344012093F8C840138CA0409BB25F
:1097F00023EA00031384138CA140194389B2118416
:1098000010BD00BF90140608F0B5EFF311841023CB
:1098100083F31288C568AA68136823F001031360F4
:10982000426816685779114AB38902EB47029BB226
:10983000B2F8702023EA02032A69B3811F2A4FF08D
:1098400020036D6885BF203A93409340EB6098BF3A
:10985000AB60E3B283F31188C3689B6859601A68F0
:1098600042F001021A6001230374F0BD901406084F
:109870000268137D012B04BF0223137592F82C108C
:109880000CBF4FF400730023012904BF022182F8AA
:109890002C1092F8441008BF43F48063012904BFE0
:1098A000022182F8441092F85C1008BF43F4006370
:1098B00001290DD1022182F85C1043F480534268E3
:1098C000116800224A628A8992B213438B8101E0B7
:1098D000002BF4D17047034B0348D3F8A410FEF7D4
:1098E000ABBE00BFE82600200000014010B5064CCA
:1098F0000648D4F8A410FEF79FFED4F8C41004481C
:10990000BDE81040FEF798BEE826002000000140A8
:109910000040014010B5064C0648D4F8A410FEF7EC
:109920008BFED4F8C8100448BDE81040FEF784BE92
:10993000E8260020000001400044014010B5064C1C
:109940000648D4F8A410FEF777FED4F8CC100448EB
:10995000BDE81040FEF770BEE82600200000014080
:1099600000480140034B4FF08040D3F8A810FEF7A9
:1099700063BE00BFE8260020024B0348D3F8AC10BA
:10998000FEF75ABEE826002000040040024B0348C0
:10999000D3F8B010FEF750BEE826002000080040C3
:1099A000024B0348D3F8B410FEF746BEE826002069
:1099B000000C00400348D0F8E43513B100F5BB605B
:1099C00018477047000000200348D0F8043613B150
:1099D00000F5BF6018477047000000200348D0F82A
:1099E000243613B100F5C36018477047000000200B
:1099F0000348D0F8443613B100F5C76018477047E4
:109A0000000000200348D0F8643613B100F5CB60A5
:109A100018477047000000200348D0F8843613B17F
:109A200000F5CF6018477047000000200348D0F8C9
:109A3000A43613B100F5D36018477047000000202A
:109A40000348D0F8C43613B100F5D7601847704703
:109A5000000000200348D0F8E43613B100F5DB60C5
:109A600018477047000000200348D0F8043713B1AE
:109A700000F5DF6018477047000000200348D0F869
:109A8000243713B100F5E360184770470000002049
:109A90000348D0F8443713B100F5E7601847704722
:109AA000000000200348D0F8643713B100F5EB60E4
:109AB00018477047000000200348D0F8843713B1DE
:109AC00000F5EF6018477047000000200348D0F809
:109AD000A43713B100F5F360184770470000002069
:109AE0000348D0F8C43713B100F5F7601847704742
:109AF00000000020036823F00103036000230360DB
:109B000043608360C3600361212343612A4B984211
:109B100003D13D2243F8082C7047284B984204D1CA
:109B20004FF4746243F8202C7047254B984204D1BF
:109B30004FF4741243F8382C7047224B984204D1EA
:109B40004FF0746243F8502C70471F4B984203D17A
:109B50001E4A43F8642C70471D4B984203D11D4A9E
:109B600043F87C2C70471C4B984203D11B4A43F8A6
:109B7000942C70471A4B984204D14FF03D5243F851
:109B8000AC2C17E0174B9842C3D0174B9842C7D064
:109B9000164B9842CCD0164B9842D1D0154B9842D8
:109BA000D6D0154B9842DAD0144B9842DED0144BE5
:109BB0009842E2D0704700BF106002402860024027
:109BC0004060024058600240706002403D0000204A
:109BD00088600240400F0020A060024000003D204D
:109BE000B8600240106402402864024040640240B1
:109BF000586402407064024088640240A0640240DD
:109C0000B86402402DE9F0410022012603250B68CB
:109C100006FA02FC3CEA030331D10368540005FA5A
:109C200004FE23EA0E0303600B79D0F800806FEA8C
:109C30000E0703FA04FE013B4EEA080E012BC0F8A2
:109C400000E011D883681F4087604B798768A34084
:109C50003B438360436823EA0C0343608B79476886
:109C600093409BB23B434360C36805FA04F723EA81
:109C70000703C360CB79C768A3403B43C36001328D
:109C8000102AC4D1BDE8F081F7B51C2005F000FD15
:109C90001121044605F0E8FB204605F0D7FBC8205B
:109CA00009F02BF8204605F0CCFB1B2005F0F0FC5A
:109CB00020B140F21113C3800023037224B140F29B
:109CC0001123E38000232372C74B502283F84323E0
:109CD0000822C3F88820BFF34F8FBFF36F8FC34CA8
:109CE000C34D236B43F0010323634FF4C05040F294
:109CF0000233CDE90003BF486946FFF783FF436A9B
:109D000023F470434362436A43F420434362436A4B
:109D100023F470234362436A43F420234362636C59
:109D200043F480436364636B43F080036363B24B2B
:109D3000B24C01205861B24BC4F8C03603F12C027A
:109D40004833C4F8C836AF4BC4F8C426C4E9375307
:109D5000022384F8E4304FF0A043C4F8E83003F560
:109D60000063C4F8EC3003F58073C4F8F43003F5F5
:109D70000073C4F83031A3F5F073C4F8F83003F57C
:109D80000073C4F83431A3F5F073C4F8FC3003F564
:109D90000073C4F83831A3F5F073C4F8003103F54B
:109DA0000073C4F83C31A3F5EC63C4F8F0304033E1
:109DB000C4F8A831C03384F8E700C4F86C3120330C
:109DC000C4F870312033C4F874312033C4F87831CA
:109DD0002033C4F87C312033C4F880312033C4F8F8
:109DE00084312033C4F8883103F52263C4F8AC31E0
:109DF00003F58053C4F8B03103F58053C4F8B4318F
:109E000003F58053C4F8B8314FF05023C4F8BC3187
:109E100003F58053C4F8C03103F58053C4F8C4314E
:109E200003F58053C4F8C831A3F5E4430022C4F815
:109E3000E83104F1DC0384F8EE0184F8F0211946DE
:109E40001546402681F81C21A1F822210132042A5E
:109E5000C1E9496581F81D0181F81F51C1F83051F0
:109E600001F12801EED100221146402083F874232D
:109E7000A3F87A230132042AC3E9DF0183F87513BA
:109E800083F87713C3F8881303F12803EED14FF05A
:109E9000A04300259A6822F001029A60DA6842F035
:109EA0004002DA604FF0B0F894F8E53094F8DF2023
:109EB0005B1B18BF01231B0143F0210363F317450C
:109EC000D4F8E830012A9D6307D19A6822F03E0158
:109ED00041F02A0161F307029A60DA68C2F3076170
:109EE00021F0600141F0400161F31F62DA60D4F8B3
:109EF000E82100201060D4F8EC20116860F3CC2138
:109F0000116094F8E710012912D1116841F00301A2
:109F1000116080225A6202F580029A6202F14012B8
:109F2000C3F804214FF4A072C3F80821C3F80C2130
:109F300010204FF04BF800230093009B43F01003D8
:109F40000093D4F8E830009A1A612F4A19690091F9
:109F5000013A02D00099C906F8D4D4F8EC1094F86C
:109F6000DD502A4E00224FF0FF300A6117464A6149
:109F70004FF0FF0C8861CA61AA4251D30022244EDF
:109F800017464FF0FF0C95425CD80A6942F4807284
:109F90000A6194F8DF20012A04BF1E4808630021EB
:109FA00099614FF0FF306FF08041596158605961FD
:109FB00019499961B2FA82F21849520941EA02122A
:109FC00099690A439A619A6842F001029A60D4F84A
:109FD000C4361B689847044B502283F84323082259
:109FE0009A6003B0F0BD00BF00E100E0003802401D
:109FF0000804010000000240003C0140E826002067
:10A00000D807002040004001410D0300DC2700205C
:10A0100018280020030181000008008008383C0057
:10A0200056F8040BD0F800E0BEF1000FACBF4FF0C3
:10A03000000E4FF0904EC0F800E001320761C0F80A
:10A0400008C099E756F8040BD0F800E0BEF1000F05
:10A05000ACBF4FF0000E4FF0904EC0F800E0013260
:10A060000761C0F808C08EE7204A936803F00C032C
:10A07000042B10B520D0082B20D01D4B1B4C0360A7
:10A08000A3681C4AC3F30313134493F83C180368F2
:10A09000CB404360A168C1F38221114491F83C1880
:10A0A00023FA01F18160A168C1F342310A4492F8B8
:10A0B0003C28D340C36010BD0F4BDFE753685168A5
:10A0C00013F4800F01F03F01536814BF0A4A084A95
:10A0D000B2FBF1F1054A5268C2F30142C3F388139F
:10A0E00001324B435200B3FBF2F3C7E700380240A2
:10A0F0000024F4000000002000127A00F0B5446B48
:10A100008668A38923F400531B041B0CA381827966
:10A11000278A0546BFB2100312F0040F4FEA02214E
:10A1200000F400506A7927F4405740EA0700208283
:10A1300014BF4FF4805C4FF0000C12F0010F0CBF05
:10A14000002304239207A28922F4B05201F4806113
:10A1500022F00C0248BF43F0080341EA0C0112044C
:10A160000B43120C1A43A281A38A23F440731B04ED
:10A170001B0C85B0A3826846FFF776FF214B9C42FB
:10A1800003D003F580639C423AD1039BA289192135
:10A19000170401FB03F34FF064014CBF7600B600D7
:10A1A000B3FBF6F3B3FBF1F001FB10330201A0891E
:10A1B00000044BBFDB001B01323332334BBFB3FB18
:10A1C000F1F3B3FBF1F303F0070303F00F031343C1
:10A1D0009BB223816A6BAB7913F0080F938A0BBF94
:10A1E00023F008039BB21B0443F0080308BF1B0CB9
:10A1F000938293899BB243F40053938105B0F0BDE1
:10A20000029BC3E7001001402DE9F8431E46204B96
:10A210009DF820509DF824709842894690462CD194
:10A220003B462A4631460020FFF786F804460020C8
:10A23000C4E90700C4E90900C4E90B986571A66088
:10A24000A7712046FFF75AFFEA0707D5636B4FF661
:10A25000DF721A80DA6842F02002DA60626BAB07C4
:10A2600042BFD36843F08003D36093899BB243F429
:10A27000005393812046BDE8F883064B984204D1F1
:10A280003B462A4631460120CEE70024F2E700BFD4
:10A29000001001400044004081602FE741712DE72C
:10A2A0002DE9F043654F07EBC00985B005464FEA3D
:10A2B000C00899F8500805F0EBF9064699F85108DE
:10A2C00005F0E6F9044699F852084EF02DFD6B1C96
:10A2D000DBB21EB140F60E12F28033721CB140F6B2
:10A2E0000E22E280237204223A21304605F0E2F881
:10A2F000204604223A2105F0DDF807EB0803D3F8E5
:10A300004C484F4B9C4263D103F5F2331A6A42F436
:10A3100000121A621A6A22F400121A62474497F86D
:10A320005338022B6ED0032B6ED0464E464A012B7B
:10A3300008BF1646A78827F03F0768463F04FFF787
:10A3400093FE3F0C029A414BB2FBF3F398B20743E2
:10A35000A780218821F001010904090C21803C49D2
:10A360008E4253D13B4BB2FBF3F2013092B2042A3E
:10A3700080B238BF04222084A28323889BB243F09A
:10A3800001032380238823F4816323F002031B0449
:10A390001B0C43F4806323804FF480432381238884
:10A3A00023F080031B041B0C238023889BB243F003
:10A3B00001032380284B03EB4513012283F8D126A8
:10A3C000002283F8D05683F8D22605B0BDE8F0838A
:10A3D000224B9C4209D103F5F0331A6A42F4800201
:10A3E0001A621A6A22F4800297E71D4B9C4295D1AB
:10A3F00003F5EE331A6A42F400021A621A6A22F472
:10A4000000028AE7124E95E7124E93E706EB4606E6
:10A41000B2FBF6F291B2C2F30B020AB941F00101AC
:10A4200041F400424FF496714B434FF47A71B3FB01
:10A43000F1F301339BB223849EE700BF00000020AC
:10A4400000540040801A060000350C0040420F0006
:10A45000A0860100400D0300E826002000580040BF
:10A46000005C00402DE9F047B84E440106EB40196E
:10A4700008F004FC99F9D026B54B8846D10003EBCF
:10A48000C2020746D2F84C5899F8D226013A142A4B
:10A4900000F28380DFE812F079008900A100BA00A1
:10A4A000C700D100DC00F40001010A0117016801B6
:10A4B0008601B8010F02220234023F025F028202CB
:10A4C00015005F184FF0090A97F8500805F0E0F8FA
:10A4D000054697F8510805F0DBF8B6F83037013338
:10A4E0009BB207462846A6F8303704F0AAFF384644
:10A4F00004F0A7FF1121284604F0B6FF11213846C9
:10A5000004F0B2FF4FF0650803E00520002108F0D9
:10A51000E3FB284604F084FF10B9B8F10108F4D138
:10A52000284604F093FF0021052008F0D5FB2846BB
:10A5300004F087FF0520002108F0CEFBBAF1010AE4
:10A54000E0D1284604F082FF0021052008F0C4FB7A
:10A55000384604F07BFF0021052008F0BDFB2846AB
:10A5600004F06FFF0520002108F0B6FB384604F028
:10A5700068FF331993F9D006431C01D0FFF790FE12
:10A580003319002283F8D22607E02B8813F40073D6
:10A5900040F0D081321982F8D236331993F8D2368E
:10A5A000002B7FF465AFBDE8F0872B8823F40063B0
:10A5B0001B041B0C2B802B889BB243F480632B80E5
:10A5C0002B889BB243F480732B803319032283F8CA
:10A5D000D226604B2344C3E902785F492846FDF741
:10A5E00008FE002800F0A681331993F8E2265AB934
:10A5F00093F8E326FF2A04D193F8E0260AB10A2251
:10A60000C0E733190422BDE70F22BBE7321992F8E5
:10A61000E13603F0FE032B82052382F8D2364D4B40
:10A620002344C3E902784D492846FDF7E2FD00289E
:10A6300000F0788133190622A4E7331993F8E32652
:10A640002A82072283F8D226424B2344C3E90278A8
:10A6500043492846FDF7CDFD002800F063813219FB
:10A66000D2F8E43653B92B889BB243F400732B80A5
:10A67000384B2344C3E9027801238CE708238AE797
:10A680002B889BB243F480732B803319092283F803
:10A69000D226304B2344C3E902782F492846FDF7E0
:10A6A000A8FD002800F046813319A8E7321992F876
:10A6B000E13643F001032B820B2382F8D236254B7F
:10A6C0002344C3E9027827492846FDF792FD002874
:10A6D00000F028813219D2F8E436012B1BD12B88E7
:10A6E00023F480631B041B0C2B80EFF311811023D8
:10A6F00083F312882B8B2B889BB243F400732B803F
:10A70000CBB283F311880C2382F8D236114B234449
:10A71000C3E9027841E7022B15D12B889BB243F4A1
:10A7200000632B80EFF31181102383F312882B8BAE
:10A730002B8823F480631B041B0C2B80CBB283F388
:10A7400011880D23E0E72B8B0E23DDE7E8260020A0
:10A7500000000020B82D0020010003008200070047
:10A76000840007000200030094492846FDF74CFDD1
:10A77000934B002800F0DF8031192344D1F8E826FC
:10A78000501CC1F8E806288A1070D1F8E426013A76
:10A79000C1F8E4260122C3E9027881F8EC2681F8A9
:10A7A000D226FAE687492846FDF72EFD844B00287D
:10A7B00000F0C180EFF3118C102282F312882A88F6
:10A7C000301992B2D0F8E81642F400722A804A1C7E
:10A7D000C0F8E8262A8A0A705FFA8CF282F31188A0
:10A7E000D0F8E826511CC0F8E816298A11706FF0DD
:10A7F0000102C0F8E42623440122C3E9027880F86C
:10A80000EC2680F8D226C8E66E492846FDF7FCFC07
:10A810006B4B002800F08F803219D2F8E416032920
:10A820002AD1298821F480610904090C2980EFF3D9
:10A83000118C102181F31288D2F8E806411CC2F86D
:10A84000E816298A0170298889B241F400712980AB
:10A850005FFA8CF181F31188D2F8E816481CC2F82F
:10A86000E806288A0870D2F8E4160239C2F8E4161D
:10A870000C2182F8D2164AE702290FD8298821F440
:10A8800080610904090C2980298889B241F400718A
:10A890002980298A002182F8EC16EAE6D2F8E81627
:10A8A000481CC2F8E806288A0870D2F8E416013974
:10A8B000C2F8E4162BE72B8823F4806332191B04BB
:10A8C0001B0C2B8092F8E13603F0FE032B82102341
:10A8D00082F8D2363A4B2344C3E902783A492846F3
:10A8E000FDF787FCF0B1331993F8E326FF2A04D172
:10A8F00093F8E0260AB1132244E63319112241E607
:10A90000331993F8E3262A82122283F8D2262C4B9D
:10A910002344C3E902782D492846FDF76AFC08B1B3
:10A920003319E8E72A492846FDF76EFC10B13319C0
:10A93000142227E6224B2344D3E9020142F210738A
:10A94000381A68EB0108984278F10003FFF425AE4D
:10A950003319152216E63119194BD1F8E4268AB1BC
:10A96000D1F8E806234410F801CBA5F810C0013A4D
:10A97000C3E90278C1F8E806C1F8E426122381F899
:10A98000D2360AE62A8892B2234442F400722A8020
:10A99000C3E90278012381F8EC36F0E72B889BB2FB
:10A9A00043F400732B804FF6FF33AB82044B2344F8
:10A9B000C3E9027801223319E4E500BF400000102A
:10A9C000B82D00200400001082000700840007005A
:10A9D0000004001038B5114C04EB401494F8D15623
:10A9E000D5B1C4F8E436049BC4F8E836002384F8F3
:10A9F000EC360223490084F8E32684F8D23601229B
:10AA00009DF8143084F8E11684F8E22684F8E036E4
:10AA1000FFF728FD94F8EC56284638BDE8260020BC
:10AA200038B5114C04EB401494F8D156CDB1C4F8AC
:10AA3000E436049BC4F8E8360223490084F8E32690
:10AA400084F8D23600229DF8143084F8E11684F898
:10AA5000E22684F8EC2684F8E036FFF703FD94F84C
:10AA6000EC56284638BD00BFE8260020F0B587B078
:10AA7000002300930193744B1A6842F480321A60E9
:10AA80001A6802F400320192009A01320092019A8F
:10AA90001AB9009AB2F5A04FF2D11B6813F4003333
:10AAA00018BF01230193019B012B40F0B180664B3D
:10AAB00066491A6C42F080521A640A6842F44042B5
:10AAC0000A609A689A609A689A609A6842F480521A
:10AAD0009A605F4A5A601A6842F080721A601A6877
:10AAE0009201FCD55B4A40F2027111609A6822F033
:10AAF00003029A609A6842F002029A60524A93688E
:10AB000003F00C03082BFAD19368534C03F00C03A9
:10AB1000042B7FD0082B7FD0504BC4F8D4354A4B40
:10AB20004F4D9A684F48C2F303122244002692F810
:10AB30006418D4F8D425CA40C4F8D4254A4AEA6037
:10AB40005A6F4A4AAA605A6B22F080025A635A6FBF
:10AB500042F080725A67196B454A0A431A635A6B6E
:10AB60005A631A6C42F0875242F4F61242F41F62A2
:10AB700042F00F021A64596C3E4A0A435A6402A911
:10AB800048F2FF73CDE902364FF6FF77FFF73AF848
:10AB900000F580600297FFF735F800F580600297B6
:10ABA000FFF730F800F58060FFF72CF800F58060C3
:10ABB000FFF728F80846FFF757FA029B2E4AB3FB27
:10ABC000F2F32E4AC2F83437D5F8FC302C4A43F061
:10ABD0008073C5F8FC302B4BC3F8B02F5E601A6849
:10ABE00042F001021A60D4F8D4354FF47A72B3FB04
:10ABF000F2F3013BB3F1807F08D24FF0E0225361C2
:10AC0000F02385F8233007239661136107B0F0BD68
:10AC100000BFFDE71C4B80E75368516813F4800FB9
:10AC200001F03F01536814BF174A0C4AB2FBF1F11F
:10AC3000054A5268C2F30142C3F3881301324B4301
:10AC40005200B3FBF2F368E70038024000700040A6
:10AC500008304004003C0240000000200024F400C2
:10AC600000ED00E0000002400003FA0500000008CB
:10AC70001F9067003357070040420F00E82600206E
:10AC800055CEACC5001000E000127A0082B000235F
:10AC90000193054B0193019B03EB80000190019B05
:10ACA000196002B0704700BF50280040436D064A4B
:10ACB0001A61C278012A06D100F2CC5058611A6894
:10ACC0004FF080221A6070471800086038B50446BB
:10ACD00000296FD190F81131022B2AD1D0F83821F8
:10ACE000D0F824118A4232D9C378012B04BFD0F89E
:10ACF00028315B18A2EB010208BFC0F828314FF4DD
:10AD00008071D0F82831C0F83821002592B2A0F81F
:10AD10001C11C0F82C31C0F83451C0F8302100F5B6
:10AD20008E714FF045FC2B462A46294620464FF0AF
:10AD300055FD94F81631012B07D1244A236952F8A6
:10AD4000B42C5A60002384F81631002038BDD0F8A6
:10AD50003C31B3FBF1F501FB1535A5B9994212D889
:10AD6000D0F8402193420ED24FF48073C0E94A5587
:10AD7000C0E94C55A0F81C3100F58E714FF018FC5D
:10AD8000C4F84051CFE7D4F8E435DB682BB194F830
:10AD90001221032A01D120469847052384F8113156
:10ADA000002320461A4619464FF018FD2046FFF7AB
:10ADB0007DFFBEE7D0F8E4355B69002BC5D090F885
:10ADC0001221032AC1D19847BFE700BFE82600201F
:10ADD00070477047704710B5114C94F8E630CBB10E
:10ADE0004FF0E022D2F8103D23F00603C2F8103DE8
:10ADF000FEF7B6F994F8E63063B1D4F8EC309B680E
:10AE0000DB0707D5D4F8E821136823F0030161F3C9
:10AE100007031360034B4FF480225A6110BD00BF3B
:10AE2000E8260020003C01402DE9F04F954CD4F875
:10AE3000E8305A69D0078DB000F1A1825A699B6948
:10AE40001340019300F09B82C3F307430293019BDD
:10AE5000190311D5D4F8EC30DFF834929E69DB6920
:10AE600004F1DC0B1E40360C04F598774FF0000817
:10AE7000DA46002E40F01281029B5A070FD5D4F813
:10AE8000EC30814E9F69DB691F40BFB2A6F1180507
:10AE90004FF00009A6F1F408002F40F04481019B17
:10AEA0009DF80470980741BF764BD3F8E830022232
:10AEB0005A61019B002B1BDA724D95F8E6303BB1CD
:10AEC000D5F8E821136823F0030161F30703136049
:10AED000D5F8EC206D48536823F0010353606C4BA8
:10AEE000D3F88C389847D5F8E8304FF000425A61D3
:10AEF000019B1905C3F3072631D5624D00238DF858
:10AF00001F3095F8EE318DF81F30614B05F1DC00F4
:10AF1000D3F888389847D5F8E820D5F8EC304FF4C6
:10AF200000619B68516195F8E620C2B1DA0716D539
:10AF300095F8F131012B12D19DF81F30032B0ED162
:10AF4000D5F8E8311A6842F001021A601A6842F036
:10AF500003021A604F4A136943F0060313613B076B
:10AF60000AD5484D4A4B05F1DC00D3F880389847A4
:10AF7000D5F8E83008225A61FD0615D5414BD3F8C3
:10AF8000E800826922F010028261026AC2F3434142
:10AF9000022902F00F0500F08381062900F0A78145
:10AFA000836943F010038361F00634D5354DD5F83D
:10AFB000EC205368002723F00103536038464EF01D
:10AFC00005F8B84695F8DD003B46F435FF2183428D
:10AFD000C0F09B81D4F8EC302C484FF0FF329A61DE
:10AFE0004FF00112DA610B2262F3070762F30708E0
:10AFF0005F61C3F810801A686FF30A121A60FFF7D6
:10B0000055FED4F8E83021484FF480525A61204B65
:10B01000D3F884389847B10640F19381194CD4F89D
:10B02000EC30D4F8F40099680268C1F341010229B8
:10B0300006BF032161F30A026FF30A0202605A6835
:10B0400042F480725A6008A8FFF70EF8D4F8E810AE
:10B05000D4F8EC00CB68099A6FF38D23CB60856838
:10B060000D48C5F34105284490F8CC00032840F072
:10B070005381002284F8DE204FF40072A4F8E0200F
:10B08000092258E1E8260020DC270020C427002000
:10B090000000002000ED00E090140608F2073BD508
:10B0A0005FFA88F104EB8103D3F830319D68D4F85E
:10B0B000EC305B691D40EB0720D594F8DF003B685E
:10B0C0000125A8429D6007D11869DBF87C33C0F3E5
:10B0D00012001B1ACBF88C33D9F8743850469847B5
:10B0E00094F8DF30012B09D1B8F1000F06D194F8A4
:10B0F000ED31052B02D15046FFF7D8FDA80742BF1E
:10B100003B6802259D60290706D5D9F87C38504652
:10B1100098473B6808229A6008F1010876080437CE
:10B120000BF1280BA5E6FB0777D5D8F8EC305FFAD2
:10B1300089FA1969586B08EB8A0220FA0AFBD2F8DF
:10B14000F4204FEACB1B92685FFA8BFB4BEA010BB2
:10B150000BEA020B1BF0010F1ED05A6BA8484FF0F0
:10B16000010B0BFA09F122EA01025A633368C3F8B2
:10B1700008B0A44B5146D3F87838984798F8DF3098
:10B180005B4509D1B9F1000F06D198F8ED31042BD8
:10B1900002D19B48FFF78AFD1BF0080F1EBF3368E2
:10B1A0004FF0080BC3F808B01BF0100F1EBF336838
:10B1B0004FF0100BC3F808B01BF0400F1EBF3368F0
:10B1C0004FF0400BC3F808B01BF0020F1EBF3368EE
:10B1D0004FF0020BC3F808B01BF0800F1DD0D5E96B
:10B1E0004C329B1AD5F82421D6F800E098F8DFB04D
:10B1F000DEF81800934228BF13460333D8F8EC203A
:10B2000003920AF1320A9B0808EB8A0A80B298423C
:10B2100003D9D5E94C03984205D809F101097F0803
:10B220000436283538E6C01AD5F82431984228BFAC
:10B230001846C31C9B08BBF1000F1CD0D5F8281181
:10B24000D5F834210144C5F82811D5F8301102444D
:10B250008A42DEF81800C5F83421D7D1039A95F850
:10B260001C11526B4FF0010C0CFA01F122EA0102A1
:10B2700003994A63CAE7D5F82821049282B2DAF822
:10B28000E410033292108C4605925946059A8A4280
:10B29000D4D0049A52F82120CCF800200131F5E7EF
:10B2A00047F6F07111423FF47BAE282101FB0531D6
:10B2B000C2F30A12D71CD3F8ACE1D1F85CC4BF10BA
:10B2C00000218F420DD1282101FB0533D3F85C14F6
:10B2D0001144C3F85C14D3F868140A44C3F8682412
:10B2E0005EE6DEF800804CF821800131E9E7D3F812
:10B2F000AC110F68C3F8A8760968C3F8AC1628210A
:10B3000001FB0533C2F30A12E5E755F8042B9160FF
:10B31000AA6B013391605AE6012084F8DE004020D8
:10B32000A4F8E000A0F56400374CA0F5624010449A
:10B33000A04227D80E2262F38D23CB604FF4005336
:10B340004B61029BDA060BD5304C2E4B04F1DC002E
:10B35000D3F890389847D4F8E8304FF480125A6107
:10B36000029B9B060BD5294C264B04F1DC00D3F83D
:10B3700094389847D4F8E8304FF400125A610DB071
:10B38000BDE8F08F224CA2F57400A0F51050A04249
:10B3900001D80D22CFE71F481F4C1044A04201D214
:10B3A0000C22C8E71D4CA2F18C70A0F54340A042CE
:10B3B00001D80B22BFE71A481A4C1044A04201D210
:10B3C0000A22B8E71848194C1044A042FFF458AEBE
:10B3D000174CA2F1B770A0F55850A04201D2082234
:10B3E000A9E71448144C1044A04201D20722A2E756
:10B3F00012481044124A904234BF062205229AE7AE
:10B40000C4270020000000203F420F00E826002053
:10B41000DFC810002013FBFE20D61300FF691800C0
:10B4200000D3CEFE40771B00C05BB3FEC09121006D
:10B4300040AC2700C01D6AFE40E13300803C36FE70
:10B44000E09C41004A09012301F01F0103FA01F1C8
:10B4500050F822300B4340F8223070474A0901234C
:10B4600001F01F0103FA01F150F82230194214BF14
:10B4700001200020704780EA0120082341F22102C8
:10B4800010F4004F4FEA400018BF5040013B80B21B
:10B49000F6D170474840082310F0800F4FEA400073
:10B4A00018BF80F0D500013BC0B2F5D1704710B590
:10B4B0000A440C46944200D110BD14F8011BFFF75A
:10B4C000E9FFF7E738B50A46056804460020AA42B6
:10B4D00003D36B1C2360287038BD12F8011BFFF7E3
:10B4E000D9FFF4E782B08DED010A019802B07047F0
:10B4F000C31783EA400070479FED087AC0ED020A47
:10B50000C7EE007A0023036030EEA77AC0ED017A1F
:10B51000C0EE877AC0ED037A704700BF83F9223E00
:10B5200080ED010A704700BF90ED017AD0ED007AFE
:10B53000C0ED020A30EE877AC0EE876A30EE677A95
:10B54000E6EE877AB0EE670AC0ED007A704700BF7A
:10B5500080ED000A704700BF9FED047AC7EE007AC5
:10B5600077EEA07A80EEA70A704700BF4E2DA63D69
:10B57000002303604360836080ED030A704700BFCF
:10B58000F5EEC00AF1EE10FA06DCF0EE407A80ED3E
:10B59000000AB0EE670A704760EE810A90ED007A0B
:10B5A00077EE607AF4EEC07AF1EE10FA0ADC77EE0C
:10B5B000200AF4EEC00AF1EE10FA8CBFF0EE407AE9
:10B5C000F0EE607AC0ED007AB0EE670A704700BF17
:10B5D000B4EEE00AF1EE10FA07D4B4EEC10AF1EECF
:10B5E00010FA88BFB0EE410A7047B0EE600A7047AB
:10B5F000874BB3FBF2F399420DD300234FF07E52F9
:10B60000026043608360C360036100238361436120
:10B610000362C361704707EE902ADFED7E6AB8EEE1
:10B62000677A07EE901A27EE267AF8EE677A27EE09
:10B63000277AFDEEC77A17EE903A2033402B00F2BE
:10B64000D880DFED757AB4EEE77AF1EE10FAF0EE1D
:10B65000477A0CDDDFED715A9FED716AF0EE676A93
:10B66000F4EEC66AF1EE10FA77EEE57AF6DCDFED7D
:10B670006D6AF4EEE67AF1EE10FA0CD5DFED675A5A
:10B680009FED696AF0EE676AF4EEC66AF1EE10FAB1
:10B6900077EEA57AF6D4DFED656AF4EEE67AF1EEA0
:10B6A00010FA00F39C80DFED626AF4EEE67AF1EEC8
:10B6B00010FA03D5DFED5B6A76EEE77A27EEA76A2C
:10B6C000DFED5C5ADFED5C6A9FED5C5ADFED5C4AB2
:10B6D000E6EE256ADFED5B5AA6EE265A27EE864A8D
:10B6E000E6EE055AF7EE006AE4EE257AF0EE665AC9
:10B6F000E7EEA45AE7EEE46A86EEA54ADFED4B6A70
:10B7000077EE267ABDEEE76A16EE103A2033402B2C
:10B7100068D8B4EEE67AF1EE10FA0CDD9FED3F6AE0
:10B72000DFED3F6AB0EE677AB4EEE67AF1EE10FA3A
:10B7300077EEC67AF6DC9FED3B7AF4EEC77AF1EE4F
:10B7400010FA0CD59FED356ADFED376AB0EE677AF7
:10B75000B4EEE67AF1EE10FA77EE867AF6D49FED43
:10B76000337AF4EEC77AF1EE10FA47DD9FED2A7ACC
:10B7700077EE677A67EEA76A9FED2E6A9FED2E7AC5
:10B78000DFED2E4A9FED2F5AA6EE867A27EEA63AD7
:10B79000E6EE874AB7EE006AA6EEA45AB6EE007A45
:10B7A000E3EE057AF8EE003A36EE676A67EEA37AC2
:10B7B00026EE077AB7EE005AC5EE256A80ED044AF8
:10B7C00026EE877A26EE866A66EEA77A80ED007A04
:10B7D00080ED016A80ED027AC0ED037A15E7DFEDB6
:10B7E0000E6A69E7DFED187AB6EE007AB7EE006A06
:10B7F000E0E7B7EE004AF0EE445A7FE79FED0C7A9F
:10B80000F4EEC77AF1EE10FAB4D59FED067AAFE701
:10B8100020A1070027D4D236DB0F4940DB0FC940F7
:10B82000E4CB1641DB0F49C0E4CB16C1DB0FC93FA7
:10B83000DB0FC9BF9A7C2E36FAAF4FB93587083C6B
:10B84000F304353FA4AA2ABE00000000FDEEC07A32
:10B8500017EE903A2033402B51D8DFED2A7AB4EE20
:10B86000E70AF1EE10FA0CDDDFED276A9FED277A8B
:10B87000F0EE407AF4EEC77AF1EE10FA30EE660A96
:10B88000F6DCDFED237AB4EEE70AF1EE10FA0CD520
:10B89000DFED1D6A9FED1F7AF0EE407AF4EEC77A75
:10B8A000F1EE10FA30EE260AF6D4DFED1B7AB4EE94
:10B8B000E70AF1EE10FA18DDDFED127A37EEC00A72
:10B8C00060EE007A9FED157A9FED156ADFED156A3F
:10B8D000A7EE876A9FED147AE7EE866A60EE275A34
:10B8E000A7EEA67AA5EE870A7047DFED107AB4EED0
:10B8F000E70AF1EE10FAE3D5DFED057ADEE79FED1A
:10B900000C0A7047DB0F4940DB0FC940E4CB1641FE
:10B91000DB0F49C0E4CB16C1DB0FC93F9A7C2E3642
:10B92000FAAF4FB93587083CA4AA2ABEDB0FC9BFBE
:10B93000000000009FED2F7A70EE077AFDEEE76AB7
:10B9400016EE903A2033402B51D8B4EEC70AF1EEF0
:10B9500010FA0CDD9FED286ADFED286AB0EE677AF9
:10B96000B4EEE67AF1EE10FA77EEC67AF6DC9FEDE9
:10B97000247AF4EEC77AF1EE10FA0CD59FED1E6A28
:10B98000DFED206AB0EE677AB4EEE67AF1EE10FAF7
:10B9900077EE867AF6D49FED177AF4EEC77AF1EE59
:10B9A00010FA1ADD9FED187A77EE677A27EEA77AFC
:10B9B000DFED166ADFED165A9FED166AE7EE265A9E
:10B9C000DFED156AA7EE256A27EE875AE7EE066ACD
:10B9D000E5EE267AB0EE670A70479FED107AF4EE36
:10B9E000C77AF1EE10FAE1D59FED057ADCE79FED1D
:10B9F0000C0A7047DB0FC93FDB0FC940E4CB16418F
:10BA0000DB0F49C0E4CB16C1DB0F49409A7C2E36D0
:10BA1000FAAF4FB93587083CA4AA2ABEDB0FC9BFCD
:10BA200000000000B5EE400AF1EE10FA25D007EE56
:10BA3000902AF8EE670ADFED117A08B5034660EE4A
:10BA4000A70A0846F0EE406A4BB9FFF755FDFCEE39
:10BA5000E66A16EE903A99B2BDE80840C8E5022BB6
:10BA600006D0032BF3D1FFF777FDBDE808407FE553
:10BA7000FCF738FDFCF742FDE9E77047BD37863536
:10BA8000B5EE400AF1EE10FA02D1044B0B6070479C
:10BA900003280CBF024B034BF8E700BF7984000872
:10BAA000098500089185000890ED0E7AB5EEC07A00
:10BAB000F1EE10FA00F3978030EE607AD0ED015A83
:10BAC000037867EE255A002B5BD101F00103D0ED1E
:10BAD000117A002B61D077EE677AF0EE470AD0ED4D
:10BAE0000F6AC0ED110AF5EEC06AF1EE10FA87EEAA
:10BAF000816A55DCD0ED037A26EE276AD0ED056A1F
:10BB000090ED105A60EE266A76EE857A77EEA57A89
:10BB100077EE867AF4EEE71AF1EE10FA00F38480FD
:10BB2000B4EEE72AF1EE10FA8CBFB0EE670AB0EE81
:10BB3000420A70EE677A90ED044AD0ED024AC0EDF9
:10BB4000135A67EE847A4A07E7EE247AB0EE457A14
:10BB5000A1EE277A80ED125A80ED146AC0ED156AC5
:10BB600080ED160A08D5F0EEC77AF0EEC56AF4EE5D
:10BB7000E67AF1EE10FA6BD580ED107A0B0756D409
:10BB8000704711F001034FF000020CBFF0EE607A35
:10BB9000F0EE477A0270002B9DD177EEE07A9EE7B7
:10BBA000D0ED0B7AD0ED034A80ED0C1AF5EE407A19
:10BBB000F1EE10FA04BF9FED285AC5EE267A71EE19
:10BBC000276A08BFC0ED0B7A81EE265AD0ED0A7ABB
:10BBD00080ED0D5A36EE676AE5EE067A24EEA76A26
:10BBE000C0ED0A7A8AE7D0ED077A80ED081AF5EE03
:10BBF000407AF1EE10FA04BF9FED176AC6EE077A9D
:10BC000070EE606A08BFC0ED077A71EE277A90ED9A
:10BC1000067A81EE276A76EEC77A80ED096AA6EE8B
:10BC2000277A80ED067A49E7B0EE610A81E7F4EE03
:10BC3000C71AF1EE10FA08DCB4EEC72AF1EE10FADA
:10BC40008CBFF0EE471AF0EE421AC0ED101A7047A2
:10BC5000B0EE457A92E700BF83F9223E002301222D
:10BC60000270C36483640365036443644365836251
:10BC700083657047DFED1A7A80ED010AF4EEE70A7A
:10BC8000F1EE10FAC0ED020A80ED031AC0ED051ABC
:10BC900012DC0023836003610023012280ED0F2A60
:10BCA000C0ED0E2A0270C3648364036503644364B9
:10BCB0004365836283657047B4EEE70AF1EE10FADC
:10BCC0000CDD81EE007AC0EE207AF0EE006A77EEAD
:10BCD000877A86EEA77A80ED047ADDE70023DAE73B
:10BCE000BD378635F0EEC07AB0EEE07AB4EEE77A92
:10BCF000F1EE10FAB4BFB0EE676AB0EE476AB5EE87
:10BD0000406AF1EE10FA46D0B4EEE77AF1EE10FA9E
:10BD10008CBFF0EE675AF0EE475AC5EE866ADFED4B
:10BD20001F2ADFED1F3ADFED1F4A9FED1F5A9FEDDF
:10BD30001F3A9FED1F4ADFED1F5AE6EEE23AA6EEEC
:10BD4000834AE6EEA34AB7EE006AA6EEA45AA6EE30
:10BD5000846AE6EE855AC5EE866AB4EEE77AF1EEBD
:10BD600010FA48BFDFED147AF5EEC00A48BF77EE4F
:10BD7000E66AF1EE10FA48BFDFED107AB5EEC00AC0
:10BD800048BF77EEE66AF1EE10FA48BFF1EE666A58
:10BD9000B0EE660A7047DFED076ADEE739094E3D0F
:10BDA000E3B59E3E88FA163E45FE7F3F99FB243F51
:10BDB00069A2163EA7DFA834DB0FC93FDB0F49405D
:10BDC000B7EE007AF0EEC07AF4EEC77AF1EE10FA30
:10BDD00077EE676A1DD8B1EEE67ADFED0F5ADFED38
:10BDE0000F6A9FED0F6AE7EEA65ADFED0E6AA7EE27
:10BDF000A56AE7EE866A67EE266AB5EEC00AF1EE3E
:10BE000010FA44BF9FED087A77EE666AB0EE660AD4
:10BE10007047DFED066AF0E72716983D306E99BC53
:10BE2000843459BEA40DC93FDB0F49400000000017
:10BE3000B0FBF1F301FB130308463BB11946B0FB1D
:10BE4000F1F301FB13030846002BF7D1704700BF45
:10BE500044F25063984203DDA0F50C40A0387047CF
:10BE6000034B9842BCBF00F50C40A030704700BFA8
:10BE7000B0B9FFFF48F6A043984203DDA0F50C409F
:10BE8000A03870470028B8BFC018704780EAE07338
:10BE9000A3EBE0738B4203DB002803DD401A7047FD
:10BEA00000207047FDD00844704700BF884203DB84
:10BEB0009042A8BF104670470846704700230361B0
:10BEC000704770B50378012B044635D10369214DC5
:10BED00023B9426812B955F8C42C4260D4ED067AF1
:10BEE00077EE807A013304F11C062361C4ED067AF3
:10BEF0003046FCF773FB626855F8C43C9B1AA26895
:10BF0000934219D9E06A94ED0A0A4EF087FAD4ED0B
:10BF1000057AB4EEE70AF1EE10FA0EDD237B4BB999
:10BF200055F8C42C236100236260A3613046BDE84C
:10BF30007040C3E70323237070BDD4ED047AD4EDC1
:10BF4000066AF8EE677A022386EEA77A84ED067A0F
:10BF5000F1E700BFE82600202DE9F04104461C303F
:10BF6000254604F16402064650ED017AB1EC010A5F
:10BF700077EE807A40ED017AFCF730FB1830904282
:10BF8000F2D12369294F62680133236157F8C43C19
:10BF90009B1AA268934246D904F13008E86A95EDED
:10BFA0000A0A4EF03BFAA845D4ED057A1CD0B4EE4F
:10BFB000E70AF1EE10FA05F11805EFDD237B83BBEC
:10BFC00057F8C42C6260002223613046A261FFF75B
:10BFD00075FF04F134002263FFF770FFA26404F1DF
:10BFE0004C00BDE8F04169E7B4EEE70AF1EE10FA63
:10BFF000E4DCD4ED047AD4ED066AF8EE677A022325
:10C0000086EEA77AD4ED0C6A84ED067A86EEA77ADE
:10C01000D4ED126A84ED0C7A86EEA77A84ED127A5A
:10C0200000E003232370BDE8F08100BFE826002074
:10C0300010B4019C401AA4EB030C00FB0CFC511A39
:10C040005DF8044B9CFBF1FC0CEB0300704700BF58
:10C0500030EE600A32EE612A71EE600A22EE002AAA
:10C0600082EE200A30EE210A704700BFD1ED007A3F
:10C07000DFEDE16A37EEA67ABDEEC76A16EE103A3A
:10C080002033402B00F25882F4EEE67AF1EE10FAFB
:10C090000CDDDFEDDB5A9FEDD96AF0EE476AF4EE76
:10C0A000C66AF1EE10FA37EE657AF6DCDFEDDE6A8D
:10C0B000B4EEE67AF1EE10FA0CD5DFEDD15A9FED31
:10C0C000D16AF0EE476AF4EEC66AF1EE10FA37EE86
:10C0D000257AF6D4DFEDC86AB4EEE67AF1EE10FA0E
:10C0E00040F30282DFEDC96A36EEC77A67EE076A6F
:10C0F0009FEDC76A9FEDC75ADFEDC75AA6EE865A75
:10C100009FEDC66AE6EE855A27EE264AA6EEA56A98
:10C11000A4EE067AF0EE474ABDEEE77A17EE103A43
:10C120002033402B00F205829FEDB87AF4EEC77AF7
:10C13000F1EE10FA0CDD9FEDB26A9FEDB07AF0EEF1
:10C14000676AF4EEC76AF1EE10FA77EEC67AF6DCAB
:10C150009FEDB57AF4EEC77AF1EE10FA0CD59FEDAB
:10C16000A86A9FEDA87AF0EE676AF4EEC76AF1EE6E
:10C1700010FA77EE867AF6D49FED9F7AF4EEC77ABE
:10C18000F1EE10FA40F3DB819FEDA07A77EE677A4B
:10C1900027EEA77ADFED9E6ADFED9E5A9FED9E6A3D
:10C1A000E7EE265ADFED9D6AA7EE256A27EE874A5D
:10C1B000E7EE066AE4EE267AB0EE675A91ED017A70
:10C1C000DFED8D7A77EE276ABDEEE66A16EE103A5D
:10C1D0002033402B00F2A681B4EEE77AF1EE10FA9C
:10C1E0000CDDDFED875ADFED857AB0EE666AB4EEDE
:10C1F000E76AF1EE10FA76EEE56AF6DCDFED8A7AB0
:10C20000F4EEE76AF1EE10FA0CD5DFED7D5ADFEDC2
:10C210007D7AB0EE666AB4EEE76AF1EE10FA76EE79
:10C22000A56AF6D4DFED747AF4EEE76AF1EE10FA5F
:10C2300040F39B81DFED757A77EEE66A66EEA67ACB
:10C24000DFED735A9FED734A9FED736AA7EEA54A1F
:10C25000DFED725AA7EE846A66EEA73AE7EE865AD9
:10C26000E3EEA56A66EEC52A24EEA63AB0EE666A4B
:10C27000FDEEC77A17EE903A2033402B00F24F8143
:10C28000DFED627AB4EEE77AF1EE10FA0CDDDFED65
:10C290005C5ADFED5A7AF0EE476AF4EEE76AF1EEA7
:10C2A00010FA37EE657AF6DCDFED5F7AB4EEE77A06
:10C2B000F1EE10FA0CD5DFED525ADFED527AF0EEC6
:10C2C000476AF4EEE76AF1EE10FA37EE257AF6D413
:10C2D000DFED497AB4EEE77AF1EE10FA40F33A81F5
:10C2E000DFED4A7A37EEC77A67EE077ADFED485A14
:10C2F0009FED484ADFED486AA7EEA54ADFED475AB1
:10C30000E7EE846A67EE273AE7EEA65AA3EEA57A2F
:10C31000F0EE476AD1ED027ADFED375A37EEA57AB3
:10C32000BDEEC74A14EE103A2033402B00F2EC80E9
:10C33000F4EEE57AF1EE10FA0CDDDFED313A9FED27
:10C340002F4AF0EE475AF4EEC45AF1EE10FA37EEE7
:10C35000637AF6DCDFED345AB4EEE57AF1EE10FAEA
:10C360000CD5DFED273A9FED274AF0EE475AF4EE61
:10C37000C45AF1EE10FA37EE237AF6D4DFED1E5AE6
:10C38000B4EEE57AF1EE10FA40F3FA80DFED1F5AD1
:10C3900035EEC77A67EE075A9FED1D4A9FED1D2ABD
:10C3A000DFED1D3AA5EE842A9FED1C4AE5EE823AA8
:10C3B00067EE251AA5EEA34AA1EE847A25EE072A98
:10C3C00064EE871A26EE821A26EE077A26EEA10A76
:10C3D000FDEEE75A15EE903A2033402B00F28F80A5
:10C3E000DFED0A5AF4EEE57AF1EE10FA27DDDFED23
:10C3F000043A9FED024A19E0DB0FC93FE4CB164136
:10C40000DB0FC940E4CB16C1DB0FC93FDB0F49404E
:10C410009A7C2E36FAAF4FB93587083CA4AA2ABEBB
:10C4200000000000DB0FC9BFDB0F49C0F0EE675A08
:10C43000F4EEC45AF1EE10FA77EEE37AF6DC5FED33
:10C44000065AF4EEE57AF1EE10FA0CD55FED143AE7
:10C450001FED144AF0EE675AF4EEC45AF1EE10FAEA
:10C4600077EEA37AF6D45FED185AF4EEE57AF1EEA2
:10C4700010FA40F390805FED1B5A75EEE77A27EED5
:10C48000A74A5FED1D5A5FED1D3A5FED1D0AE4EE10
:10C49000253A67EE845AE4EE230A5FED203AE4EE93
:10C4A000203AE5EEA37A64EEA74A65EE275AA6EE97
:10C4B000A42AE6EEE51A67EEC67A31EE241A75EE86
:10C4C000C05A80ED007AC0ED017AC0ED026A80EDBD
:10C4D000031AC0ED041AC0ED052AC0ED065A80ED1E
:10C4E000072A80ED083A70475FED326AB4EEE67ACB
:10C4F000F1EE10FA7FF5FAAD5FED356AF4E55FED28
:10C50000385AF0EE657ADAE71FED3B2AF0EE421A70
:10C51000B0EE420AB0EE421AB0EE427A58E75FED52
:10C52000406AF7E61FED423AF0EE432AB0EE436A66
:10C530009EE61FED455A41E65FED474AECE51FEDEB
:10C54000477AF4EEC77AF1EE10FA7FF521AE1FEDCF
:10C550004A7A1BE65FED4D7AB4EEE77AF1EE10FA17
:10C560007FF5C2AE5FED507ABCE65FED527AF4EE35
:10C57000E76AF1EE10FA7FF561AE5FED557A5BE6A2
:10C580005FED585AB4EEE57AF1EE10FA7FF502AF9E
:10C590005FED5B5AFCE65FED5D5AF4EEE57AF1EE95
:10C5A00010FA7FF56CAF5FED605A66E70023036118
:10C5B00043618361C3610360036243628362C36258
:10C5C0004360036343638363C363836003644364BF
:10C5D0008364C364C3607047D1ED017A91ED007A42
:10C5E000D0ED044A90ED065AD0ED075A90ED050AB9
:10C5F000D0ED080AD0ED0A1AD0ED0C2A90ED0D3AD4
:10C60000D0ED0E3A90ED091A90ED0B2AF8EEE76A9C
:10C61000D1ED027AB8EEC77AF8EEE77A26EEA64AAE
:10C62000A7EE275AE7EE074AB0EE446A75EE875A3E
:10C63000A7EE076AE7EE272AE7EEA73AA7EE260A53
:10C64000E7EE260AE6EEA71AA6EEA73A31EE041A9E
:10C65000C0ED044A90ED0F4AD0ED104A80ED065A25
:10C66000C0ED075A90ED115AD0ED125AC0ED0E3AB6
:10C67000A7EEA76A34EE274A74EE874A75EEA75AEA
:10C6800035EE265A32EE262A80ED0F4AC0ED104ACA
:10C6900080ED115A80ED050AC0ED080A80ED091AF7
:10C6A000C0ED0A1A80ED0B2AC0ED0C2A80ED0D3A80
:10C6B000C0ED125A90ED004A90ED025AD0ED014AB9
:10C6C000D0ED133AD0ED035AA7EE064AB0EE457A04
:10C6D000A7EE867AE6EE864AF7EE007A73EEA77A40
:10C6E00035EE866AC0ED137A80ED004AC0ED014A4E
:10C6F00080ED027A80ED036A704700BF10B5002418
:10C70000034684468646002C00F00D81DEED006A6B
:10C710009CED007AD3ED007AE6EEC77A012CC3EDEA
:10C72000007A00F00F81DEED016A9CED047AE6EEFE
:10C73000C77A032CC3ED007A6CD1DEED026A9CED62
:10C74000087AE6EEC77AC3ED007AD2ED007A90ED72
:10C75000085AD0ED0C5AD0ED044A92ED017AD2ED90
:10C76000026A92ED036AA7EEE47AE7EEC56AA7EEE5
:10C77000E56A90ED095AD0ED0D5AE7EE456AA5EE4F
:10C78000C76AD0ED0E5AA5EEE66A81ED036A90ED18
:10C790000F5AC1ED026AC6EE055AC1ED035A90ED7B
:10C7A0000B6AE5EEC66AC1ED026A90ED0A5A81EDA8
:10C7B000017A86EE856A81ED026AD0ED066AA6EE00
:10C7C000667A81ED017AD0ED076AA5EEE67A81ED11
:10C7D000017A90ED055AC1ED007AC7EE056AC1ED08
:10C7E000016A90ED017AE7EE667AC1ED007A90ED8C
:10C7F000027AE7EE467AC1ED007A90ED037AE7EE31
:10C80000657AC1ED007AD0ED006A87EEA67A81EDF7
:10C81000007A10BD9EED007ADCED016AD3ED017A5D
:10C82000E7EE667A022CB1EE476AC3ED017ADEEDDF
:10C83000016A9CED057AE6EEC77AC3ED017A40F015
:10C84000AC80DEED046A9CED007AD3ED047AE6EE6E
:10C85000C77A012CC3ED047A40F28780DEED056AC9
:10C860009CED047AE6EEC77A032CC3ED047A7FD1FF
:10C870009EED066ADCED086A93ED007AE6EE667AD4
:10C88000C7EE876AC3ED046A9EED086ADCED006AB4
:10C89000D3ED087AE6EE667A012CC3ED087A70D9FA
:10C8A0009EED096ADCED046AE6EE667A032CC3EDC0
:10C8B000087A07D19EED0A6ADCED086AE6EE667A30
:10C8C000C3ED087A93ED086AD3ED0C7AC6EE076AD9
:10C8D000032CC3ED086A9CED006ADEED0C6AE6EEFF
:10C8E000667AC3ED0C7A9CED046ADEED0D6AE6EE25
:10C8F000667AC3ED0C7A07D19EED0E6ADCED086A0C
:10C90000E6EE667AC3ED0C7AD3ED0C6AC6EE877A52
:10C91000C3ED0C7A013414330EF1100E0CF1040C3B
:10C92000002C7FF4F3AED3ED047A93ED007A93ED0F
:10C93000086AC7EE876AC6EE077AC3ED046AC3EDDC
:10C94000087AE1E7DEED006A9CED016A93ED017A79
:10C95000D3ED027AA6EEC67A83ED017A9CED027AD7
:10C96000E7EE667AC3ED027A6BE793ED007A87E72C
:10C9700093ED007AC7EE876A022CC3ED046AC9D032
:10C9800082E7C7EE876AC3ED086AC3D09CED006AF0
:10C99000DEED0C6AD3ED0C7AB2E79CED027AD3EDB2
:10C9A000027AE6EE077A032CC3ED027ADCED066A22
:10C9B0009EED017AE6EEC77AC3ED027A7FF441AFCD
:10C9C000DEED026A9CED0A7AE6EEC77AC3ED027AE2
:10C9D000BBE600BF10B584B00C4602466946103075
:10C9E000FFF78CFEDDED006A9DED017ADDED027A48
:10C9F000B6EE006A66EE866A27EE067A67EE867AFB
:10CA00000120C4ED006A84ED017AC4ED027A04B01D
:10CA100010BD00BF20EE000AFEEE007A60EE277A1D
:10CA200060EEA00A9FED020AC7EEA00A51F054BCC6
:10CA300054F82D4008B54EF0D9FC07EE900AF5EEFB
:10CA4000C07AF1EE10FAACBFB1EEE70A9FED010A31
:10CA500008BD00BF0000000060EEA00AE0EE000A82
:10CA6000B1EEE00A704700BF21EE011AA0EEA01A55
:10CA7000A0EE001AB1EEC10A70472DE9F74F9046BB
:10CA80009DF83020002A14BF4FF030094FF02009E4
:10CA90000D9A1C1E05460F46BABF644201230023AF
:10CAA00012F8011B01B12CB9A24663B100240D9EFE
:10CAB000A41B12E0013CF3E7BD4204D249462846DC
:10CAC0000193C047019BBAF1010AF5D2EFE7BD42DD
:10CAD00003D228460193C047019B06EB040B16F8CE
:10CAE000011B0029F3D133B15446002C07DCBAF105
:10CAF000000FA8BFD344584603B0BDE8F08FBD4235
:10CB000002D249462846C047013CEEE70FB437B58C
:10CB10000B4D06ABD5F83C1753F8042BD5F8380766
:10CB200001934BF025FF0446D5F8A00003F0BCFFAD
:10CB30000028F9D0204603B0BDE8304004B070476B
:10CB4000E82600200EB403B503AB084953F8042BC4
:10CB5000CDE9003001A84BF00BFF019B00221A70B9
:10CB600002B05DF804EB03B0704700BF2F860008E9
:10CB70000CB430B5294CD4F84037A5B01BB9D4F863
:10CB80004437002B38D094F84837994206D901230E
:10CB900003FA00F0D4F84C3718422DD054F8C41CD6
:10CBA0004FF47A7304A8B1FBF3F203FB12131C4990
:10CBB000FFF7C8FF04AB0344289A1A4903930546BC
:10CBC00029AB03A802934BF0D3FE039B591C03919E
:10CBD0000A211970039B0246591CD4F8400703919F
:10CBE0000021197068B103681B6A03B19847D4F833
:10CBF000400704A903F026FF25B0BDE8304002B08D
:10CC00007047D4F84437002BF6D002212A44009113
:10CC10000A44FD2004A924F085F9EDE7E826002068
:10CC200021A30608D385000830B54FF4004087B033
:10CC300022F030FB0446A0B34FF4004122F08CFCFC
:10CC400002281CD1226848F201039A4229D1234CC0
:10CC5000002584F8E4594FF400404BF0EFF800B39E
:10CC6000D4F8503783421ED0D4F82C3883422FD0CA
:10CC7000D4F8083998422ED0C4F8445711E0002364
:10CC8000022294F90400CDE901234FF461220092BD
:10CC90004FF400411A4622F0B9FC104BC3F840078C
:10CCA00028B907B030BD04F5EA63C4F844370C4B2B
:10CCB00004930C4B03930C4B02930C4B01930C4BC2
:10CCC00000930C4A0C4B02210020FFF751FFE8E7CC
:10CCD00004F62C03E9E704F60813E6E7E82600204B
:10CCE0002DA3060836A306083FA306084BA3060893
:10CCF00051A3060882A90608F9A20608174A38B502
:10CD0000D2F8E849033004EB9003B3F5007F19D85B
:10CD100002F6EC15C2F8E839114A02EB810120F065
:10CD20000300D1F8F420C3F500731044C1F8F400F7
:10CD30000C4A9B000421002005EB8404FFF718FF38
:10CD4000204638BD0021084A0846FFF711FF074A70
:10CD5000136843F0007313600024F1E7E826002015
:10CD6000E03700205DA3060880A30608F00001203C
:10CD70002DE9F04706460068FBF7C4F90D28054683
:10CD800008DD1F4A00210520FFF7F2FE002420469F
:10CD9000BDE8F0871B4F07EB80094FEA8008D9F800
:10CDA000A4A0BAF1000F1CD10A216420FFF7A6FF4E
:10CDB0000446C9F8A40028B90146134A0520FFF724
:10CDC000D7FEE4E76422514654F0C5FA0F48D9F87B
:10CDD000A4302DB200EBC505C3E90053DB615B63F2
:10CDE000DB6447447179D7F8A440182000FB014365
:10CDF00000221C46C3E903229E601A750434C6E76C
:10CE00008EA30608E8260020B3A30608901406089F
:10CE100003685A1C026019700368090A5A1C0260F0
:10CE20001970704703685A1C0260197003685A1C15
:10CE300002600A0A1A7003685A1C02600A0C1A700F
:10CE40000368090E5A1C02601970704703685A1C67
:10CE500002600A0A1A7003685A1C0260197070474F
:10CE600038B504460068154654F03CF823682B4456
:10CE7000236038BD03685A1C026018787047036845
:10CE80005A1C02601A4612F8021B0260587841EAE6
:10CE90000020704710B502681146531C036011F85A
:10CEA000024B0160D31C5178036093781B0443EA62
:10CEB0000123111D0160D078234343EA006010BDB7
:10CEC000D1E900329A4206D05A1C0A6008B11B7898
:10CED00003700120704700207047D1E900239B1A9E
:10CEE000012B10B50446084604DDFFF7C8FF20807B
:10CEF000012010BD0020FCE730B50A4404469142F1
:10CF000001D1002011E014F8013BA3F141001928E0
:10CF100011F8010BA0F1410598BF2033192D98BFDE
:10CF200020301B1A02D10028E9D130BD1846FCE799
:10CF30006FF00042E0E710B50288C378A2F5FA620C
:10CF4000910840F2B554013B04FB013381780C2475
:10CF5000013902F0030204FB02120D49847901EB4E
:10CF600042021821B2F8D0201344027901FB0322B7
:10CF7000437900893C2101FB0233064A224401FB2C
:10CF800003224FF47A730021C2FB030110BD00BFDE
:10CF90009014060880436D382DE9F04190461F46F5
:10CFA00005464FF47A720023404639464EF07CFB2A
:10CFB000284B3C21034493FBF1F201FB1233AB718C
:10CFC00092FBF1F301FB13226A7140F2B551182272
:10CFD00093FBF2F402FB143394FBF1F201FB1244D5
:10CFE000B4F5896F2B714FEA82032EDA40F2DA2210
:10CFF00094422CDCB4F5B77FB4BF00210121164A5E
:10D00000182000FB01220B2632F81600A04201DD99
:10D01000013EF9D103F5FA630B442B80731CAB700E
:10D020000C2303FB01660D4B03EB46060134B6F8F7
:10D03000D030E41AEC704FF47A720023404639463F
:10D040004EF032FB2A81BDE8F0810321D7E70221AF
:10D05000D5E700BF80BC92C760150608901406088B
:10D06000F0B5274D06460F460FCD8DB06C460FC468
:10D070000FCD0FC495E80F0084E80F0016F00303EE
:10D080003AD1642196FBF1F201FB126242B94FF4EE
:10D09000C87296FBF2F302FB1363003B18BF012337
:10D0A000721EC3F11D03002A019340F26D13104656
:10D0B00006FB03F3B8BFB01C03EBA0006FF06303E3
:10D0C00092FBF3F318444FF4C87392FBF3F210444D
:10D0D0000630694600240725013F51F8042BA7427A
:10D0E00002EB000393FBF5F0C0EBC000A3EB0000E4
:10D0F00004D1101A0DB0F0BD0123D1E70134ECE7E3
:10D10000C0150608084BD3E9621251EA020309D0A0
:10D11000064B53F8C43C5B1842F10002C0E90032F0
:10D120000120704700207047E0370020E8260020EB
:10D1300037B505466846FFF7E5FF044638B1DDE937
:10D1400000232846FFF728FF204603B030BD40F2F9
:10D15000011328806B80A880A8712881F4E700BFA4
:10D160008842F0B54FF0010461D301FB04F4B0FB39
:10D17000F4FC8C45F9D284B3002A45D0002511E097
:10D18000BCF1090F2646CCBF372230229444B1426D
:10D1900083F800C0744603F1010305F101051CD8B2
:10D1A000B0FBFEFCB4FBF1FE04FB1C00002DE7D13C
:10D1B000BCF1000FE4DCA1420BD8B0FBFEFCBCF1DB
:10D1C000000F74460EFB1C00BEFBF1FED8DCA14232
:10D1D000F3D90CF1300C03F801CB00221A70F0BD2A
:10D1E000BCF1090F2646CCBF4FF0570E4FF0300E62
:10D1F000F444B14283F800C02C4603F1010302F16C
:10D200000102EAD8B0FBF5FCB4FBF1F504FB1C000D
:10D21000002AE5D1BCF1000FE2DCA142D9D8B0FB75
:10D22000F5FC2C4605FB1C00B5FBF1F5F2E7844646
:10D23000002AA3D1E8E700BF0028BCBF2D2340424D
:10D2400070B5B8BF01F8013B092804464FF001034F
:10D2500007DD03EB83035B00B0FBF3F2092AF8D888
:10D260003BB3164D4FF0000C0AE0092A8CBF572142
:10D2700030210A44092B0EF8012B16D971460346BA
:10D28000A5FB0320B4FBF3F25CEA02068E464FEAEC
:10D29000D00003FB12440CF1010CE6D1092B01D99B
:10D2A000B446EBE730320EF8012B00238EF8003045
:10D2B00070BD8E4600238EF8003070BDCDCCCCCC36
:10D2C00090422DE9F0410B46044615460AD2B0FBC8
:10D2D000F5F6134A05FB16441846135D00F8013BAA
:10D2E000BDE8F081B0FBF2F69642B6FBF2F706D24B
:10D2F0000B4A05FB1767D15D03F8011BEAE7BA4249
:10D30000B7FBF2F807D9064A05FB187812F808109F
:10D3100003F8011BEDE74046FFF7D2FF0346F2E7B3
:10D32000E8A30608B5EEC00ADFED307AF1EE10FA98
:10D33000CCBF30EE270A30EE670ADFED2D7A20EE03
:10D34000270A70B5FDEEC07A86B017EE904A054602
:10D3500084EAE470002303A9A0EBE470CDE9003374
:10D3600002934BF003FD002CACBF20232D2303A818
:10D370008DF800304DF0A6FB01286E4626D002281D
:10D380002DD003281CD003A9304653F0ECFF3046C3
:10D390004DF098FB0338C4B222463146284653F07C
:10D3A000A1FD00232B5528464DF08CFB2E232B543A
:10D3B00001303119284453F0F2FF284606B070BD01
:10D3C000302303A930468DF80130DEE743F2300206
:10D3D000302303A9ADF801208DF80330D4E743F2E0
:10D3E000300303A93046ADF80130CEE76F12033A9F
:10D3F00000007A440378202B024600F10100F9D0A6
:10D40000092BF7D02D2B25D02B2B00F0A280B7EEC7
:10D41000000AA3F13001C8B209289FED587A10D84C
:10D42000F2EE046A07EE901AF8EEE77A12F8013F7E
:10D43000E7EE267AA3F13001C8B20928B0EE677A88
:10D44000F0D92E2B62D003F0DF03452B07D020EE5E
:10D45000070A70475378BFEE000A0246D9E710B4B6
:10D4600051782D297AD02B290BBF9178A1F1300367
:10D47000A1F13003013208BF0232092B64D8002425
:10D48000002303EB830301EB430312F8011FA1F117
:10D4900030000928A3F13003F3D9B3F59A7F1A4677
:10D4A00028BF4FF49A72072B64D9DFED356A134613
:10D4B000F7EE007A083B072B67EEA67AFAD802F05F
:10D4C0000702DAB1F2EE046A012A67EEA67A15D0F5
:10D4D000022A67EEA67A11D0032A67EEA67A0DD04B
:10D4E000042A67EEA67A09D0053A67EEA67A05D037
:10D4F00067EEA67A012A18BF67EEA67A34B387EEE4
:10D50000277A5DF8044B20EE070A70475378A3F1A1
:10D510003001C8B2092802F1010294D8F2EE046A7F
:10D52000F0EE665A07EE901AF8EEE77A12F8013F2D
:10D5300087EEA66AA3F13001C8B2092866EEA56A93
:10D5400037EE067AEED97EE7F7EE007A27EE277AF5
:10D55000D7E75378B7EE000A02465AE79178A1F16F
:10D560003003092B02F1020288BFF7EE007AC6D819
:10D57000012485E7F7EE007AA3E700BF0000000072
:10D5800020BCBE4C0378202B024600F10100F9D0EC
:10D59000092BF7D0303BDBB2092B4FF000000AD843
:10D5A00012F8011F00EB8000303903EB4000CBB2D2
:10D5B000092BF5D9704770470378202B024600F1FC
:10D5C0000100F9D0092BF7D02D2B0CBF024601200A
:10D5D00092F800C0ACF13001CBB208BF4FF0FF3081
:10D5E000092B4FF0000302D903FB00F0704712F83B
:10D5F00001CF03EB830301EB4303ACF130015FFA8E
:10D6000081FCBCF1090FEEE710B50023802804D897
:10D6100093420AD2C854581C10BD934205D060F002
:10D620007F04CC54C0090133F0E74FF0FF30F3E73B
:10D6300038B50C468D18AC4200D138BD14F8011B2A
:10D64000FDF719FFF7E770B51249134C134E01228D
:10D650000020FFF7EDFF228862B1A31DB34217D26D
:10D66000A518B54214D2052A12D92146FFF7E0FFCA
:10D670002C46F0E721460222FFF7DAFF63880849CB
:10D68000084AC31A641A5842A2F89041584170BD22
:10D690000020FCE70040000801400008008000086E
:10D6A000FC3F0008E037002003682DE9F041044604
:10D6B0004068134483421AD80D468E1804F10C07B3
:10D6C0004FF00008B54202D16069BDE8F0812369DE
:10D6D0005A1C2261234415F8011B1973042AF1D145
:10D6E00039462046FBF763FDC4E90480EAE74FF0C2
:10D6F000FF30EAE7034AD2F8943123EA0000C2F887
:10D7000094017047E03700200346064906488842E6
:10D7100001D3002070470288C2F30B029342F9D074
:10D720001430F4E798040708ACFF060813B54288E4
:10D730000B460446C2F30B0200211846019253F037
:10D740000AFE216903460A48814209D30948019A21
:10D75000814205D2184602B0BDE8104053F0C2BB6A
:10D7600021B1184602B0BDE81040084702B010BD14
:10D77000980407080E09070810B4B0F9024042885F
:10D78000002C0B4641685DF8044BBEBFC2F30B0290
:10D79000DBB203FB0211C9E730B5094B094CA342C8
:10D7A00000D330BDB3F902205988002A06DA5A683E
:10D7B000DD68C1F30B0100FB01222A601433EEE7A0
:10D7C000ACFF06089804070830B502460144002063
:10D7D00012F8015B082480EA050313F0010F4FEAF9
:10D7E00050001CBF80F08C03D8B2631E13F0FF04FE
:10D7F0004FEA5505EFD18A42EAD130BD2DE9F04F0D
:10D8000087B0CDE902120025804604930195039B61
:10D81000404603EBC50AFBF7D3FBEC0002460028A9
:10D820006DD0002201214046FBF7B4FB02460028E0
:10D8300065D098F80430990761D5F0214046FBF790
:10D84000C9FB024600285AD0039BA4F108024FF0FE
:10D85000000B012713443C465E460593029B002BB8
:10D8600055D0082C53D804F1FF3943FA09F909F0CF
:10D87000010949464046FBF786FB024600283ED098
:10D88000002201214046FBF785FB0246002836D0E6
:10D8900098F8041001F0600CBCF1600F4FEAD11051
:10D8A00016D0029B1BB1082C01D8814527D1002836
:10D8B00041D01AF8061039437F00013417F0FF07F2
:10D8C0000AF80610E4B2C9D10136F6B2082E1CD10E
:10D8D000402C10D9072150460592FFF775FF9AF8A2
:10D8E0000710059A814206D10135EDB2BBF1000F58
:10D8F00005D0CDF804B0049B1B78AB4287D8049BBD
:10D9000010461D7007B0BDE8F08F0127A6E75DB196
:10D91000019BA34208D9059B9A5D174214BF4FF0A3
:10D9200001094FF00009A4E7019B1B1BD3F100097B
:10D9300049EB03099DE7880940EA511111F0010FF5
:10D940001AF8061008BFA34621EA0701B4E700BF92
:10D950000123037750F8043C0BB11838184770477F
:10D9600090F83420034602F0FF0012B1002283F841
:10D97000342070474FF4805383817047064A002358
:10D9800052F8041B814204D00133042BF8D100204B
:10D9900070470120704700BF004100200120704700
:10D9A000012070472DE9F84F614FDFF88881B7F803
:10D9B00006E0D8F8004015463A88C2EB241352001E
:10D9C000C2EBE402B7F90240624303FB03F4B7F988
:10D9D000043024135C43A41304EBE224B7F90A30A7
:10D9E000BC610E46A4F5FA3181FB019AD81703FBFE
:10D9F0000AF209FB0022A3FB09304FEA132CB7F906
:10DA00000830104483FB013212034CEA006C42EAF6
:10DA100013521B031CEB030342EB202202F50042CE
:10DA2000A3FB0E3C0EFB02CC4FEAEC734FEA6C02F8
:10DA300053EA6C0C4FF000006ED0B7F910B04FEA0B
:10DA4000EB7E0BFB0AFC09FB0ECCABFB099B0CEB42
:10DA50000B0EB7F90EC08CFB01A14FEA414C4FEA07
:10DA60004A4111EB0909D8F804104CEADA3C4EEBB4
:10DA70000C0CC1F5801E0EF00048B7F90C1048EAF6
:10DA80005E0810EB09004FEACE7EBEEB00000CEB07
:10DA9000C10C68EB0C0840F6354CA0FB0C010CFBEC
:10DAA00008114DF001FEB7F916304FEA613E4FEA1A
:10DAB000503C4CEAC14C03FB0EF24FEAE3790CFBFD
:10DAC0000929A3FB0C324A4403FB0EFE0CFB02EEB9
:10DAD000A3FB0C3CB7F91420E6445B0E43EACE13DB
:10DAE00013EB000C804602FB01F34FEAE27941EBB5
:10DAF0006E6EA2FB082809FB00314144D00C40EABD
:10DB000041301CEB0000B7F912304EEBE141000A46
:10DB100040EA016000EB03100EB1000A306025B14D
:10DB200004EB8404803424122C600120BDE8F88FBB
:10DB300050400020385D00202DE9F74F534BCDE9D0
:10DB40000012534A99685389D68897891B02C91ACB
:10DB500013896EEB0E0EA3FB010403FB0E449388A6
:10DB6000C00940EA44601B04C018A6FB013506FB4F
:10DB70000E5556884FEA132343EA05634FEAC6362B
:10DB80004FEAE41444F100049B19A7FB012607FBAC
:10DB90000E664FEAD25242EA46224FEA252545F167
:10DBA0000005F61512F5FA6C46F1000BBCF5FA6F9C
:10DBB0007BF100074CDAA2FB02784FF0050A02FB6A
:10DBC00006F908EB4909A7FB0A780AFB09884FEA1E
:10DBD000570949EAC879BF08B0EB090047EA8877D6
:10DBE00064EB6804DB1B2B4F65EBA805BC454FF0CD
:10DBF000FF377BEB070720DA40F6AC57D21946F126
:10DC000000065643A2FB027202EB46064FEAC60824
:10DC1000FA00BA1A48EA577866EB0808101844EB7D
:10DC200008044FF00B08A7FB087208FB06267F08C4
:10DC300047EAC677DB1B65EB660501FB0EFEA1FB21
:10DC4000011202EB4E0EC90F41EA4E01BCEB010C72
:10DC5000009A92B10D4AD168A1FB032301FB05355F
:10DC6000520D42EAC522121A4FEA6555009B65EB38
:10DC70000404D20B42EA44421A60019B0BB1C3F880
:10DC800000C0012003B0BDE8F08F00BF385D002068
:10DC90004040002024FAFFFF01207047094B0A484A
:10DCA0001B6800691B1AFA2B09D811B1074B1B68B6
:10DCB0000B6012B1064B1B681360012070470020F7
:10DCC000704700BF24260020385D0020D048002087
:10DCD000D4480020034B0022C3E90522C3E90722F0
:10DCE00001207047385D0020084B1A68084B196AFC
:10DCF000521AFA2A9FBF5A69C2869A69DB699DBF88
:10DD00000287438701200020704700BF242600209F
:10DD1000385D002090F85F3230B53BB990F85D1265
:10DD200090F85E320124DAB2914200D830BDB0F8EA
:10DD3000665204FA03F22A43A0F866220133F2E79E
:10DD4000437913F001031FBFD0E90732C0689B1A63
:10DD500000F1FF3014BF184018467047437913F0A4
:10DD600002031FBFD0E9093200699B1A00F1FF309E
:10DD700014BF98431846704710B5437913F0010358
:10DD800001460DD0FFF7DCFF60B10A6A4B69C86835
:10DD90009B5C0132B2FBF0F400FB1422DBB20A629E
:10DDA000184610BD0346FBE743799B070AD5436A33
:10DDB0008269D154436A02690133B3FBF2F102FB79
:10DDC00011334362704741717047D0E90920131A3B
:10DDD000584258417047024B1B685B68184700BFA8
:10DDE0000C430020024B1B6808309B68184700BF9B
:10DDF0000C4300200120704701207047012070472C
:10DE00000120704731B10C4BD3ED007AF8EEE77A80
:10DE1000C1ED007A72B1094BDFED096A1B68A3F509
:10DE2000D543333B07EE903AF8EEE77A87EEA67AD1
:10DE300082ED007A704700BFC8480020CC4800201F
:10DE40000000C842704700BF044B03EBC00040F223
:10DE5000FF739942A8BF194601857047385D0020BD
:10DE6000194B1A4A9B7982F88430032B21D9191F48
:10DE700002291AD8052B10B41DD0062B14BF4FF45D
:10DE80007A614FF47A519FED0E7B00241048114BBC
:10DE9000C2F89440B3FBF1F382ED267B5DF8044BAE
:10DEA000C2F88800C2F8903070470B4BC2F8883037
:10DEB00070470A4BFAE74FF4FA51E4E7AFF30080FA
:10DEC0000000000000000000083E0020385D002037
:10DED00049DE000840420F0045DE00083DE2000830
:10DEE000044B03EB8000D0F8A0300BB19B681960A5
:10DEF000704700BF385D0020084AD2F8E0305BB1BF
:10DF000040B19968B2F8E420054BB3FBF2F35B1023
:10DF10000B6070479B681860704700BF385D002039
:10DF200040420F000C4A13787BB10C4B93F8E6107B
:10DF300059B193F8E71059B150680021FA2883F8D5
:10DF4000E710A8BF4FF0FF3070476FF00100704737
:10DF50006FF00200704700BF5C090020385D0020B0
:10DF60000B4B93F8E8206AB193F8E9206AB10022DC
:10DF700083F8E920074B9868B0F5967FA8BF4FF06B
:10DF8000FF3070476FF0010070476FF0020070477C
:10DF9000385D00205C090020014B1B685B68184756
:10DFA00000430020014B1B689B681847004300207A
:10DFB000014B1B68DB68184700430020014BD86801
:10DFC000704700BF5C090020044B93F8EA3013B19E
:10DFD000034B186970476FF001007047385D0020EF
:10DFE0005C09002010B54A4C94F8EB30C0B24BB13C
:10DFF000484BD4F8EC201B689B1A0A2B84BF0023E3
:10E0000084F8EB3094F8EB30ABB9EE2809D1414AF3
:10E010001268C4F8EC20012284F8EB2084F8F03078
:10E0200010BDBB28FCD13B4B1B68C4F8EC3001236E
:10E0300084F8EB30F2E7012B10D194F8F03023B9DB
:10E0400084F8F10084F8EB30EAE7012BE8D10023F3
:10E0500084F8083184F807010223F3E7022BDFD1AB
:10E0600094F80831E218013382F8F10094F807219E
:10E07000DBB29A4284F80831D2D1002384F8EB3025
:10E0800094F80931012B31D1B4F9F320DFED226A84
:10E09000224B9FED236A07EE102AB8EEC77AC7EE2F
:10E0A000267AFDEEE77A17EE902A1A80B4F9F52069
:10E0B00007EE102AB8EEC77AC7EE067AFDEEE77AC9
:10E0C00017EE902A5A80B4F9F12007EE102AB8EE24
:10E0D000C77AC7EE267AFDEEE77A17EE902A9A8085
:10E0E00020F0C2FD002384F8093199E7022BF9D111
:10E0F00094F8F130094A03F003015172C3F381012E
:10E100001172C3F301119B09D1719371EAE700BF4A
:10E11000385D002024260020CDCCCC3F000101201A
:10E12000CDCCCCBF08B500684CF049F8014B9860E5
:10E13000012008BD385D002008B500684CF03FF8AC
:10E14000014BD860012008BD385D002038B5144669
:10E150000D46002944D0354A9FED356AD2ED437A09
:10E16000344BF8EEE77AB3F91410C7EE866A07EE7F
:10E17000901AB3F9101007EE101AF8EEE77AB8EE1D
:10E18000C77AB3F91210A6EEA77AD3ED027AF8EEA9
:10E19000E77AE6EE877A93ED017AB8EEC70AA6EE43
:10E1A000A70A07EE901AB3F90E10B3F90C3007EE78
:10E1B000101AF8EEE77AB8EEC77AA6EEA77A07EE5D
:10E1C000903AF8EEE77AE6EE877A92ED447AB8EE86
:10E1D000C77AC7EE066AA6EEA70A4FF097FE286038
:10E1E00014B3144BDFED126AB3F90020B3F9023017
:10E1F00007EE102A0D4AD2ED447AF8EEE77AB8EE2F
:10E20000C77A87EEA60A07EE903AF8EEE77AF6EEBE
:10E21000006A60EE277A9FED080AE7EE267A27EE7D
:10E22000800A4FF073FE2060012038BD385D002069
:10E230000000F04A6C4000200000C84210B50B4BB3
:10E2400003EBC00082B0446A01916CB107EE901AF2
:10E2500094ED047A94ED030AF8EEE77AA7EE870AC4
:10E260004FF054FEA368186002B010BD385D002066
:10E270002DE9F0410B4DDFF830802C686B690127E8
:10E280001C400CB9BDE8F081B4FA84F3C3F11F035C
:10E2900007FA03F658F823000368984724EA0604AF
:10E2A0006E61EEE7003C0140043C00202DE9F04F98
:10E2B0009B4D002605F58A7C95F85811A7B00A24D5
:10E2C0003246E646374605F5A87AA0E003EBC703D9
:10E2D00005EB4300C3F30726B0F85C01019646073F
:10E2E000DFB25FFA80FE4FEA102B40F1C98048068A
:10E2F00014D402F10209B9F18C0F41F0400100F28F
:10E30000008126A802F1010802444FF0040002F83F
:10E310008C0C26AA90444A4608F88C1C019802F1FD
:10E320000208B8F18C0F40F0020900F2EA8026A83A
:10E33000104400F88B9C4FF0050900F88C9C02F10A
:10E340000409B9F18C0F00F2DC8026AEB0444FF026
:10E35000060608F88C6C02F106084FEA8E0EB8F13A
:10E360008C0F00F8897C5FFA8EFE00F2CA8026AE20
:10E37000B1444FF0070609F88C6C00F887EC02F105
:10E38000080EBEF18C0F00F2BC8026AEB0444FF0F8
:10E390000509019E08F88C9C00F8856C02F10A06BC
:10E3A0008C2E00F2AE800DF19809CE444FF0060895
:10E3B0000EF88C8C00F8837C02F10C078C2F00F295
:10E3C000A0804E444FF0070006F88C0C0B324846F4
:10E3D000024402F88CBC3A465F09012003F01F0694
:10E3E00000FA06F65CF82700013C20EA06004CF82B
:10E3F000270000F089805E1CB6F5F07F80F08480F5
:10E4000073090CEB830ED6454FEA83077CD2DEF806
:10E4100000004FF0FF3306F01F0603FA06F606EA87
:10E42000000393FAA3F3B3FA83F3DBB2202B7FF458
:10E430004DAF0EF1040050451AD23A4BA3EB0E0734
:10E4400027F003070EF1080E774401E0B8420FD021
:10E4500006460430336893FAA3F3B3FA83F3DBB2CE
:10E46000202BF3D0A6EB0C0613EBC6037FF530AFE1
:10E4700085F858111046002A48D127B0BDE8F08F22
:10E480004E0603D401F03808F04515D021F078018C
:10E4900002F102080143B8F18C0FC9B231D826A8A5
:10E4A00002F1010E02444FF0040002F88C0C26AA7F
:10E4B000964442460EF88C1C901C8C2821D826AE1F
:10E4C00006EB020E019E0EF88B6C4FF005060EF85F
:10E4D0008C6C161D8C2E14D80DF1980840444FF00A
:10E4E000060800F88C8C0EF8897C971D8C2F08D8B4
:10E4F00026A806444FF0070006F88C0C053226A823
:10E5000066E76FF0004267E785F85811D5F85001CB
:10E5100003A94CF0DEF9012027B0BDE8F08F00BF61
:10E52000385D0020835E002037B583681C686379FE
:10E53000DB0724D5A57994F85C3205F001010D467E
:10E54000FBB1E06B43681A68D36AC3F34E035362AE
:10E5500094F86D32012B07D094F8613223B1B4F8EE
:10E5600068320133A4F8683285F001014AF078F985
:10E570000023A4F866324FF08073C4F85C3203B015
:10E5800030BD94F85F320191012B04BF94F85D32E5
:10E5900084F85E322046FFF7BDFB94F85F320199A4
:10E5A00053B9012384F85F3285EA0301E06B03B0BD
:10E5B000BDE830404AF054B9002384F85F32F5E7F3
:10E5C00010B5C14C04EB8003D3F8A0300BB19B68AD
:10E5D00019600F2822D8DFE810F02200310048002F
:10E5E00063007A009100AC00C300D500E400FB009A
:10E5F00016012D0144015F011000084627F024F8A0
:10E6000094F8313500F0070203F01F0343EA421388
:10E61000C0F3C70084F8313584F8320510BD0846D0
:10E6200027F012F894F81E3584F81D05C0F3022275
:10E6300023F00703134384F81E3510BD084627F066
:10E6400003F894F81E2594F81F3500F01F0102F01E
:10E650000702C0F3451023F03F0342EAC10218430A
:10E6600084F81E2584F81F0510BD084626F0ECFF2F
:10E6700094F81F2594F8213500F0030102F03F02C1
:10E6800042EA811223F00103C0F380210B43C0F35F
:10E69000870084F81F2584F8200584F8213510BDF3
:10E6A000084626F0D1FF94F8212594F8223500F091
:10E6B0007F0102F00102C0F3C31023F00F0342EA0E
:10E6C0004102184384F8212584F8220510BD08462C
:10E6D00026F0BAFF94F8222594F8233500F00F01B4
:10E6E00002F00F02C0F3061023F07F0342EA01128A
:10E6F000184384F8222584F8230510BD084626F027
:10E70000A3FF94F8232594F8253500F0010102F0C9
:10E710007F0242EAC11223F00303C0F341210B43FD
:10E72000C0F3470084F8232584F8240584F82535B0
:10E7300010BD084626F088FF94F8252594F8263564
:10E7400000F03F0102F00302C0F3841023F01F0326
:10E7500042EA8102184384F8252584F8260510BD75
:10E76000084626F071FF94F8263500F0070203F002
:10E770001F0343EA4213C0F3C70084F8263584F828
:10E78000270510BD084626F05FFF94F8293584F868
:10E790002805C0F3022223F00703134384F8293528
:10E7A00010BD084626F050FF94F8292594F82A3524
:10E7B00000F01F0102F00702C0F3451023F03F03F1
:10E7C00042EAC102184384F8292584F82A0510BDBD
:10E7D000084626F039FF94F82A2594F82C3500F0E5
:10E7E000030102F03F0242EA811223F00103C0F369
:10E7F00080210B43C0F3870084F82A2584F82B0579
:10E8000084F82C3510BD084626F01EFF94F82C2500
:10E8100094F82D3500F07F0102F00102C0F3C3101F
:10E8200023F00F0342EA4102184384F82C2584F8B0
:10E830002D0510BD084626F007FF94F82D2594F805
:10E840002E3500F00F0102F00F02C0F3061023F086
:10E850007F0342EA0112184384F82D2584F82E051F
:10E8600010BD084626F0F0FE94F82E2594F83035B9
:10E8700000F0010102F07F0242EAC11223F003031B
:10E88000C0F341210B43C0F3470084F82E2584F8E0
:10E890002F0584F8303510BD084626F0D5FE94F8D3
:10E8A000302594F8313500F03F0102F00302C0F347
:10E8B000841023F01F0342EA8102184384F83025B4
:10E8C00084F8310510BD00BF385D002010B5094C3B
:10E8D00094F84035012B05D0022B07D0064BC4F825
:10E8E000443510BD4BF0FEF8044BF8E74BF0FAF856
:10E8F000034BF4E7385D0020E1DE00087DCF02081D
:10E90000C1E5000808B5202152F03CFD034620B1C6
:10E910001A78202A00F10100F8D0184608BD2DE928
:10E92000F0410D461646044600274FF019082046D0
:10E93000FFF7E8FF044690B1FEF73EFE40F63402D2
:10E940004FF46171FDF7B2FAA0F5617090FBF8F039
:10E95000302804D84FB9287033780133337017B199
:10E960002046BDE8F0810127E1E76870F4E7244B19
:10E970001A6810B513460446B3FBF1F0B0F5803FBA
:10E9800003D3012BFAD95B08F6E781B22046FAF7E8
:10E99000A5FD23681B68587990B1032140B2FAF7AE
:10E9A000B7FC23681B685A7993F90530002B07DB05
:10E9B00002F01F0101228A405B09124941F823201D
:10E9C00023681B68987990B1032140B2FAF7A0FC44
:10E9D00023681B689A7993F90630002B07DB02F055
:10E9E0001F0101228A405B09064941F82320636820
:10E9F0001A6813889BB243F00103138010BD00BF57
:10EA0000D405002000E100E08160C06BAFE7154B4A
:10EA100053F8200070B508B3134D0C2202FB0052CE
:10EA200092F94935591C1AD092F85105B0B1E9183C
:10EA3000642491F8846592F85015002014226343F1
:10EA40005C1805EB4404013AB4F88845314410FAE7
:10EA500084F0F5D11423B0FBF3F080B270BD002038
:10EA6000FCE700BF00410020385D002038B50320DE
:10EA70000D461446FFF7CBFF07EE900A8DB19FEDD0
:10EA80000B7AF8EE677AF0EE006A67EE877AB8EEF6
:10EA9000047AA7EEA67ADFED067A67EE277AC5ED4F
:10EAA000007A0CB1034B236038BD00BF6740533A76
:10EAB00000007A443313904310B5427A044632B1D1
:10EAC0000146406851F80A3B98470023637210BD25
:10EAD00010B4447A621C0444D2B24272A172037A26
:10EAE000934202D85DF8044BE6E75DF8044B7047AB
:10EAF000EEE710B503681A79022A044602D1987A23
:10EB00004BF04EFB00232360237110BD73B50279D7
:10EB1000022A34D190F910301B4C8DF802201426B3
:10EB200006FB0343194E5B6900250120B3428DF8B3
:10EB300000508DF8010024D0154DAB4203D015488C
:10EB400083421CD1104602AA11441A8811F8085CAD
:10EB500022F040021204120C14211A8001FB004022
:10EB60001A88016A22F0380231F825101204120CBA
:10EB70000A431A801A8892B242F040021A8002B008
:10EB800070BD2846DFE700BF5C090020003001406F
:10EB900000380040003C0040C36910B5044623B96A
:10EBA0000C211420FEF7AAF8E061E06910BD10B551
:10EBB00004460068FFF7F0FF83783BB18388E38168
:10EBC000C388238203896382012010BD1846FCE7B5
:10EBD00038B500680D461446FFF7DEFFD0F8013067
:10EBE00007EE103ACDB1D0F80530DFED176A9FED92
:10EBF000176A07EE903AF8EE677A77EEE67A77EEE4
:10EC0000A77AC7EE866AF7EE007A76EEE77ADFED4E
:10EC1000106A67EEE67AC5ED007A9CB1DFED0D7AF9
:10EC2000DFED0D6AB8EEC77A27EE277AC7EE267AAF
:10EC30009FED0A7A77EEC77A9FED097A77EE877AA9
:10EC4000C4ED007A38BD00BF9AC9CC449AC94C467D
:10EC50000E76D7450000484300E0FF4400004842DC
:10EC6000339388430368DB6B13B504462BB92368E1
:10EC70005B6B3BB9FF23638202E098470028F6D123
:10EC800002B010BD214601A898470028F2D0BDF877
:10EC90000630013B9BB2EEE710B5036804469B6863
:10ECA000984701236373FF23A37310BD036810B556
:10ECB00004461B689847236820469B689847E37B77
:10ECC0000133E37310BD036810B504465B689847D1
:10ECD000236820469B689847E37B013BE37310BDA4
:10ECE000F0B585B0044618460D46164603934BF022
:10ECF000E9FE2268E67228440021A072009157695B
:10ED0000039B324629462046B84705B0F0BD03684C
:10ED10009B6A184738B504468B6801600D469847D2
:10ED20000B4BE360002323742B6B13B120469847F1
:10ED30002074084B93F8E0371BB1237C23F00103C8
:10ED40002374002363822046BDE838408AE700BF71
:10ED50000001FF00385D002003681B6803B11847FD
:10ED6000704703685B6803B11847704703681B6A04
:10ED700003B11847704703685B6A03B118477047CF
:10ED800030B40468A46A14B1A44630BC604730BCF7
:10ED9000704730B40468E46A14B1A44630BC6047DC
:10EDA00030BC704703685B6C03B118477047036859
:10EDB0009B6C03B11847704703689B6F03B11847FA
:10EDC00070470368D3F8803003B118477047036871
:10EDD000D3F8843003B1184770470368D3F88830FC
:10EDE00003B11847704721B10B68D3F88C3003B1D9
:10EDF00018470020704738B5094B052404FB003044
:10EE0000A0F1A00515F8010B013C4BF048F914F0F6
:10EE1000FF04F7D12046BDE838404BF040B900BFB1
:10EE20009018060810B5441E14F8010F00B910BD63
:10EE3000FFF7E1FFF8E7FFF71BBAFFF719BAFFF793
:10EE400017BAFFF715BAFFF713BAFFF711BA30B1C7
:10EE5000006800F13F4000F57E00800A70474FF0E7
:10EE6000FF30704728B18088B0FA80F0C0F11F00F1
:10EE700070474FF0FF307047F7B50646FFF7E7FFE2
:10EE8000194B18440C4690F8A302154649F04CFF64
:10EE90003046FFF7E7FF3768C0F3CC0307EB830387
:10EEA00000F00702196A92000F20904021EA000149
:10EEB0001962196A95400D431D62B388009304F0EE
:10EEC00003038DF80430C4F381038DF805306946DF
:10EED000C4F30013384664098DF806308DF80740F6
:10EEE000FAF790FE03B0F0BD901806082DE9F04F38
:10EEF00087B099469DF84430BDF840B00293CDE903
:10EF000000019046FDF734FF0646002800F0988087
:10EF10004E4F97F8E157052D00F28D805C2303FBDF
:10EF200005730022C3F8E42783F8E827009B1A79C9
:10EF3000130905EB450A6C1C013BC5EBCA01E4B2A1
:10EF400007F2E47A032B87F8E14702F00F020AEB9D
:10EF5000810A3ED83E49039331F8130040FA02F18A
:10EF6000CB0736D5012101FA02F2013A10404CF0EC
:10EF700003FC3849039B384A0B444FF0020C93F8CA
:10EF8000AC32184400EB400002EB8003019A9A7106
:10EF9000029A1C7283F807C000FA0CF4002A43D1CD
:10EFA00018460093FFF753FF084490F8A30249F076
:10EFB000BBFE009B284A998804914FF0011110591B
:10EFC000059104A9FAF71EFE234A009BA2589B88CC
:10EFD00053835C2303FB0575424649463046C5F81A
:10EFE000E467FAF77BFAD5F8E4075946FAF7CEFA60
:10EFF000D5F8E40743681A68B2F844306FEA43432F
:10F000006FEA53439BB2A2F8443013889BB243F09B
:10F0100001031380FAF7CAFB0023C5F8EC0703606D
:10F02000504607B0BDE8F08F009A6146127A184644
:10F03000FFF722FFCDE7094A00210420FDF798FDE4
:10F040004FF0000A504607B0BDE8F08F385D002051
:10F05000F0150608901806087839002010A4060854
:10F060002DE9F043824E96F8843083B00D46062B8E
:10F0700000F2F980DFE803F02DBD6393040404007F
:10F08000052B00F0E4807B497B4C062B08BF214612
:10F090004FF000090192CDF800900A461423042194
:10F0A000FFF724FF0746002800F0DB80804612228D
:10F0B00058F8140B414649F085FD0446002840F0FD
:10F0C000C880012406EBC5035F62204603B0BDE89B
:10F0D000F0830192694A6A4B1468A3FB04214FF63E
:10F0E000FF7202EBD112120CB4FBF2F4A3FB042367
:10F0F00000220092C3F3CF1322460421FFF7F6FE4D
:10F1000098B107EE904A9FED5F7ADFED5F6AF8EE07
:10F11000677A012367EE877A037127EE877AE7EE35
:10F12000667A80ED047AC0ED037A041E06EBC5030F
:10F1300018BF01245862204603B0BDE8F083019255
:10F140004E4A524B1468A3FB04214FF6FF7202EBA8
:10F15000D112120CB4FBF2F4A3FB042300220092A0
:10F16000C3F3CF1322460421FFF7C0FE0028DCD0F2
:10F1700007EE904ADFED466A9FED437A9FED456AC0
:10F18000F8EE677A012367EEA66A037127EE667AC6
:10F19000C0ED046AA7EE867A80ED037AC5E7019296
:10F1A0003D4B364A9B881268B2FBF3F101F57F4173
:10F1B000FF31090CB2FBF1F2B2FBF3F40023009330
:10F1C0000421A3B2FFF792FE0028AED007EE904ACA
:10F1D000DFED2C6A9FED2C7AF8EE677A012367EE5B
:10F1E000A67A037127EE677AC0ED047A80ED037A80
:10F1F0009BE70192214A254B1468A3FB04214FF69B
:10F20000FF7202EB9112120CB4FBF2F4A3FB042385
:10F2100000220092C3F38F1322460421FFF766FEFB
:10F22000002882D007EE904ADFED1C6A9FED157A28
:10F23000F8EE677A012367EEA67ADFED136A0371B1
:10F2400027EE877AE7EE667A80ED047A6BE7144959
:10F250001EE749464046482252F07DF801233B71A3
:10F2600030E704462EE706EBC50300245C622CE77A
:10F27000385D0020C0C62D00001BB700D40500205B
:10F280001F85EB516F12833A00007A44D34D621010
:10F2900077CCAB32ACC5A736083E00206F120339DD
:10F2A000808D5B002DE9F04F87B09B469DF8403084
:10F2B000019381468A469046FDF75AFD0446002890
:10F2C00000F09D80504D95F8E177052F00F2928077
:10F2D0005C2303FB07530022C3F8E42783F8E827E5
:10F2E00099F8042007EB470113097E1CC7EBC10105
:10F2F000013B05F2E470F6B200EB8101032B85F8C7
:10F30000E16702F00F0202913BD84049039331F8C4
:10F31000130040FA02F1CB0733D5012101FA02F2C2
:10F32000013A10404CF028FA3949039B394A0B4402
:10F3300040F2052C93F8AC32184400EB400002EB8D
:10F340008003019A1E72A3F806C08600002A4AD1E3
:10F3500018460193FFF77BFD084490F8A30249F09B
:10F36000E3FC019B2B4A998804914FF001119059BD
:10F37000059104A9FAF746FC264A019BB2589B88DE
:10F3800053835C2303FB0757234AC7F8E447B2FBC8
:10F39000F8F1204689B2FAF7A1F8D7F8E407594600
:10F3A000FAF7F4F8D7F8E40743681A68B2F844307B
:10F3B0006FEA43436FEA53439BB2A2F84430138889
:10F3C0009BB243F001031380FAF7F0F90023C7F86A
:10F3D000EC0705EB8A050360029BC5F8A03001200D
:10F3E00007B0BDE8F08F99F8082018460221FFF712
:10F3F00043FDC6E7094A00210420FDF7B9FB0020C0
:10F4000007B0BDE8F08F00BF385D0020F01506089A
:10F41000901806087839002040420F0010A4060812
:10F4200030B1036882881B691A4214BF0120002092
:10F43000704728B10368828809B11A8370475A83DC
:10F44000704710B1036882881A83704710B103684F
:10F4500082885A8370478379806BDB0748BF81F0CD
:10F46000010101B1EDE7F1E737B50C460546E8B11A
:10F47000FFF7EDFC0E4B184490F8A30249F054FC42
:10F48000AB88009304F003038DF80430C4F38103C8
:10F490008DF805302868C4F300136946C4F341149D
:10F4A0008DF806308DF80740FAF7ACFB03B030BD9D
:10F4B0009018060800B1DFE4704710B5837913F0A7
:10F4C000010F03F020020446C36B12D05B68002AD0
:10F4D0001A7A14BF02214221606BFFF7EBFF012172
:10F4E000E06B84F86012A4F85C12BDE81040FAF7F3
:10F4F00073B95B68002A18BF02211A7A08BF22215B
:10F50000EAE7036C806B1BB15B6801211A7AD1E7D3
:10F510000121A9E770B583681C6863799A0731D522
:10F5200094F86152D5B194F962329BB1B4F8641287
:10F530004B08A4F86432204601F00101FFF78BFF6D
:10F5400094F86232A279013B5BB2500684F86232D1
:10F5500018D5BBB9002384F8613213E0A36A626A4C
:10F5600094F860129A4226D161B9A3791B0709D594
:10F57000236CA06BDBB15B681A7AFFF79BFF204618
:10F58000FFF79BFF6379D90740F1818094F85C32E3
:10F59000002B7CD194F85D320133DBB2092B84F867
:10F5A0005D3235D12046BDE87040FEF7B3BB194649
:10F5B000FFF75AFFE3E75A1CA069A262C35C266901
:10F5C0005B0043F40073A4F864320A23B24234BFF0
:10F5D0001046284684F862320123A06284F8613222
:10F5E00091B1A3791E070FD5E06B2946FAF7F4F81D
:10F5F000E36B606B5B6829461A7AFFF75BFF84F860
:10F6000060522046FFF77DFFA3795D068BD4B9E7F2
:10F610000A2B3CD194F85F322BB9B4F8663243F030
:10F620000103A4F86632B4F86602820501D4C30768
:10F630001AD4B4F86A320133A4F86A3294F85F52EB
:10F6400001239D42A4F85C3221D1A179E06B002313
:10F6500084F85F3201F0010149F002F9E06B2946BC
:10F66000BDE87040FAF7B8B8E36AC0F3470013B1D9
:10F67000216B9847E2E7E3696269D054E369E26885
:10F680000133B3FBF2F102FB1133E361D6E770BD46
:10F6900010B50409013C032C00F00F0219D80E4BE1
:10F6A00033F8141041FA02F313F0010010D00123D3
:10F6B00003FA02F2013A02EA01004CF05DF8074A4F
:10F6C00014440C2294F8AC321844054B02FB003071
:10F6D00010BD0020FCE700BFF015060890180608D2
:10F6E000783900202DE9F04F3C2204460021B9482A
:10F6F00093B051F030FEB849621E033412F8013F56
:10F70000581E032888BF0023944241F8043BF5D1DA
:10F710000120FEF733F940B1B04B142283F8542591
:10F7200093F88425013283F884250220FEF726F918
:10F7300040B1AA4B152283F8602593F88425013245
:10F7400083F884250320FEF719F940B1A34B162254
:10F7500083F86C2593F88425013283F884250420EE
:10F76000FEF70CF940B19D4B172283F8782593F8EA
:10F770008425013283F88425994E964CDFF87082F7
:10F780004FF00F094FF0000A06F52C77207B38B3B5
:10F7900094F90D50FFF77CFF28B1072383710023F4
:10F7A00080F8079003721321FFF75EFE227B00238F
:10F7B00017F83310914240F0DC8006EBC303D3F816
:10F7C000B4322361182303FB0585AB6F23755A1CE4
:10F7D0000723A3750123AA67637585F874309A44DB
:10F7E00009F101095FFA89F9B9F1130F04F10C0469
:10F7F000CCD1BAF1000F00F0B9807A4CDFF8F49167
:10F800004FF00008237C002B00F0A6806079714D3A
:10F8100049F08AFA207949F087FAA068FAF76AF97C
:10F820000023CDE90E33CDE9103306930893236806
:10F83000A068CDF814904C330493E3680393636994
:10F840001422534307934FF480624FF40063CDE9D1
:10F8500009234FF400514FF48073CDE90B134FF49B
:10F86000003303A90D9349F083F9A268136843F0AC
:10F87000010313605C4A536823F4733323F4477322
:10F8800023F0030343F440335360226863695168F3
:10F89000012B21F04071D4BF0020012021F48071A0
:10F8A00041EA0021516090685049014041F0020155
:10F8B0009160D16A013B21F47001DBB241EA03534C
:10F8C000D3624FFA88F101239C4601914FF01F0E3D
:10F8D000697D51B395F90D100198814225D1297C9C
:10F8E000AE7D5F1C0929FFB249D9A1F10A00D2F807
:10F8F0000CA000EB40004FF0070B0BFA00FB2AEACC
:10F900000B0A06FA00F040EA0A00D060062B44D841
:10F91000013B506B03EB83030EFA03F620EA06006B
:10F9200001FA03F3034353633B460CF1010CBCF1B2
:10F93000050F05F10C05CBD1936843F40073936078
:10F94000936843F480739360936843F0010393607A
:10F95000936843F08043936008F10108B8F1030F06
:10F9600004F1180409F1C8097FF44CAF13B0BDE8E5
:10F97000F08F0133102B7FF41BAF002321E71069B8
:10F9800001EB410A4FF0070B0BFA0AFB20EA0B00D0
:10F9900006FA0AF630431061B8E70C2B0CD8073B87
:10F9A000106B03EB83030EFA03F620EA060001FA5C
:10F9B00003F303431363B7E70D3BD06A03EB830301
:10F9C0000EFA03F620EA060001FA03F30343D362BA
:10F9D000AAE700BF8062002000410020385D0020BF
:10F9E00090180608C009002000230140FDF7FFC061
:10F9F0005C090020C06200202DE9F74FAE4D009356
:10FA0000AE4B9D4221D26C798C4240F06D812C79B5
:10FA1000844202D0002840F06781EC79944240F0A3
:10FA200063812C68DCB11C220021201D51F093FC65
:10FA300025602B79237195F80690C4F808902A7AEE
:10FA4000E260012B03D0022B0DD0002407E0E87AFE
:10FA5000FFF71EFE6B7A2374AB7AA06163742046B5
:10FA600003B0BDE8F08FE87AFFF712FE95F9096060
:10FA7000A0612674A87AFFF70BFE6061002800F0F1
:10FA80002F818F4D4FF0140808FB0658D8F814301A
:10FA9000002B00F0258198F82630002B40F0C5801F
:10FAA00098F81C0049F040F998F81C3003F01F0248
:10FAB0005B090121023B01FA02F2032B08D8DFE8BF
:10FAC00003F0726C02667F490B6923EA02020A6145
:10FAD000142303FB0653587EFFF7DAFD731CDFB2D5
:10FAE000834618B140F60D32C2800772142202FB21
:10FAF0000652D07EFFF7CCFD824618B140F60D527B
:10FB0000C2800772142202FB0652907EFFF7C0FDEE
:10FB1000804618B140F60D42C2800772142303FBE1
:10FB2000065319F004095A7F019242D04A215846DF
:10FB3000FFF7C0FC019A2A215046FFF7BBFC019A4F
:10FB400040460A21FFF7B6FC142303FB0653019A33
:10FB500093F81880B8F1000F07D040460192FFF7E4
:10FB600097FD019A0921FFF7A5FC142303FB065317
:10FB70005A69554B9A4223D103F58433596A41F4AB
:10FB800080515962596A21F48051596225E04D49EA
:10FB90004B6923EA02024A619AE74A490B6A23EA5F
:10FBA00002020A6294E747494B6A23EA02024A6268
:10FBB0008EE70A215846FFF77DFC019A0A21BBE730
:10FBC000424B9A4240D103F50033196A41F4804117
:10FBD0001962196A21F480411962B9F1000F67D0E6
:10FBE000002108461388014303F44153194341F4AB
:10FBF00045711180938B23F400631B041B0C9383CA
:10FC00000723138213889BB243F040031380B8F19B
:10FC1000000F04D04046FFF73BFDFFF712FC142312
:10FC200003FB0655012385F82630606928B1009B47
:10FC300083710E23C371002303720921FFF714FCA3
:10FC40006069FFF7FEFB0AE7214B9A4209D103F5F1
:10FC5000FE33196A41F400411962196A21F4004126
:10FC6000BAE71C4B9A4209D103F58233596A41F431
:10FC700000515962596A21F4005186E7164B9A42A5
:10FC800009D103F56843596A41F480115962596AF0
:10FC900021F4801179E7114B9A429ED103F5644318
:10FCA000596A41F400115962596A21F400116CE754
:10FCB0000121022096E700BFA00100080803000808
:10FCC0005C0900200038024000300140003800404C
:10FCD000003C00400034014000500140005401400D
:10FCE0002046FEF706FFB0E60C358AE6064B53F8D1
:10FCF00020303BB19A881B6859690A4201D05A8367
:10FD000070471A83704700BFF8150608034B81F04F
:10FD1000010153F82000FFF78CBB00BFF81506085F
:10FD20002DE9F84F6A4FD7F80C0A037C03F0FF0C5B
:10FD3000002B40F0CB8097F8122A97F8133A97F8E7
:10FD4000149AA7F810CA07F6162EE2463C259EF82C
:10FD500002109EF80360C1F1FF0189B2002900F092
:10FD6000B180C1F1FF017143BEF80040B4FBF5FB67
:10FD70000912BBF1050F22D8DFE80BF0030E637404
:10FD80008593731A6343B3FBF5F353FA81F35FFA78
:10FD900081F9DBB2324610E0B4FBF5F205FB12420A
:10FDA00092B2C2F13C02741A6243B2FBF5F252FA0B
:10FDB00081F25FFA81F9D2B233464FF0010A16029E
:10FDC00046EA034646EA090600214FF001080CEB1B
:10FDD0000104C1F1170B08FA0BFBA4B21BEA060FD2
:10FDE00007EB8404414414BF4FF0020BC3461829AB
:10FDF000C4F898BAE9D10CF1180C1FFA8CFCBCF5C8
:10FE0000407F0EF1040EA2D13249A1F848C6BAF1E2
:10FE1000000F05D087F8122A87F8133A87F8149A4A
:10FE20002023A7F8103A91F84A36002B4ED040F222
:10FE30002A31F9F7E9FCD7F80C0ABDE8F84FF9F7D1
:10FE400017BDB4FBF5F305FB1344A6EB0109A4B2FF
:10FE5000CAB204FB09F9B9FBF5F959FA81F15FFA65
:10FE600081F9A9E7B4FBF5F305FB13439BB2C3F19A
:10FE70003C03741A6343B3FBF5F353FA81F3CAB23C
:10FE8000DBB2B14699E7B4FBF5F905FB1944721AE8
:10FE9000A4B26243B2FBF5F252FA81F2CBB2D2B213
:10FEA000EFE7B4FBF5F205FB124292B2C2F13C025D
:10FEB000741A6243B2FBF5F252FA81F2CBB25FFAE6
:10FEC00082F967E7B1463346324676E7BDE8F88FF8
:10FED000385D0020306E0020F8B500211820F9F7B9
:10FEE000E4FA054650B3FCF743FF1B4F0446C7F83E
:10FEF0000C0A18B31820FFF7CBFB184EC6F84C06B7
:10FF000020B140F21723C380002303722A7A4A21CA
:10FF1000FFF7D0FA124A03212046F9F7DFFAD7F8A3
:10FF20000C0A0021F9F732FB0E49D7F80C0A40F20F
:10FF30002A3248F047FE10B986F84A06F8BD09484B
:10FF400040F6A842002151F006FA012386F84A360D
:10FF5000BDE8F840E4E600BF385D0020306E0020C8
:10FF6000009F2400D0670020084B93F855214AB128
:10FF700093F8573113F0400F14BF4FF4F0704FF463
:10FF8000C37070474FF4F070704700BF385D0020B9
:10FF9000054B93F8550130B193F8573113F0400FEA
:10FFA0000CBF0D2010207047385D0020104A70B53E
:10FFB000002302F5707E4FF40056A2F1460501249D
:10FFC00032F8020F4FEA531CB0F5005F1CBF55F822
:10FFD0002C00168003F01F0104FA01F11CBF01433D
:10FFE00045F82C10724503F10103E9D170BD00BF43
:10FFF000925E00204FF01E0C43EA0223FF2A0CFB06
:020000040801F1
:1000000001011BB288BF43F00403B1F5F07F07DAAA
:100010000C4A02EB41009BB2B0F85CC19C4500D198
:1000200070474FEA511C02F58A72A0F85C3101F06A
:100030001F0152F82C30012000FA01F10B4342F865
:100040002C307047385D00204FF01E0C0CFB010176
:10005000B1F5F07F01DB002070470B4800EB410158
:10006000B1F85C11080AC9B210801970490709D5A6
:10007000118841F4807111801A7822F00402012065
:100080001A70704701207047385D00202DE9F04755
:100090001E2404FB010114788CB31D282FDC194E9B
:1000A0000FFA83FE06EB410CC1F10105483E012722
:1000B00001E01D2B23DCB1F5F07F4EEA042405EBB3
:1000C000010313D2BCF800A04FEA5119A24518BF92
:1000D000ACF8004001F01F0818BF56F8294007FA95
:1000E00008F81CBF44EA080446F8294012F8014FFA
:1000F000DBB20CF1020C03440131002CD9D1BDE874
:10010000F08700BF945E00202DE9F04F012885B0F4
:1001100014BF4FF0100B4FF01F0BCDE90212044635
:100120004FF00001584614BF4FF0110A4FF0230A58
:100130009946F9F7BAF980465846FFF7A9FADA4521
:100140009DF838609DF83C70054605D106F0030225
:10015000032A08BF47F0080717F00803009325D0CB
:10016000B8F1000F05D14FF0000A504605B0BDE8C8
:10017000F08F98F806205107F5D44046FCF7F8FDBB
:100180007F4B4FF41C7202FB0433C3F88C0600282B
:10019000E9D0C3F88856C3F88456631CDBB2002D3F
:1001A00044D040F20672EA802B723FE016F0010361
:1001B00001931FD000995046F9F777F90028D2D063
:1001C00082795207CFD4FCF7D3FD6D4A4FF41C71EE
:1001D00001FB042BCBF88C060028C4D05046FFF757
:1001E00057FA621CCBF88406D2B218B140F206610D
:1001F000C1800272B30719D5614A019B4FF41C7A82
:100200000AFB042ACAF88856002B40F09880B8F1FF
:10021000000FA8D04046FCF7ABFDCAF88C060028BA
:10022000A1D0631CDBB2002D40F09480544A5549A4
:100230004FF41C7B0BFB04FB02EB0B0502F5CA63BE
:10024000C5F850160BF15C011944029AC5F8641602
:100250000BF5AE714FF0000819444FF4807CC5F8DF
:100260007C26039AC5F88026D5F88C0685F8556655
:1002700085F85676C5F85CC6C5F86816C5F860C638
:100280004946C5F85896C5F87086C5F86C86C5F815
:100290007886C5F8748685F8BC48C5F8B888A5F88E
:1002A000B08803EB0B0AFEF762FB07F00101D5F8FB
:1002B0008C0648F0D5FA344B0BF1440716F0020FC8
:1002C0001F44324EA3F5CA6247D0D5F890060028E5
:1002D00043D0D5F88C36596843680968D3F800C014
:1002E0008C453AD0012285F8BD284946FEF73FFBF0
:1002F000274BD5F88C06C5F8A8363946C5F894A61C
:10030000C5F89866C5F89C86C5F8A0A6C5F8A48669
:10031000F9F79EF81C4BD5F890060BF150011944E3
:10032000F9F796F8009B33B95046FFF7EAF8012138
:100330005046FFF790F85046FFF7BFF815E74046E4
:10034000FCF716FDDAF88C36CAF89006002B7FF41D
:1003500068AF08E740F2065225E74FF41C7000FB37
:100360000422002382F8BD38094BD2F88C06C2F86B
:1003700094A6C2F89866C2F89C363946D0E700BF0A
:10038000306E0020C01B06088074002029E500089C
:1003900015F50008002ABCBF80185242002BBCBFD4
:1003A000C9185B420028BCBF121A0020F0B585189E
:1003B000CC180029A5F11D05BCBF234600210F3C28
:1003C000002DC8BF521B002CC8BF1B1B0A4E024485
:1003D0000B443C274FF0200C90420CDC06EB400510
:1003E0000C4604E007FB04FE013425F80EC09C42D5
:1003F000F8DD0130F0E7F0BD945E0020154B07B545
:100400001A6C42F080521A64134A01211162134A95
:10041000FF215162CA215162532151625B6FDB009F
:100420000AD5002301930E4B0193019B0193019B7D
:100430001A680C4B9A420AD000210120FAF726FCD8
:100440000849002003B05DF804EBFAF71FBC03B0C5
:100450005DF804FB0038024000000E420028004016
:100460005028004076614E692DE9F84F0026C0E91A
:100470000066544CDFF85881DFF8589105460F4666
:1004800098F80630022B2AD1E368580742BF23F0C0
:10049000040343F00803E360E368990604D523F0FE
:1004A000200343F04003E36001201FF069F850B3DC
:1004B000036843B3444A237992F83C1092F83D20F4
:1004C0009A421ED1414A334601210420FCF750FBD9
:1004D00001360B2E04F11404D2D1BDE8F88F012BA4
:1004E000E2D1E3681A0742BF23F0080343F0040394
:1004F000E360E3685806D7D523F0400343F02003B8
:10050000D1E78B42DED0D9F800A01AF0400F2BD0F3
:1005100000211120F8F7C9FF002183461020F8F7C9
:10052000C4FFBBF1000F04D0DBF8002023689A421F
:10053000C8D018B1026823689A42C3D00021232092
:10054000F8F7B3FF002183461F20F8F7AEFFBBF199
:10055000000F04D0DBF8002023689A42B2D018B113
:10056000026823689A42ADD01AF4803F08D0002177
:100570001820F8F79AFF18B1226803689A42A1D0B0
:100580002379143B032B9DD998F80120E3680AB125
:10059000032A0CD10FB119070ED413F0040F97D012
:1005A0002B685A1C2A60023345F8234090E75A060C
:1005B00002D413F0200FF2E76B685A1C6A6008330C
:1005C000F2E700BFF8040020AC0200204BA40608AC
:1005D0000C460020F4000120F7B5054616F0C0FCDB
:1005E0000C2804460CDD224B01221A700C23214AF0
:1005F0000093034600210420FCF7BAFA03B0F0BDD3
:10060000FDF72EFC1C4B9A791C4B03EB420393F82D
:1006100060333BB91A4A0221042003B0BDE8F04020
:10062000FCF7A6BA2B68A34219DB164F0835002643
:10063000A642E3DA3A6855F8040BF1B2C2F300724D
:10064000FEF70EFD014688B9094B05221A700E4AC5
:100650003346042003B0BDE8F040FCF789BA044AF1
:10066000032111700093094A2346C3E70136DFE7EF
:10067000143E002063A40608083E002090180608D7
:100680008FA40608F4000120E6A40608ADA406081D
:100690002DE9F3412E4B1C78064634B12D4B93F8CF
:1006A000304B93F8313B0134E41A2B4B1B783BB9A8
:1006B0002A4A0221042002B0BDE8F041FCF758BAF2
:1006C000102C0DDD264B02221A701023254A0093B0
:1006D000002123460420FCF74BFA02B0BDE8F0816C
:1006E000214FFEF7F3F897F8401511F0FD0101D006
:1006F0001E4ADEE77368A34220DBDFF87C802036E9
:100700000D46A542E9DAD8F80030B7F83A25C3F328
:1007100000730093E9B2B7F8383556F8040BFEF7CA
:10072000C1FD014688B90E4B05221A70104A2B46AE
:10073000042002B0BDE8F041FCF71ABA084A0420D0
:10074000107000930B4A2346C5E70135D9E700BF77
:10075000043E0020306E0020063E00200BA5060857
:10076000143E002025A50608385D002051A5060886
:10077000C3A506088DA50608F4000120024B00223F
:1007800083F8AC20704700BF5C090020024B0122B7
:1007900083F8AC20704700BF5C090020044A054B79
:1007A00092F8842003EB420393F86103704700BF83
:1007B000385D0020901806081049114B91F88420EC
:1007C00003EB420393F8613303B9704710B50D4B47
:1007D0001C788CB12431002301EBC00C4FF0010ECA
:1007E00051F833202AB112791AB1984208BF8CF817
:1007F00006E001339C42F3D110BD00BF385D0020FC
:1008000090180608D801012010B5154CD4F8442BD7
:10081000D4F8483BD4F83C1B82B002FB03F38B4274
:100820008DF807001AD0D4F8383BD4F8400B0DF1FE
:100830000701184450F056FBD4F8383BD4F8442B49
:10084000D4F83C1B1344D4F8482BB3FBF1F001322D
:1008500001FB1033C4F8383BC4F8482B02B010BD7C
:10086000306E00200B4B10B4002203F64C340820ED
:100870000121C3F8404BC3F83C0B5DF8044BC3F8AF
:10088000441BC3F8342BC3F8382BC3F8482BC3F8E8
:10089000582B7047306E00200F4B93F88430062B96
:1008A00017D8DFE803F00416070A0D1013004FF401
:1008B000C87070474FF4FA607047084B98887047CB
:1008C0004FF47A6070474FF4FA5070474FF47A5003
:1008D00070474FF47A707047385D0020083E002062
:1008E000044B03EBC000406A10B103685B681879E1
:1008F000704700BF385D0020034BD3F8442512B188
:100900000F2800D810477047385D002010B53F20F1
:10091000FEF7BEFE044678B140F223230121C380D6
:100920000172FEF7A1FD2046FEF790FD0E4B00225E
:10093000C3F85C4BA3F8602B2A20FEF7A9FE0446FF
:1009400080B140F22323C380022303720121FEF70A
:100950008BFD2046FEF77AFD034B0022C3F8644B63
:10096000A3F8682B10BD00BF306E002050B10138D5
:10097000002330F0FF019AB203F1010303D140EAF2
:10098000022080B270474008F3E703681B681847ED
:100990002DE9F041134E144B07460C46D6F87C0B5C
:1009A0004FF00008AA21154683F8EB80FFF7EDFF12
:1009B000D6F87C0B4146FFF7E8FFD6F87C0B3946AA
:1009C000FFF7E3FF2946D6F87C0BFFF7DEFF25444F
:1009D00014F8011BD6F87C0BFFF7D7FFAC42F7D118
:1009E000BDE8F081306E0020385D002007B501229F
:1009F0008DF8041001A9FFF7CBFF03B05DF804FBED
:100A000070B50E4C0E4B002206460D46D4F87C0BFA
:100A100083F8EB20AA21FFF7B8FFD4F87C0B012163
:100A2000FFF7B3FFD4F87C0B3146FFF7AEFFD4F8E5
:100A30007C0B2946BDE87040A7E700BF306E002060
:100A4000385D002038B505460C4614F8011B01B985
:100A500038BD2846FFF799FFF7E703685B6818473A
:100A600003689B6818470368DB6970B506460C4647
:100A7000154683B1BDE8704018473046FFF7F0FFD8
:100A80000028FAD014F8011B3046FFF77EFF2B1B1D
:100A9000002BF2DC70BD0D44F9E7E4E70368DB6886
:100AA000184703681B69184703685B6918470368A0
:100AB0009B6A03B1184770470368DB6A03B11847A4
:100AC0007047074B9B7A01460BB1FDF715BA054BF2
:100AD0001868054B1B780BB981F00101FEF7A9BC22
:100AE000E43E0020DC3E0020E03E002072B6002202
:100AF0004FF0FF31930003F1604303F5614301328E
:100B0000082AC3F88010C3F88011F3D1BFF34F8FC8
:100B10000549064BCA6802F4E0621343CB60BFF399
:100B20004F8F00BFFDE700BF00ED00E00400FA05B5
:100B3000012108B50846FAF7A9F8FFF7D7FF07B56E
:100B40000B4B002101910193019B04330193019B05
:100B50001868012808D1FAF799F8064B1A6882F349
:100B600008885B689847FEE703B05DF804FB00BFA8
:100B7000502800400000FF1FEFF31183102282F382
:100B8000128809490A6801320A604FF0E0220749D9
:100B90009069C1F8800B0020C1F8840B1269DBB2A8
:100BA00083F31188704700BF24260020306E002098
:100BB000064A074B51681B6858434FF47A73B0FBE1
:100BC000F3F053685B1A8342FBD97047001000E0D2
:100BD0001C2E002010B504464FF4FA70FFF7E8FF12
:100BE0006069BDE81040FEF72CBC73B5104B15468C
:100BF00090F910200446142000FB02335E69A368BC
:100C00009A0704D46069019149F0C2FA019930460B
:100C100049F084FE2946304649F080FEA3689B07D0
:100C200002D42046FFF7D6FF012002B070BD00BFFE
:100C30005C0900207FB50379012B0D460AD0022BF9
:100C400019D18368DB0758BF01F07F0104B0BDE80C
:100C50007040CAE781688DF80F2001F001010DF1A5
:100C60000F0200920191417C90F910002A46F9F799
:100C7000B1FE04B070BD0020FBE708B53122F421BD
:100C80000068FFF7D7FF012008BD00680122582146
:100C9000D0E7006801224821CCE700680222082141
:100CA000C8E7006801220821C4E710B50446002205
:100CB00021210068FFF7BEFF2068FC222021FFF7FA
:100CC000B9FF206840222421FFF7B4FF20680C22DE
:100CD0002321FFF7AFFF206800222221FFF7AAFFA0
:100CE000012010BD10B5012204460B210068FFF75A
:100CF000A1FF20B120681D220921FFF79BFF00F012
:100D0000010010BD034B0246D3F8880B08B18021C7
:100D100090E77047306E002010B5B020FFF7F2FF6B
:100D20004020FFF7EFFF0020FFF7ECFF1020FFF758
:100D3000E9FF4FF48064013C0020A4B249F0AFF910
:100D4000002CF8D110BD503910B50446C8B2FFF7D9
:100D5000D9FF04EB4400400004EB440400F00E0013
:100D6000FFF7D0FFC4F3C3001030BDE81040C9E75F
:100D700008B55038C0B2FFF7C5FF0020FFF7C2FF2B
:100D8000BDE808401020BDE738B5002222233221FB
:100D90000120FEF731FE3D4BC3F8880B10B900244B
:100DA000204638BDAE20FFF7ADFF04460028F6D040
:100DB000D420FFF7A7FF8020FFF7A4FFA820FFF7AC
:100DC000A1FF3F20FFF79EFFD320FFF79BFF0020EE
:100DD000FFF798FF4020FFF795FF8D20FFF792FF68
:100DE0001420FFF78FFFA120FFF78CFFC820FFF72B
:100DF00089FFDA20FFF786FF1220FFF783FF8120AB
:100E0000FFF780FFCF20FFF77DFFD920FFF77AFFA4
:100E1000F120FFF777FFDB20FFF774FF4020FFF79B
:100E200071FFA420FFF76EFFA620FFF76BFFAF2036
:100E3000FFF768FFA620FFF765FFAE20FFF762FF10
:100E40002020FFF75FFF0020FFF75CFFB020FFF7D7
:100E500059FF4020FFF756FF0020FFF753FF1020F7
:100E6000FFF750FF4FF48065013D0020ADB249F01F
:100E700016F9002DF8D18120FFF744FFC820FFF7B5
:100E800041FFAF20FFF73EFF8AE700BF306E002032
:100E900008B5FFF7CFFE014B187008BD5C090020B4
:100EA000F7B515461E4690F91020104B0446142045
:100EB00000FB02335F69A3689A0704D4606901915B
:100EC00049F066F90199384649F028FD33462A462B
:100ED0000021384649F0D2FCA3689B0702D4204683
:100EE000FFF778FE012003B0F0BD00BF5C090020D1
:100EF000F7B50779012F16460AD0022F15D184685D
:100F0000E40758BF41F0800103B0BDE8F040C7E7F7
:100F1000826802F00102CDE900620A46417C90F944
:100F20001000F9F757FD03B0F0BD0020FBE707B54F
:100F3000130A8DF804308DF80520022301AAFFF76B
:100F4000D7FF024B187003B05DF804FB5C0900206A
:100F500010B50A4C002384F88C3B84F88D1B84F870
:100F60008E2B032304F68C32FF21FFF7C1FF0028EC
:100F70000CBF6FF00C00002010BD00BF306E0020D1
:100F800010B50B4C002384F88C3B130A84F88D1B9E
:100F900084F88E3B84F88F2B042304F68C32FF21D7
:100FA000FFF7A6FF00280CBF6FF00C00002010BD5B
:100FB000306E0020024A00680023512198E700BFEC
:100FC000BC7A0020F7B515461E4690F91020104B4C
:100FD0000446142000FB02335F69A3689A0704D417
:100FE0006069019149F0D4F80199384649F096FCBE
:100FF000334600222946384649F040FCA3689B0747
:1010000002D42046FFF7E6FD012003B0F0BD00BF8B
:101010005C090020F7B50779012F16460AD0022F88
:1010200015D18468E40758BF41F0800103B0BDE8E2
:10103000F040C7E7826802F00102CDE900620A468B
:10104000417C90F91000F9F7EBFC03B0F0BD0020F3
:10105000FBE738B504460068FDF79EFD0D23054605
:10106000C21C0C212068FFF7D5FFA87028B16B893E
:101070002384AB896384EB89A38438BD13B5032330
:101080000C46006801AA2221FFF7C4FF30B1BDF968
:10109000053003EB83031B12E633238002B010BD3F
:1010A00037B50623F7210068154C6A46FFF7B2FFF3
:1010B0001449E8B19DF801209DF800309DF80350D7
:1010C000120142EA03329DF8023042EA13129DF8FF
:1010D00004304A601B0143EA05339DF80550C4F80B
:1010E0008C2C43EA15130B60C4F8903C03B030BD60
:1010F000D4F88C3C4B60D4F8903C0B60F6E700BF12
:10110000306E0020385D002007B50323006801AA77
:101110001946FFF77FFFA0B19DF804309DF8051038
:101120009DF904201B0443EA01239DF80610002AC0
:10113000B4BF4FF07F4200220B431343024AC2F870
:10114000103103B05DF804FB385D002007B50323C0
:10115000006801AA0021FFF75DFFA0B19DF80430EF
:101160009DF805109DF904201B0443EA01239DF816
:101170000610002AB4BF4FF07F4200220B431343F6
:10118000024AC2F80C3103B05DF804FB385D002060
:1011900013B5044600680379022B0CBF43210321D9
:1011A00006236A46FFF736FF18B9E086A06302B04F
:1011B00010BDBDF800305BBAE386BDF802305BBA03
:1011C0006387BDF804305BBA2387F0E713B50623C5
:1011D00004466A4600681121FFF71CFF18B9E08633
:1011E000A06302B010BDBDF9003007EE103AB8EEB2
:1011F000C77AF7EE086A27EE267ABDEEC77A17EEB1
:10120000103AE386BDF9023007EE103AB8EEC77A1D
:1012100027EE267ABDEEC77A17EE103A2387BDF97E
:10122000043007EE903AF8EEE77A67EEA67AFDEE24
:10123000E77A17EE903A6387D3E713B50023C386A6
:1012400083630446062300686A460321FFF7E2FE33
:1012500078B1BDF8003003EB4303E386BDF90230FB
:101260005B4203EB43032387BDF8043003EB4303E6
:10127000638702B010BD07B5012301AAFF210068F2
:10128000FFF7C8FE03B05DF804FBF7B5054600683C
:10129000FDF782FC00230370042304460DEB0302D8
:1012A0002868FF21FFF7B6FE10B9002003B0F0BD9B
:1012B000286804236A46FF21FFF7ACFE0028F4D01B
:1012C0009DF804108A09023A012AEED99DF80020FF
:1012D0009DF805309DF8015003EB012305EB022535
:1012E000C3F30D03C5F30D055A1B002AB8BF5242C4
:1012F000FF2ADADC9DF806109DF807209DF80270A1
:1013000002EB01229DF8031001EB07214911561150
:10131000C1EB5212002AB8BF5242FF2AC5DC01229B
:101320002B443144134111412270C4F80530C4F8F4
:101330000110BBE707B5022301AAFFF76BFE044BC0
:101340001870BDF8040040BA80B203B05DF804FB29
:101350005C09002038B515460D4A0B0A82F88C3B13
:1013600082F88D1B022302F68C32FF210446FFF720
:10137000BFFD10B96FF00C0038BD01232A46FF21D4
:101380002046FFF747FE0028F4D00020F4E700BF16
:10139000306E0020F8B5124D164685F88D1B05F607
:1013A0008C3200240223FF21074685F88C4BFFF77F
:1013B0009FFD05F68C3210B96FF00C00F8BD0223CA
:1013C000FF213846FFF726FE0028F5D095F88C2B34
:1013D00095F88D3B03EB022333802046EEE700BFF8
:1013E000306E00202DE9F341754D0468DFF8DC8193
:1013F0000023064685F8E8302D27B9B218F8012BEE
:1014000020460137FFF7A4FD882FF6D1402287211F
:101410002046FFF79DFD00238DF806300DF10601F3
:10142000204648F0A0FD9DF80630002BF6D00122A2
:1014300086212046FFF78CFD002287212046FFF7FA
:1014400087FD092208212046FFF782FD00220B219B
:101450002046FFF77DFD002853D137680DF10602C5
:101460005E213846FFF796FFBDF80630B3F5D77F0B
:1014700000F0A18055D8512B00F09B8049D81D2B3E
:101480006CD01E2B00F095803068212148F0DAFCEA
:1014900034680DF10602DE212046FFF77BFFBDF820
:1014A00006309FED487AC3F309032822ADF80630D1
:1014B000534307EE903AF8EEE77A434A67EE877AAD
:1014C0000021FCEEE77A82F88C1B17EE903A6C2133
:1014D00082F88D1B190E82F88E1B190C82F88F1B57
:1014E000190A82F8901B82F8913BFF2102F68C3298
:1014F00006232046FFF7FCFC306840228721FFF7D7
:1015000027FDB0FA80F0400985F8E80002B0BDE898
:10151000F081AD2B4FD0D62B01D0602BB4D121243C
:101520001DE040F2E132934247D00CD840F2D9227C
:10153000934242D040F2E122934202D0B3F5E67FDB
:10154000A2D164240BE040F28F42934203D040F2D8
:101550009152934298D14FF4FA7400E00F2400287E
:1015600092D10A224B213846FFF7F2FC0F2260216C
:101570003846FFF7EDFC0D2263213846FFF7E8FC03
:10158000B82269213846FFF7E3FC40F60D72782156
:101590003846FFF7F5FC40F60E627A213846FFF731
:1015A000EFFC00287FF470AF2146384648F04AFC33
:1015B0006AE71424D3E73224D1E7C824CFE700BF79
:1015C000385D00209A99893F306E0020FE1B060886
:1015D00037B5124D95F8E8300446E3B100680DF1D7
:1015E000050148F0C0FC9DF805307BB10DF1060205
:1015F00020689621FFF7CEFE0A22BDF80630B3FB25
:10160000F2F3074A9360012385F8E930206801224C
:101610008621FFF79DFC03B030BD00BF385D002080
:101620005C09002013B5022301AA04465121006879
:10163000FFF7F0FC114AF0B1BDF804305BBA9BB281
:10164000D360D368B3F5C87F02DD4FF0FF33D360BA
:101650000B4B0C4A1968D2F8943C32338B4208D2B7
:10166000C2F8941C2068002302F68C425121FFF737
:101670003FFC02B010BD6FF00103E8E75C090020F9
:1016800024260020306E002007B50223006801AA3E
:101690000021FFF7BFFC0F4B83F8EA00B0B1BDF8A3
:1016A00004300D4A5BBA9BB2B3F5FA6F3FBF0A2113
:1016B000B3FBF1F307EE903AF8EEE77A2BBF4FF069
:1016C000FF33FDEEE77A1361C2ED047A03B05DF8F3
:1016D00004FB00BF385D00205C09002013B5022325
:1016E0000C46006801AA0021FFF794FC60B15CB1D0
:1016F0009DF805309DF90420DB0903EB830302EB21
:10170000820203EB4203238002B010BD73B5114B7C
:10171000154690F910200446142000FB02335E6940
:10172000A3689A0704D46069019148F031FD0199DA
:10173000304649F0F3F8012300222946304649F0AB
:101740009DF8A3689B0702D42046FFF743FA0120C7
:1017500002B070BD5C09002073B50379012B1646F9
:101760000AD0022B15D18368DB0758BF41F08001F6
:1017700002B0BDE87040C9E7826802F00102CDE91D
:1017800000620A46417C90F91000F9F749F902B06D
:1017900070BD0020FBE730B5002385B00446C3864A
:1017A00083630DF1070200680221FFF7D5FF18B926
:1017B0000025284605B030BD9DF80730DB07F7D57A
:1017C000062302AA03212068FFF724FC20680DF1FC
:1017D00007020921FFF7C0FF05460028E8D09DF861
:1017E000073013F00C0FE3D1BDF808302068C3EBCD
:1017F00083339B00E386BDF80A309B002387BDF846
:101800000C30C3EB83339B00638701220A21FFF76F
:1018100011FACEE71FB50446002300688DF80730A3
:101820000DF107022721FFF797FF68B19DF80730F8
:1018300013F0080320D02068062302AA2821FFF70E
:10184000E9FB18B9E086A06304B010BDBDF908300B
:10185000002BB8BF03339B10E386BDF90A30002B81
:10186000B8BF03339B102387BDF90C30002BB8BFE2
:1018700003339B106387E7E71846E5E71FB50021B0
:101880000446C18681630DF107020068FFF764FF1B
:10189000C0B19DF8073013F0080315D02068062367
:1018A00002AA0121FFF7B6FB60B1BDF808305BBAB0
:1018B000E386BDF80A305BBA2387BDF80C305BBA0B
:1018C0005B42638704B010BD1846FBE730B50025C6
:1018D00085B00446C58685630DF1070200680621C0
:1018E000FFF73AFFA0B19DF8073013F0040311D0C1
:1018F0002068062302AA2946FFF78CFB40B1BDF8F9
:101900000830E386BDF80A302387BDF80C306387C2
:1019100005B030BD1846FBE707B50DF10702FFF72C
:101920001BFF034B18709DF8070003B05DF804FB24
:101930005C090020F8B5144E144F41F0010200215B
:101940000446FFF7A5FA3568C7F8985C13212046CE
:10195000FFF7E2FF10F007000BD001220B21204619
:10196000FFF796FA002220461146FFF791FA012070
:1019700008E0D7F89C2C002AE8D033689BB25B1BA8
:101980009A42E3D2F8BD00BF24260020306E00202A
:1019900010B50C460121FFF7BFFFC0F30013237001
:1019A000C0F3C003A370C0F380036370C0F380135F
:1019B000C0F3C010E370207110BD2DE9F0478846D8
:1019C000502114460646FFF7A7FF01304000C0B281
:1019D000208046213046FFF79FFF2D4F23780130AE
:1019E00080B27B434FF47A79A08003F5FA734FF409
:1019F000FA6AB3FBF9F25121B3FBFAF300FB0233AD
:101A00003046B3FBF9F3E360FFF794FCC3B2C0F3D5
:101A10000F22257803FA02F2013293B27D43E3806C
:101A200005F5FA723046B2FBF9F1B2FBFAF203FBAC
:101A300001227021B2FBF9F22282FFF76DFF013023
:101A40004000C0B2608071213046FFF773FCC3B222
:101A5000C0F30F208340013398F803209BB2238109
:101A600012B1E2889B1A2381A37820897B4303F576
:101A7000FA734FF47A724FF4FA65B3FBF2F1B3FBE9
:101A8000F5F300FB0133B3FBF2F36382BDE8F087AB
:101A9000002F3A002DE9F047DA4FDFF87083DFF8C6
:101AA00070934FF4FA738CB00446002689210068C5
:101AB000C7F89C3C88F8E660FFF72EFF40F0010075
:101AC000C2B289212068FFF7E3F9324620688821F5
:101AD000FFF7DEF9206801228021FFF7D9F920689D
:101AE0000122FF21FFF7D4F9324631462068FFF783
:101AF000CFF991212068FFF70FFF314687F8A00C3E
:101B000001222068FFF7C4F932462068FF21FFF761
:101B1000BFF9324620688021FFF7BAF960212068BA
:101B2000FFF7FAFE40F01200C2B260212068FFF712
:101B3000AFF9206820224421FFF7F9F92068FF223D
:101B40000121FFF7A5F92568012280212846FFF72A
:101B50009FF90122FF212846FFF79AF932463146C4
:101B60002846FFF795F90622FF212846FFF790F94E
:101B700083212846FFF7D0FE40F00400C2B2832143
:101B80002846FFF785F90722FF212846FFF780F94D
:101B9000012281212846FFF77BF901228021284676
:101BA000FFF776F96B2294212846FFF771F9324648
:101BB00083212846FFF76CF9D9F80060C7F8986CC4
:101BC00083212846FFF7A8FE002800F05083012259
:101BD00028468321FFF75CF992212846FFF79CFEF7
:101BE0000022C0F3C716814681212846FFF750F92D
:101BF00006222846FF21FFF74BF983212846FFF7ED
:101C00008BFE832100F0FB022846FFF741F92846AE
:101C10000122FF21FFF73CF9284601220021FFF7AE
:101C200037F928460022FF21FFF732F92846002223
:101C30008021FFF72DF9062305AAB0212068FFF7C0
:101C4000E9F920680122FF21FFF722F9206800222C
:101C50004F21FFF71DF920682C224E21FFF718F9BC
:101C600020680022FF21FFF713F9B4222068B62173
:101C7000FFF70EF90025002E18BF0C2609F07F098A
:101C80002A464FF0010C0CABC5F3C4005FFA85FE89
:101C90001844764510F81C3C05F0070102D8914520
:101CA00040F0F0820CFA01F123EA010300F81C3C39
:101CB0000135302DE7D1062305AAB0212068FFF7B2
:101CC00017F9514B01221870FF212068FFF7E0F847
:101CD000002211462068FFF7DBF820680022FF2170
:101CE000FFF7D6F8206800220921FFF7D1F8206815
:101CF00000221021FFF7CCF8206800221121FFF705
:101D0000C7F8206801222421FFF7C2F82068FF22CB
:101D10002521FFF7BDF8206800227521FFF7B8F8EC
:101D200020680122FF21FFF7B3F820682C224E2102
:101D3000FFF7AEF8206800224821FFF7A9F82946EE
:101D400020682022FFF7A4F820680022FF21FFF777
:101D50009FF8294620680922FFF79AF82068002298
:101D60005421FFF795F8206804223121FFF790F8FD
:101D7000206803223221FFF78BF82068832240215C
:101D8000FFF786F8206825224621FFF781F82068B2
:101D900000226021FFF77CF8206800222721FFF74E
:101DA00077F8206806225021FFF772F82068002299
:101DB0005121FFF76DF8206896225221FFF768F84D
:101DC000206808225621FFF763F82A462068572129
:101DD000FFF75EF8206800226121FFF759F82068BC
:101DE00000226221FFF754F8206800226421FFF7E7
:101DF0004FF8206800226521FFF74AF82068A022EA
:101E0000662107E0306E00205C090020385D00206C
:101E100024260020FFF73CF820680122FF21FFF76D
:101E200037F8206832222221FFF732F82068142286
:101E30004721FFF72DF82068FF224921FFF728F8F6
:101E4000206800224A21FFF723F820680022FF21A2
:101E5000FFF71EF820680A227A21FFF719F8206898
:101E600000227B21FFF714F8206821227821FFF758
:101E70000FF820680122FF21FFF70AF820683422BA
:101E80002321FFF705F8206800224221FFF700F820
:101E90002068FF224421FEF7FBFF2068262245210F
:101EA000FEF7F6FF206805224621FEF7F1FF4022EB
:101EB00011462068FEF7ECFF206806220E21FEF78F
:101EC000E7FF20681A222021FEF7E2FF2068402267
:101ED0004321FEF7DDFF20680022FF21FEF7D8FF37
:101EE000206803223421FEF7D3FF206844223521E5
:101EF000FEF7CEFF20680122FF21FEF7C9FF206810
:101F000004223121FEF7C4FF206809224B21FEF78D
:101F1000BFFF206805224C21FEF7BAFF206804228B
:101F20004D21FEF7B5FF20680022FF21FEF7B0FF2C
:101F3000206800224421FEF7ABFF206820224521C3
:101F4000FEF7A6FF206808224721FEF7A1FF2068C0
:101F500028224821FEF79CFF206800226721FEF717
:101F600097FF206804227021FEF792FF206801226B
:101F70007121FEF78DFF2068FE227221FEF788FF97
:101F8000206800227621FEF783FF20680022772157
:101F9000FEF77EFF20680122FF21FEF779FF20680F
:101FA00001220D21FEF774FF20680022FF21FEF7B9
:101FB0006FFF206801228021FEF76AFF2068F82267
:101FC0000121FEF765FF20680122FF21FEF760FF77
:101FD000206801228E21FEF75BFF2068012200218C
:101FE000FEF756FF20680022FF21FEF751FF206810
:101FF00000228021FEF74CFF042220680A21FEF710
:1020000047FF256884212846FFF786FC842100F0DD
:10201000EF022846FEF73CFF012220680B21FEF765
:1020200037FF2068019003A9FFF7B2FC019807AAC7
:1020300003A9FFF7C2FC9DF80C30002B00F02881AB
:102040000A9D05F684559DF80E30002B00F0238183
:102050000A9B03F2B22305EB43059DF80F3023B131
:10206000BDF82C3003F525731D449DF8103023B1C5
:10207000BDF82E3003F226231D442068C7F8A45C67
:10208000E8220121FEF704FF44F61F639D4203D9B5
:102090002068294647F087FF012220681146FEF795
:1020A000F7FE20684021FFF745FC002800F0E7809C
:1020B000206801210222FEF7EBFE20680021FFF7D5
:1020C00039FC002800F0DB802068DFF8E491E8228A
:1020D0000121FEF7DDFE202220684421FEF727FFC4
:1020E000256803A92846FFF753FC07AA03A9284639
:1020F000FFF763FC502257212846FEF7C9FE08224D
:1021000056212846FEF7C4FE082250212846FEF735
:10211000BFFEBDF82C004FF47A7A48F20E660AFB37
:102120000060B0FBF9F080B2FEF720FC51210246BE
:102130002846FEF7FCFE0A9A5C4B0AFB02669E42AA
:102140009DBFB6FBF9F202F1FF32D2B2FF22462167
:102150002846FEF79DFED7F8A41C44F61F6399425B
:1021600002D9284647F01FFF01212846FFF7D4FB7C
:102170000222064601212846FEF78AFE0021284653
:10218000FFF7D8FB324601212846FEF781FE24687E
:1021900003A92046FFF7FCFB07AA03A92046FFF787
:1021A0000CFC482211462046FEF772FE0822472109
:1021B0002046FEF76DFE032232212046FEF768FE20
:1021C000072230212046FEF763FE0122FF21204630
:1021D000FEF75EFE202230212046FEF759FE002247
:1021E000FF212046FEF754FE062220467021FEF70E
:1021F0004FFEBDF82E304FF47A7246F6440002FBD3
:1022000003004DF28803B0FBF3F09DF80F3080B26D
:102210001BB1BDF82230184480B2FEF7A7FB712134
:1022200002462046FEF783FED7F8A41C44F61F633F
:10223000994202D9204647F0B6FE01212046FFF719
:102240006BFB0222054601212046FEF721FE0021FC
:102250002046FFF76FFB2A4601212046FEF718FEB5
:102260006423C7F89C3C012388F8E63007E0D9F8DE
:1022700000309BB29B1BB3F5FA7F7FF6A1AC0CB08C
:10228000BDE8F0870B41DB0744BF0132D2B20FE556
:1022900040F63635D7E69DF80D30002B3FF4DDAE25
:1022A0000A9B03F525731D44D7E600BF1B280D01CB
:1022B0001C0C0100F8B53B4F97F8E6300446002BA4
:1022C00037D0394D95F8A86C012E33D0022E4FD05F
:1022D0007EBB006801228021FEF7DAFD2068012222
:1022E000FF21FEF7D5FD206832463146FEF7D0FDCE
:1022F00095F8A02C20689121FEF7CAFD20680122E4
:102300003146FEF7C5FD20683246FF21FEF7C0FDCD
:10231000206832468021FEF7BBFD2068012231464D
:10232000FEF7B6FD214B1B68C5F8983C012385F8E4
:10233000A83CF8BD00680021FFF7EEFAC20711D5EE
:10234000D5F89C2C002AF4D0184BD5F8981C1B68A3
:102350009BB25B1A9A42ECD2154B4FF0FF325A6097
:102360000023E4E7114B1B68C5F8983C0223DEE725
:1023700000681321FFF7D0FA4307E1D01E2120683F
:10238000FEF7D8FF012206460B212068FEF780FDEC
:10239000074B0A20B6FBF0F6B6B25E60012387F861
:1023A000E730DDE7385D0020306E00202426002075
:1023B0005C090020F0B513238DB0054600222921C9
:1023C0000220FDF719FB524CC4F85001002800F020
:1023D00091800221FCF79AFB02220021D4F85001DF
:1023E000FEF728FC002384F8583184F8545104F592
:1023F000AE7304F21C524FF0202143F8041B9342A9
:10240000FBD1444E444F35683235D4F8500103793E
:10241000012B71D0022B0FD183683F4ADB074FF0AD
:1024200080015CBF3C4A8021FFF770F910B133682E
:102430009D42EAD8D4F850011024112213214FF004
:10244000120E4FF0140C1527162617258DF80C4088
:102450008DF80E20182419228DF812101B2101234B
:102460008DF810E08DF814C08DF816708DF8186096
:102470008DF81A508DF81C408DF81E208DF8221012
:102480004FF01A0E4FF01C0C1D271E261F254C2442
:10249000222203A98DF80D308DF80F308DF8113000
:1024A0008DF813308DF815308DF817308DF8193000
:1024B0008DF81B308DF81D308DF81F308DF820E021
:1024C0008DF821308DF823308DF824C08DF825301B
:1024D0008DF826708DF827308DF828608DF829301A
:1024E0008DF82A508DF82B308DF82C308DF82D403A
:1024F00048F0EFF90DB0F0BD8268417C90F9100012
:1025000002F00102CDE900728022F8F789FA8DE726
:10251000385D0020242600208F5E0020F0B5514C4D
:10252000D4F8505185B015B194F856310BB105B0BF
:10253000F0BD012384F856312B79012B7CD0022B7E
:1025400037D128460DF10E028421FFF7DFF8D4F8C9
:10255000505194F858212B79012B42F0040279D183
:102560008DF80F20AA6895F91000697C02F001022D
:1025700001920DF10F0200920422F8F72BFA15E0F8
:10258000022B0ED1AB6813F0010F0DF10E024FF0CC
:102590008401284602BF0DF10E0284212846FFF770
:1025A000B5F89DF80E3013F0040616D0D4F850514B
:1025B0002B79012BE4D1AA68697C95F9100002F00F
:1025C000010201920DF10E0200928422F8F728FA1E
:1025D0009DF80E3013F00406E8D1234D234884F80B
:1025E000583131463C224EF0B6FE01273146A5F166
:1025F000460E05F5707635F8023F1A0A4FEA511C6F
:1026000003F0040322F02002134318BF5EF82C30BD
:1026100001F01F0007FA00F01CBF18434EF82C0011
:10262000B54201F10101E6D1FBF740FE0028FBD1E4
:1026300084F8560105B0F0BDAA68697C95F91000D0
:1026400002F0010201920DF10E0200928422F8F7CD
:10265000E7F97CE7022BACD128460421FEF7C5FA46
:10266000A4E700BF385D0020925E00204C5E002091
:1026700010B52D4CD4F8500184B0E8B194F8543121
:10268000012B32D0022B19D10823002104228DF80E
:102690000C1003A984F857318DF80D308DF80E20F9
:1026A0008DF80F2048F015F920483C22FF214EF00C
:1026B00052FE94F85531D3B104B010BD0379012B0B
:1026C00022D0022B1AD09DF80B3003F00503012B0A
:1026D00009D013B9D4F85001D6E7154A126840F270
:1026E000DC539A42E8D9D4F850014823CDE7FFF7EC
:1026F00015FF012384F8553104B010BD0DF10B0214
:10270000A021FFF703F8DEE7826890F910C0417C52
:1027100002F0010201920DF10B0200926046A0222C
:10272000F8F77EF9CFE700BF385D00204C5E00204F
:1027300024260020F0B53E4CD4F8505185B095B118
:1027400094F85731180702D594F856316BB194F8C4
:10275000553143B9FFF78CFF94F85531002B3BD12D
:10276000002384F8563105B0F0BD94F855310122AC
:1027700084F85621002BEDD02B79012B2FD0022B82
:10278000E8D10DF10E0280212846FEF7BFFF002898
:10279000E0D094F857219DF80E309A42DAD194F89F
:1027A0005451002DD8D1234B234E1F68D6F8AC3C92
:1027B000FB1AB3F57A7FCFD9A021D4F850010DF1DF
:1027C0000F02FEF7C9FF9DF80F30590715D5C6F85F
:1027D000B05CC6F8AC7CBFE7FBF768FDC0E7AA6851
:1027E000697C95F9100002F0010201920DF10E02D0
:1027F00000928022F8F714F9C9E703F00503012BD2
:102800000ED0002BE5D194F857315B06E1D5D6F810
:10281000B03C53B1FB1A642BDBD9FFF729FFD8E793
:1028200094F857315A06F2D5D3E7C6F8B07CD0E712
:10283000385D002024260020306E00202DE9F04372
:102840008E4ED6F8504185B0002C6ED096F8569139
:10285000B9F1000F00D0FEE796F857C101230CF044
:10286000F70C86F857C186F856312379012B0546B7
:102870000F4600F0DF80022B00F097800DF10F086B
:10288000B5F5807F00F0B4802379012B00F0BB8088
:10289000022B07D1204650220821FEF7A6F9D6F8D0
:1028A00050412379764D012B1AD0022B0AD1424692
:1028B0002046A021FEF72AFF20B19DF80F4014F01A
:1028C000200451D0D5F8A830B5F8AC205969D6F815
:1028D00050410A4214BF5A831A832379012BE4D151
:1028E000A268617C94F9100002F00102CDE9008237
:1028F000A022F8F795F8DFE7B9F1000F12D196F8AA
:102900005741D6F8505104F0F70486F857412B7917
:10291000012B00F0A580022B04D12246494628460F
:10292000FEF763F9002386F8563105B0BDE8F08361
:10293000022B16D162460A212846FEF756F9D6F830
:1029400050010379012B07EB040228D18568417CF3
:1029500090F9100005F00105CDE90025C022F8F737
:102960005FF80134362CC7D0D6F850512B79012BA3
:102970005FFA84FCDCD1AA6895F91000697C8DF8B7
:102980000FC002F00102CDE900820A22F8F722F816
:10299000D6F850010379012B07EB0402D6D0022BA5
:1029A000DFD1C021FEF7B2FEDBE749462046624692
:1029B000FEF71BF9D6F85041237981460DF10F0837
:1029C000012BEAB22ED1A16894F9100001F0010C9C
:1029D000617C8DF80F20CDF804C0CDF8008009226D
:1029E000F7F7F8FFB5F5807FD6F850417FF44CAF8C
:1029F000204640220A21FEF71DF9D6F850412379DE
:102A0000012B7FF445AFA26894F91000617C02F0BD
:102A10000102CDE9008250228DF80F200822F7F73D
:102A2000D9FF3CE7022B7FF42BAF20460921FEF7AC
:102A3000DCF8D7E7A16894F9100001F0010E0DF160
:102A40000F08617CCDF804E04A46CDF800808DF88F
:102A50000FC0F7F7BFFFD6F8504181462379AFE7A3
:102A6000A96895F9100001F001074A46697C8DF8C4
:102A70000F40CDE90087F7F7ADFF53E7385D002041
:102A8000783900202DE9F04F5E4B93F85651C7B0CE
:102A900005B1FEE75B4A92F85771012382F856317F
:102AA00007F0F707D2F8503182F8577103931B797A
:102AB000012B04460E4600F09580022B40F09080DA
:102AC0000398836813F0010118BF29463A46FEF7C0
:102AD0008CF805AD4B4BD3F850310393FF2C6C7041
:102AE0004FF0090388BFA4082B708CBF04F0C00806
:102AF0004FF00008022200204FF00A090DF1150ADC
:102B00004FF00B0B10E0BEF5827F05F80290375CAA
:102B10000AF8023013D80130362805F804B002F163
:102B2000060C6F54724612D0941C48EA0003B4F5A8
:102B3000827F02F1040EDBB202F10301E3D901301E
:102B40006FF0004E3628DFF8C4C07246ECD1BCF5F9
:102B5000827F9FBF08210DF1150305F80E10A021FB
:102B600098BF03F80E10039894BF02326FF0004232
:102B7000294647F0AEFE234B234DD3F8500103798D
:102B8000012B0DF1130419D0022B08D12246A021EC
:102B9000FEF7BCFD18B1237813F020031AD0D5F846
:102BA000A830B5F8AC2059690A4214BF5A831A8379
:102BB000144BD3F850010379012BE5D18268417C95
:102BC00090F9100002F00102CDE90042A022F7F7CF
:102BD00027FFDFE70B4A82F8563147B0BDE8F08F98
:102BE00005AD7BE7039881682A4601F0010501469F
:102BF00090F91000497C019505AD2F700095F7F70D
:102C0000E9FE67E7385D0020783900200100008088
:102C1000024BD3F8503103B134E77047385D0020E0
:102C200010B5EFF31182102383F312884FF0E023E5
:102C3000D2B29C69196911F4803F0D491EBF012071
:102C4000C1F8840B9C690B4B1868D1F8843B82F364
:102C50001188094A11684FF47A72034402FB01F0AB
:102C6000001BB0FBF1F00021E3FB020110BD00BF2F
:102C7000306E0020242600201C2E0020124B5B68A2
:102C8000C3F3080330B4EBB9EFF31183D3B90F4B9F
:102C90000F484FF0E0251968AC691A688A42FAD1EA
:102CA000D0F8801BA142F6D30A4B19684FF47A730F
:102CB00003FB01F0001BB0FBF1F00021E2FB03017C
:102CC00030BC704730BCABE700ED00E024260020AC
:102CD000306E00201C2E0020F8B506460D46FFF78A
:102CE000CDFF04460F46FFF7C9FF031B61EB070248
:102CF000B34272EB0503F6D3F8BD10B50446013CB0
:102D000000D210BD4FF47A700021FFF7E5FFF6E71F
:102D100010B504464069FCF799FB0120FFF7EDFF71
:102D20006069FCF78EFBBDE810400A20E5E72DE95D
:102D3000F04304680646A0698BB0A8B140F61503BD
:102D40000021C3800172FCF78FFBAF4BB361336886
:102D50009B691846FCF786F8002880F2EB80336800
:102D60009869002840F04481B6227E212046FDF774
:102D700061FF6420FFF7C1FF02212046FBF7C6FE7A
:102D80002046FFF7C5FF00227C212046FDF752FFB9
:102D90000120FFF7B2FF002259212046FDF74AFF2C
:102DA0000120FFF7AAFF5E2394F910208DF8273049
:102DB000964B142101FB02335D69A3689A0702D484
:102DC000606947F0E5F901230DF12702002128464B
:102DD00047F054FD4FF4A4738D4A0021284647F074
:102DE0004DFDA3689B0702D42046FDF7F3FE0A20A1
:102DF000FFF783FF012259212046FDF71BFF012029
:102E0000FFF77BFF8C2240212046FDF713FF0120B6
:102E1000FFF773FF022241212046FDF70BFF7D4F94
:102E20000120FFF76AFF96F82D30326B7A48B0FB2D
:102E3000F2F03D463A464FF0000C012192F8069020
:102E4000A3EB0908A3EB0C0EB8F1000FB8BFC8F153
:102E50000008BEF1000FB8BFCEF1000EF04502F140
:102E6000060201F10101BCBF4FFA89FC1546092990
:102E7000E4D14FF0000E80B23A7862450CD16988F7
:102E80007A88411A821A0029B8BF4942002AB8BF7D
:102E900052429142C8BF3D460EF1010EBEF1090FEC
:102EA00007F10607E8D16A7904922A7903926A88C1
:102EB00002922A780321CDE90002584A0120F9F74D
:102EC00057FE6A88544BB3FBF2F3B3632A7942216D
:102ED00042F0C0022046FDF7ADFE0120FFF70DFFD6
:102EE000082243212046FDF7A5FE0120FFF705FF3C
:102EF000042258212046FDF79DFE0120FFF7FDFE2C
:102F00000A2253212046FDF795FE0120FFF7F5FE2A
:102F100000227C212046FDF78DFE0120FFF7EDFE0B
:102F200006227D212046FDF785FE01200BB0BDE87D
:102F3000F043E2E63A4D3B492A1892F8007406F154
:102F4000180241F820201846FBF781FF0146184679
:102F5000FBF788FF00F0FC0202F1804202F59C3290
:102F600000F0030C4FEA8C0C90684FF00F0E0EFA35
:102F70000CFE20EA0E009060D2F808E0C8B200FA19
:102F80000CF141EA0E01916023B11846FBF76AFF8C
:102F90000123834024494B610A6822EA03020A6044
:102FA0004A6822EA03024A60204AD2F8000C184319
:102FB000C2F8000C886820EA03008860C86820EA2C
:102FC0000300C860D2F8080C0343C2F8083C184B51
:102FD000DA5D042A7FF6C3AE3D44042195F910045E
:102FE000D9550790F6F794F90798F6F783F9B6E6FE
:102FF000FBF738FF012313FA00F01FBF0A4A1368DA
:1030000018431060B0E600BF51D900085C090020E9
:10301000A71C06085A1C060840420F00E8A506082F
:1030200090180608043C0020003C0140003001409C
:10303000443C002037B5054605249620FFF75DFE89
:103040000DF1070200212846FEF786FB08B9013C76
:10305000F3D103B030BD38B500231A463521012025
:10306000FCF7CAFC164D0446C5F8B40C48B9154B1C
:1030700085F8B80C1B781A2B04BF0123C5F8BC3C9B
:1030800038BDFFF7D7FF70B90E4B1B781A2B08BF5E
:103090000223204608BFC5F8BC3CFBF72AFD0023ED
:1030A00085F8B83CECE70123002285F8B83C85F8A8
:1030B000B92C20464021BDE83840FDF7BBBD00BF1C
:1030C000306E0020033C002008B5054B02463D2130
:1030D0001868FDF7AFFDBDE8084019200DE600BFF8
:1030E000B848002084B070B590B014AC504E9DF834
:1030F000685084E80F0000244FF08070C6F87C4BC5
:103100001CF0C8F828B9002010B0BDE8704004B029
:1031100070474FF4E133032290F904000294CDE9A3
:1031200000324FF08071434A23461CF06FFAC6F814
:103130007C0B0028E7D001212046FDF761FC05202B
:10314000FFF7DBFD3C4B93F8F020012ADBD193F82D
:10315000F120A02AD7D193F8EB100029D3D13E203B
:103160000591FDF743FC1920FFF7C7FD0599002DD8
:1031700054D03D20FDF73AFC14AC1920FFF7BDFDFB
:103180000FCC0AAD0FC5BDF95830BDF9562094E8F3
:1031900003008DF820301B128DF82130BDF932303C
:1031A0008DF822301B128DF82330BDF93430A98000
:1031B0008DF82430BDF954108DF81C101B128DF8B9
:1031C0002530BDF936308DF81E2009121212BDF9D6
:1031D0005050BDF952408DF81D108DF81F2007A9E1
:1031E0000C228DF8263055201B128DF82730FDF764
:1031F000CFFB1920FFF781FD8DF81C508DF81E4084
:1032000067202D122412042207A98DF81D508DF875
:103210001F40FDF7BDFB1920FFF76FFD0C213D207E
:10322000FDF7E4FB1920FFF768FD01206CE700BF04
:10323000306E0020E5DF0008385D002013B5002265
:1032400004460A210068FDF7F5FC1420FFF755FD40
:103250000F220A212068FDF7EDFC0A20FFF74DFD43
:10326000032301AA10212068FDF7D4FE0A20FFF7EE
:1032700044FD00220A212068FDF7DCFC0A20FFF74C
:103280003CFD0DF1030220680221FEF765FA0DF105
:10329000030220680921FEF75FFA206801220A2153
:1032A000FDF7C8FC012002B010BD10B5782204461D
:1032B00000210068FDF7BEFC0520FFF71EFD20225F
:1032C00001212068FDF7B6FC0520FFF716FD00225E
:1032D00002212068FDF7AEFC6420FFF70EFD0120FF
:1032E00010BD10B52422044641210068FDF7A2FC60
:1032F00080B1206820223021FDF79CFC50B120686D
:1033000006223121FDF796FC20B1206800223421ED
:10331000FDF790FC0520FFF7F0FC012010BD10B573
:10332000072204460A210068FDF784FC0520FFF708
:10333000E4FC242241212068FDF77CFC0520FFF7F6
:10334000DCFCC02242212068FDF774FC0520FFF759
:10335000D4FC012010BD10B50122044610210068E4
:10336000FDF768FC48B11420FFF7C7FC2068A022D5
:10337000BDE810401121FDF75DBC10BD08B5006827
:1033800001220921FDF756FCBDE808406420B4E4A1
:1033900080B506460B25013D01D1FDF7C9FB012192
:1033A0000846FCF7B3FC00210846FCF7AFFC771C8D
:1033B0004FF0320805240120FCF798FC0020FCF7B0
:1033C00095FC0120FDF77DFB4046FFF796FC0120B0
:1033D000FCF78CFC0020FCF789FCFDF772FB4046F3
:1033E000FFF78BFC7CB1013C05D14FF4FA70FFF77D
:1033F00084FC4FF0FA0854EA0703DCD14FF47A70EA
:10340000FFF77BFCC7E7013FF5E718B103685B688E
:1034100003B11847FF20704718B103689B6803B1D8
:1034200018470020704770B450B106798E4207D318
:103430004579954204D30368DB680BB170BC18472B
:1034400070BC704710B440B184798C4205D30368D6
:103450001B6913B15DF8044B18475DF8044B7047C6
:1034600018B103685B6903B11847704718B1036866
:103470001B6A03B118470020704730B560B1041DC6
:103480000A4600F1140320686168154603C5083434
:103490009C422A46F7D1012030BD10B50C4670B9C8
:1034A0002D23002023750A4B2061C4E90000C4E9E4
:1034B0000200C4E90633302384F8203010BD0368CD
:1034C000DB6A002BECD098470028E9D0F6E700BF74
:1034D000DCAB060838B5054D441E14F8011F01B9D0
:1034E00038BDD5F8DC0CFBF7F3FAF6E7306E0020B8
:1034F00013B50C4C01900C480091FFF7EBFFDDE990
:1035000000320A49D4F8DC0C45F032FAD4F8DC0C6D
:10351000FBF7D2FA94F8E03C13B1012384F8E13CC4
:1035200002B010BD306E002021A60608F1EA0008A6
:1035300008B50648FFF7CEFF054BB3F8E20C18B10B
:10354000BDE80840FFF7D9BB08BD00BFAEF70608CD
:10355000306E002010B5074C02460B46D4F8DC0C48
:10356000054945F005FAD4F8DC0CFBF7A5FABDE8EF
:103570001040DDE7306E0020F1EA000808B5FFF7E3
:10358000A9FFBDE80840D3E710B504460648FFF799
:10359000A1FF2046FFF79EFF044B93F8E02C12B1E9
:1035A000012283F8E12C10BD21A60608306E002010
:1035B00010B504460348FFF78DFF2046BDE81040D4
:1035C000DCE700BF2DA606080CB4830607B500D5BE
:1035D00051B9049805A90191FFF7BCFF012003B080
:1035E0005DF804EB02B070470020F8E7024B01469B
:1035F000D3F8DC0CFBF76CBA306E00200CB407B5C6
:1036000010F0400009D069B92320FFF7EFFF0498BC
:1036100005A90191FFF79EFF012003B05DF804EBBF
:1036200002B070470020F8E70FB413B5094C0A49FF
:10363000D4F8DC0C04AB53F8042B019345F098F953
:10364000D4F8DC0CFBF738FA02B0BDE8104004B047
:10365000704700BF306E0020F1EA00080FB407B5D4
:1036600004A951F8040B0191FFF774FF03B05DF852
:1036700004EB04B070470FB407B504A951F8040B6C
:103680000191FFF735FFFFF753FF03B05DF804EB3F
:1036900004B0704770B58379164603F00F028EB000
:1036A0000446062A50D8DFE802F0041417191C1E3D
:1036B0004A000D7813F0C00348D0402B3DD1294675
:1036C000204611F0D3FF00285BD00EB0BDE870405B
:1036D000AAE791F90050EDE70D88EBE7B1F900504A
:1036E000E8E70D68E6E791ED000A03A8F9F71AFE8E
:1036F00001462948FFF798FFFEB1A37913F0C00FE8
:103700001BD1204611F0FFFE00EE100A03A8B8EE10
:10371000C00AF9F707FE01462048FFF785FF20465B
:1037200011F002FF00EE100A03A8B8EE400AF9F704
:10373000F9FD01461948FFF777FF0EB070BD164836
:103740000EB0BDE870406FE70025B3E7042A0CBF58
:10375000134814482946FFF767FF002EEDD0A379E0
:1037600013F0C00FE9D1204611F0CDFE01902046A4
:1037700011F0DAFE019902460B480EB0BDE8704028
:1037800052E703A9204611F0E3FD084803AA2946A1
:10379000FFF771FFD1E700BF0FAA060824AA0608A9
:1037A00083A60608EAE6060879F9060832A606089E
:1037B0002DE9F04F8FB001F020034D4C009381466E
:1037C0000F464FF000084B4BD3F8DC0CFBF774F9B5
:1037D00094F806B00BF030034B454BD1204611F066
:1037E00031FEF9F791FF0646204611F04DFED6F85E
:1037F00008A005460AEB0006204611F077FE0BF004
:103800000F02062A6CD8DFE802F0044045494E5208
:103810005E001AF805200078111A4A424A41009BBE
:1038200003B13ABB03A92046019211F091FD7B063A
:1038300015D5019A9AB9304803A9FFF7F5FE2F492B
:1038400003A847F035F900284CD11AF80530202B91
:1038500048D12B483146FFF7E7FEFFF769FE2948BC
:1038600003A9FFF7E1FE002231462046FFF712FFD1
:10387000FFF75EFE08F1010840F24523984504F188
:103880000B04A0D10FB0BDE8F08F1AF9052090F914
:103890000000C1E73AF805200088BDE73AF90520A5
:1038A000B0F90000B8E75AF805200068B4E796EDD3
:1038B000007AD0ED007AB4EE677AF1EE10FA0CBF20
:1038C00001220022ABE70190204611F02DFE019964
:1038D000421C30464DF08EFDB0FA80F252099EE750
:1038E00000229CE7002231462046FFF7D3FEB4E7D2
:1038F000241E0608306E00204FA606084BF9060865
:103900005AA6060850A6060813B50446019111F000
:10391000EDFD019A0146204602B0BDE81040B9E62F
:10392000F7B5847914F0C003054603D0402B18D0B6
:1039300003B0F0BD04F00F0411F0F6FD062C05D124
:103940000146164803B0BDE8F04087E601902846DE
:1039500011F0D9FD019A0146114803B0BDE8F040CD
:103960007CE611F073FE05460E480F4E0F4FFFF731
:10397000B1FD00242B79A34203D803B0BDE8F04089
:10398000D6E514B13046FFF7A5FD2B68384653F84D
:103990002410FFF749FE0134ECE700BF5FA60608DC
:1039A0006FA6060886A6060896A6060824AA060894
:1039B00008B50548FFF78EFD044BD3F8DC0CBDE8D5
:1039C0000840FBF779B800BF2DA60608306E00202E
:1039D000004850E698A6060813460A4601460148E4
:1039E00049E600BFA4A6060820B10078B0FA80F02E
:1039F00040097047012070472DE9F04F87B003461A
:103A0000FFF7F2FF064618B107B0BDE8F04FDFE759
:103A10004649DFF84091DFF840A1DFF840B105AA40
:103A200018464DF03EFC34460546B0464FF0FF3791
:103A30008DB97EB230461BF019FC10B14568002DDF
:103A40005AD1B8F1000F36D139483946F9F75EF846
:103A500007B0BDE8F08F012E0ED0022E11D01EB996
:103A60002846F9F7A9FD0746304905AA00204DF080
:103A700018FC01360546DBE72846F9F79DFD804630
:103A8000F2E7494628464DF0ECFC20B92949284682
:103A90004DF0E7FC08B144F00104514628464DF0D2
:103AA000E0FC28B9594628464DF0DBFC0028DBD065
:103AB00044F00204D8E7002C08BF03240023E4B23A
:103AC000CDE9008402931A46194630461BF09EFD4C
:103AD000054610B918483946B8E7184842463946ED
:103AE000F9F714F839461648F9F710F8154B294636
:103AF000D3F8E40C42F038FD13483946F9F706F8DC
:103B00005CB16979A14208D010482246F8F7FEFF5F
:103B10002B68E1B29B6928469847EB6A002BE1D0FD
:103B20000B48F8F7F3FF0023EB62DBE7E4A306089A
:103B3000C4A60608CED50608ECA606080BA70608FC
:103B400076A70608306E002028A7060840A70608BA
:103B500060A70608C7B40608C1A60608D6BA0608B4
:103B60002DE9F04F85B00546FFF73EFF044630B122
:103B70000021012005B0BDE8F04F42F04FBD85495E
:103B80002846F9F7D5F920B905B0BDE8F04F39F06E
:103B9000E9BC81492846F9F7CBF928B9012005B0DD
:103BA000BDE8F04F39F0D6BD7C492846F9F7C0F999
:103BB000034688BB7A4A92F9D61F82F8D00F104686
:103BC00092F89054012D08D0033D052D05D9002C05
:103BD00000F0D28080F8D61FCEE092F8A654A52D32
:103BE00003F1010313D101290ED16E4A80F8D13FB0
:103BF000002380F8D01F82F8E83C80F8D63F05B05B
:103C0000BDE8F04F39F02CBE013949B20124782BC0
:103C100002F11802D4D1DAE72846F9F7CDFC614B5E
:103C200093F9E83C009303FA80F6772E834600F27E
:103C3000A7802846FAF766FE0746002800F089802C
:103C4000F9F7BAFC0124C5B23846FAF75BFE07461D
:103C5000002800F08180F9F7AFFC01340190E4B254
:103C60003846FAF74FFE8046002877D0F9F7A4FCD3
:103C700001340746E4B24046FAF744FE8146002884
:103C80006ED0F9F799FC01340290E4B24846FAF795
:103C900039FE8246002865D0F9F78EFC01340FFA10
:103CA00080F9E4B25046FAF72DFE824600285BD038
:103CB000F9F782FC01340FFA80F8E4B25046FAF7C3
:103CC00021FE002852D00390F9F776FC03990FFAF1
:103CD00080FA0846FAF716FE0346002857D004F08B
:103CE000FD04F9F769FC042C46D1C3B2012D02D9B9
:103CF000E91E052940D81BB1A52B01D0482B3BD18B
:103D0000274C0EB984F8D66F182101FB0646019A9C
:103D1000C6F89424A52B029A86F89054C6F8987495
:103D2000C6F89C24A6F8A094A6F8A284A6F8A4A499
:103D300086F8A6340AD100981A4B0130584483F80B
:103D4000E80C94F8D63F013384F8D63F05B0BDE8BF
:103D5000F08F0446054677E7019081E707468AE73A
:103D6000029093E781469DE78046A7E75FFA88F3D4
:103D700082468046062CB9D005B0BDE8F04F27E654
:103D800009487722214605B0BDE8F04F24E601340A
:103D9000E4B2EFE7A4A70608AAA70608CCB1060874
:103DA000284D0020306E0020AFA7060808B5034656
:103DB000FFF71AFE40B10C4B0C480022A3F8E22C8E
:103DC000BDE80840FFF7DABB1846F9F7F5FB0146F6
:103DD00030B1054BA3F8E20CBDE8084004483DE4CF
:103DE000BDE80840F4E500BF306E0020B8A7060823
:103DF000CEA706082DE9F04FDFF8B8A087B0074638
:103E000016460C4615464FF0000B4FF019094FF4BB
:103E10006178002E4BD0237828788342EB7844D108
:103E200061786A78914240D1A178AA7891423CD1D8
:103E3000E178CA1A51425141CDE9041310F04EFE07
:103E4000059B049919FB03830393AB7819FB038348
:103E500002936B780193037A009352465B4638468F
:103E6000FFF7CCFB04992078049110F037FEE3783B
:103E7000049919FB03830393A37819FB038302932B
:103E800063780193037A009352465B4638460BF100
:103E9000010BFFF799FBBBF1280F04F1040405F1B6
:103EA0000405B6D107B0BDE8F08F0021C4E7314664
:103EB000D9E700BFE5A70608F7B50746FFF794FD69
:103EC000044630B127490022012003B0BDE8F0408C
:103ED00090E73846F9F770FB272805463ADC86005C
:103EE000781C8DF80740FAF70DFD044678B1F9F714
:103EF00063FB00280BDBC0B210F002FE38B11A4B96
:103F00000278334483F8E92C01238DF807302046EA
:103F1000FAF7F8FC044660B1F9F74EFB0D2808D813
:103F2000114B334483F8EA0C9DF8073001338DF8C8
:103F300007300C4FB11C0DF1070239442046FAF747
:103F4000EEFC9DF80730042B02D0002347F8253003
:103F500003B0F0BD05482722214603B0BDE8F0407C
:103F60003AE500BF197B0020306E0020CAA8060881
:103F70002DE9F04F89B0374EDFF8E0900692804689
:103F80000C46154602F13C0B94F9041000230C2258
:103F9000314F02FB03F0C057884255D00133052B47
:103FA000F6D10C355D4504F10C04EDD109B0BDE846
:103FB000F08F95F904302A68687995F806C095F86D
:103FC00008E095F807A099423CD12168914239D187
:103FD0006179814236D1A179614533D1217A714528
:103FE00030D1E179A1EB0A077942794156F82A707C
:103FF00056F82000049756F82E70039756F82C7048
:104000000297CDE900204A4640460791FFF7F6FAAD
:104010000799E27994F9043056F822200492227A22
:1040200056F822200392A27956F822200292627951
:1040300056F8222001922268009240464A46FFF735
:10404000C3FAAEE70021D1E7069B002BB1D1194698
:10405000DFE700BF901706084C3C0020F8A70608D1
:10406000F0B585B00346FFF7BFFC30B143490022ED
:10407000012005B0BDE8F0407AE718465E1CF9F76C
:104080009BFA044640B21BF07BFA054630B93C4827
:10409000214605B0BDE8F040FFF7EDBA0068696859
:1040A00001AB03C3A86818603046FAF72BFC04463E
:1040B000002852D003782B2B05D02D2B42D0F9F7B6
:1040C0007BFA019009E001342046F9F775FA019B6B
:1040D000012202FA00F00343019302260027204642
:1040E000FAF710FC044638B3F9F766FA254A0023BC
:1040F000114652F804EB70455FFA83FC04D001339B
:10410000112BF6D14FF0000C51F82C30984213D1FE
:10411000102200216046F7F7C9FE022F1FD0032F9F
:1041200020D0012F14BF8DF809008DF80A00013747
:104130000136042FF6B2D2D1012E16D805B0BDE853
:10414000F04045E401342046F9F736FA019B01229C
:1041500002FA00F023EA0003BEE70126BEE78DF86D
:104160000C00E4E78DF80B00E1E701AB03CB28601E
:1041700018686960A86005B0F0BD00BFBC450020AC
:1041800015A80608901706082DE9F04FDFF8C0B013
:1041900089B0804617460C46154600264FF0190A8E
:1041A0004FF46179002F51D06979A8780791A178EF
:1041B0002B786A7895F803C095F804E0069381425D
:1041C00042D1217899423FD1617891423CD1E17846
:1041D000614539D12179714536D1079963795B1AE7
:1041E00059425941069B06911AFB0393CDE90103FD
:1041F0001AFB0292079B03920093CDE904CE33464B
:104200005A464046FFF7FAF9069923790593E37871
:10421000049363781AFB0393039323781AFB0393A5
:104220000293A3780193637900935A46334640463C
:104230000136FFF7C9F9142E04F1060405F106054D
:10424000B0D109B0BDE8F08F0021CBE73946DCE7FB
:1042500028A806082DE9F3478246FFF7C5FB064666
:1042600030B13C490022012002B0BDE8F0478BE7A5
:104270005046F9F7A1F91328054663DC06274743A2
:104280000AF101008DF80760334CFAF73BFB04F6A6
:10429000895909EB0708064648B1F9F78DF9032853
:1042A0009FBFE31983F88E0D01238DF80730304648
:1042B000FAF728FB064668B1F9F77EF90D2809D808
:1042C000062303FB054383F88B0D9DF8073001336C
:1042D0008DF807300DF1070241463046FAF71FFB13
:1042E000FAF710FB064668B1F9F766F93A2809D8DB
:1042F0009DF80730062202FB0542013382F88C0D3F
:104300008DF807303046FAF7FDFA68B1F9F754F93D
:104310000D2809D89DF80730062202FB0544013319
:1043200084F88D0D8DF807309DF80730062B06D0E8
:10433000002349F80730A8F80430FFF749FB02B022
:10434000BDE8F08705481322314602B0BDE8F047CA
:10435000FFF742BBB97B0020306E0020CAA80608D8
:104360002DE9F04F2DED088BDFF814A197B007462B
:1043700090460C461546002694ED008AB5EE408A1C
:10438000F1EE10FA73D0D4ED019A94ED029AD4EDC7
:10439000038AB8F1000F40D095ED000A95ED01BAFF
:1043A000D5ED02AA95ED03AAB4EE408AF1EE10FA1B
:1043B00062D1F4EE4B9AF1EE10FA5DD1B4EE6A9A46
:1043C000F1EE10FA58D1F4EE4A8AF1EE10FA0CBF71
:1043D0004FF001094FF0000912A8F8F7A3FFB0EE63
:1043E0004B0A83460EA8F8F79DFFB0EE6A0A0590C7
:1043F0000AA8F8F797FFB0EE4A0A049006A8F8F763
:1044000091FF059B049A0390CDE900B302923346D5
:10441000524649463846FFF7F1F8B0EE480A12A86E
:10442000F8F780FFB0EE690A81460EA8F8F77AFF28
:10443000B0EE490A83460AA8F8F774FFB0EE680A9E
:10444000049006A8F8F76EFF049B0390CDE901B332
:10445000CDF8009033465246002138460136FFF72A
:10446000B3F80C2E04F1100405F1100584D117B037
:10447000BDEC088BBDE8F08F4FF00009ACE700BF42
:1044800046A8060870B50546FFF7AEFA064628B1FD
:10449000BDE870402C490022012061E72B4905222C
:1044A0002846F8F729FD38B9274B002201300C289F
:1044B00043F8102BFAD170BD2846F9F77DF80B2888
:1044C00004463AD82846FAF71DFA064648B3F8F7E4
:1044D00091FF1D4B03EB041383ED000A01253046C9
:1044E000FAF710FA064638B1F8F784FF164B03EBDB
:1044F000041383ED010A01353046FAF703FA064644
:1045000038B1F8F777FF104B03EB041383ED020A81
:1045100001353046FAF7F6F928B9BDE87040FFF7E3
:1045200057BA0546DBE7F8F765FF0748032D00EBB0
:10453000041484ED030AABD0EFE731460448BDE82C
:1045400070400B22FFF748BA347C0020A4A706086D
:10455000CAA806082DE9F043DFF8649085B08046CC
:104560000D4616460227002446B336F8242035F8B7
:104570002430F05B93421FD1EB5B191A4B424B4145
:104580001946CDE9002023464A4640460391FFF7ED
:1045900035F80399EB5B019335F8243000934A46D4
:1045A000234640460134FFF70FF8042C07F10407B7
:1045B000DAD105B0BDE8F0830023E1E73146E9E751
:1045C0005AA80608F8B50446FFF70EFA054628B1C2
:1045D000BDE8F840294900220120BBE728492046D0
:1045E000F8F7A6FCA8B9274B4FF47A714FF4FA629A
:1045F000A3F8C41EA3F8C62EA3F8C81EA3F8CA2E9B
:10460000A3F8CC1EA3F8CE2EA3F8D01EA3F8D22E6A
:10461000F8BD2046F8F7D0FF0328074627D82046E4
:10462000FAF770F9044670B1F8F7C6FF012506469F
:104630002046FAF767F910B1F8F7BEFF2DB9BDE8CB
:10464000F840FFF7C5B90546F2E7A6F2EE2240F2C0
:10465000DC539A42F3D8A0F2EE229A42EFD8094BEB
:1046600003EB8703A3F8C46EA3F8C60ED0E7294670
:104670000548BDE8F8400322FFF7AEB9F47C0020FE
:10468000A4A70608306E00206BA806082DE9F04F9D
:10469000DFF800A191B0834691460C4615460026EE
:1046A00004F115080422414609A84CF0B7FE002386
:1046B0008DF82830D4E90232082B72F100010BAFDB
:1046C00056D230491A463846F8F73CFAB9F1000F8D
:1046D00055D02B780793079A237893424DD1D4E98C
:1046E0000202D5E902139A4208BF884245D1227DD1
:1046F0002B7D9A4241D1042205F1150140464CF030
:1047000000FE002839D121692B69CB1A5942594141
:104710001D4B059300230493B5F912300393B5F9AB
:1047200010300293194B0193079B00935246334676
:1047300058460791FEF762FF079909AB0593237D61
:104740000493B4F912300393B4F91030CDE9017336
:1047500014F8203B00935246334658460136FEF784
:1047600033FF082E05F120059AD111B0BDE8F08F76
:1047700007493846F8F7E6F9A8E70021C8E74946AF
:10478000DBE700BFEAE606088EBF0608EFD9060899
:1047900073A806087EA806082DE9F74F0446FFF720
:1047A00023F9074630B16E490022012003B0BDE86D
:1047B000F04F6BE76B492046F8F7BAFB014638B972
:1047C00067484FF4807203B0BDE8F04F4CF0C3BDB2
:1047D0002046F8F7F1FE83B2072B054600F2B880B9
:1047E0002046FAF78FF8824600284CD0F8F7E4FE0E
:1047F00001240FFA80F95046FAF784F868B14FF0B7
:104800000008411E00F1100C464611F8013F13F05C
:10481000DF0F3BD101270134E4B2FAF773F8824687
:1048200000284CD0F8F7C8FE01340FFA80FBE4B240
:104830005046FAF767F80346002842D00190F8F78F
:10484000BBFE0134019B0FFA80FAE4B21846FAF776
:1048500059F80346002836D00190F8F7ADFE013430
:10486000019B42B2E4B218460192FAF74BF8019A62
:10487000034650B30134E4B2032C28D803B0BDE89A
:10488000F04FFFF7A5B804468146B4E76145C2D0B2
:10489000A3F13002D2B2092A05D9A3F16102052A97
:1048A00007D8573BDAB2360146EA187642EA0818CA
:1048B000ABE7A3F14102052AADD8373BF2E78346C7
:1048C000B6E78246C2E70246CDE7274BD4E71FFA98
:1048D00089F10229D2D80BF2262189B2B1F5E16F14
:1048E000CCD80AF2262189B2B1F5E16FC6D8D4B28C
:1048F000062CC3D81846019346F0E4F80428BDD826
:10490000002FBBD02DB2164A019B680102EB451166
:1049100002F8009002EB4512144DA1F810B0C1E965
:104920000286A1F812A00C751532591E033311F836
:10493000010F445D04F00304022C08BF203802F884
:10494000010B087808B18B42F1D103B0BDE8F08FBC
:1049500007480722394603B0BDE8F04FFFF73CB8DF
:10496000C0410020A4A706088EBF0608A9FE0608BD
:104970009FA806082DE9F047DFF874A086B08146AD
:1049800090460D4617460026B8F1000F2ED03B7812
:104990002A789A42D7E9010C26D16A68824223D14B
:1049A000AC68A4EB0C0254425441CDE9010C214601
:1049B00000935246334648460594FEF71FFE05997C
:1049C000AB6802936B68019315F80C3B0093524659
:1049D000334648460136FEF7F7FD082E07F10C076F
:1049E000D2D106B0BDE8F0870024DEE74146E7E714
:1049F000ACA806082DE9F8430446FEF7F5FF054686
:104A000028B1BDE8F8432E4900220120B2E72D4924
:104A10002046F8F78DFA014628B9BDE8F843284842
:104A200060224CF098BC2046F8F7C6FDC3B2072BB5
:104A3000064606D929462448BDE8F8430722FEF772
:104A4000CBBF2046F9F75EFF074628B3F8F7B4FD61
:104A5000051E18BF012501243846F9F753FF074604
:104A6000E0B1F8F7A9FD01348046E4B23846F9F721
:104A700049FF0746A0B1F8F79FFD01348146E4B233
:104A80003846F9F73FFF08B10134E4B2032C09D0EE
:104A9000BDE8F843FEF79CBF0446DDE78046E5E746
:104AA0008146EDE7094B76B20C2000FB063686F80E
:104AB000D45EC6F8D88EC6F8DC9EBDE8F88300BF89
:104AC000047D0020A4A70608C1A80608306E0020B7
:104AD0002DE9F04FDFF868908FB0074688461646FC
:104AE00000240DF1240A58F824300293514602A8FC
:104AF00041F0EEFC16B356F82430029D0393EB1AF6
:104B00005D420DF1100B5D41594603A841F0E0FCF8
:104B1000CDF800B023464A4629463846FEF76EFDDA
:104B20002346CDF800A04A46294638460134FEF710
:104B30004BFD202CD7D10FB0BDE8F08F3546EFE705
:104B4000D0A806082DE9F04F89B00546FEF74CFFC6
:104B5000044630B165490022012009B0BDE8F04F9C
:104B6000B6E72846F8F728FD1F28074600F3B68069
:104B70002846F9F7C7FE5D4B019443F827405C4B8C
:104B8000CDE902430546A046A146A24626464FF07F
:104B9000010B039B05AA13F801CB03939646002350
:104BA000284615F8011B19B18C4501D00A2B0CD1F0
:104BB00008AD2B448C454FF0000503F80C5C08D081
:104BC00009B0BDE8F04FFEF703BF0EF8011B01333B
:104BD000E6E7731E451C032B03D8DFE803F0243AF5
:104BE000687705A8F8F7E8FC01900136F6B2052EC3
:104BF000CFD1029B3F4803F00F0343EA844343EACB
:104C00008A5343EA092343EA0838019B1B0100EB5E
:104C10008707DBB248EA0303C7F8343F09B0BDE8B1
:104C2000F04F2AF051B905A8F8F7C6FC0290DCE76E
:104C30004E2B13D0452B13D0532B13D0572B13D0FF
:104C4000552B13D0442B04D105230BFA03F34AEA66
:104C5000030A12F8013B002BEAD1C6E70023F4E770
:104C60000123F2E70223F0E70323EEE70423ECE756
:104C7000DFF888C0002001461CF8010B984204D0E0
:104C8000072901F10100F6D14946542B14D04F2BCE
:104C900014D0422B14D04E2B14D0492B14D0572BA8
:104CA00004D105230BFA03F348EA0308894612F8F6
:104CB000013B002BDCD198E70023F3E70123F1E768
:104CC0000223EFE70323EDE70423EBE705A8F8F75A
:104CD00073FC10280446A8BF002486E706481F225C
:104CE000214609B0BDE8F04FFEF776BE647D002096
:104CF000EF1D0608306E0020CAA80608F41D06083D
:104D00002DE9F047DFF870A086B0814690460D4649
:104D100016460027B8F1000F2BD033882A889A4214
:104D200025D16C887188621A54425441F2780292FB
:104D3000B2780594CDE9003221463B4652464846BA
:104D4000FEF75CFC0599EB780293AB78019335F89C
:104D5000043B009352463B4648460137FEF734FC7D
:104D6000102F06F10406D5D106B0BDE8F087002467
:104D7000DCE74146E7E700BFDAA806082DE9F8437B
:104D80000546FEF731FE044628B1BDE8F843254943
:104D900000220120B4E72846F8F70EFC0F2806464B
:104DA00030DC2846F9F7AEFD20361F4FDFF884804F
:104DB00005464FEA86092846F8F7FEFB37F8023B1E
:104DC000984226DC012C08EB090311D0022C12D0EA
:104DD000A3F8340F28462C214CF0D4FA054668B1CC
:104DE000013501230134A3B1032CE4D1BDE8F883DC
:104DF00083F8360FEEE783F8370FEBE7A21E534236
:104E00005341EFE721460948BDE8F8430F22FEF77A
:104E1000E3BD074B002243F82620BDE8F843FEF728
:104E2000D7BD00BFE47D0020FC1D0608CAA8060807
:104E3000647D0020306E00202DE9F04F14462A4A90
:104E400085B00646894600274FF0060B0BFB07F599
:104E5000C0354FF0000819F805A0002C40D0635D64
:104E6000AAEB030041424141CDE9008330463B4675
:104E70000391FEF7C3FB03991B4ACDE9008A3B4629
:104E8000304608F10108FEF79FFBB8F1060F164AFD
:104E900005F10105DFD10137062FD7D1124FE425E7
:104EA00019F805A0A5F1E408E4B1635DAAEB0302DB
:104EB00051425141CDE900833A46062330460391E1
:104EC000FEF79CFB0399CDE9008A06233A4630465B
:104ED0000135FEF779FBEF2DE2D105B0BDE8F08F8B
:104EE0002146CAE72146EEE7ECA8060870B586B071
:104EF0000346FEF779FD044630B11A49002201202D
:104F000006B0BDE8704097E71749174E02AA184649
:104F10004CF0C7F903AD80B1032C03D1FEF758FD67
:104F200006B070BDF8F748FB02AA45F8040B3146FD
:104F3000002001344CF0B5F9EDE7032CEED1DDE9AA
:104F40000345059B01931A462946E0B22AF0D6F89C
:104F50000028E3D0019B05482A462146FEF77EFB48
:104F6000DEE700BF647D0020E4A30608ECA8060885
:104F70002DE9F043DFF8989087B0804617460C463D
:104F800015460026002F41D0B5F90030B4F90010C5
:104F9000B5F90220B5F9040095F906C0994233D15C
:104FA000B4F9021091422FD1B4F9041081422BD1EF
:104FB00094F90610A1EB0C0EDEF1000141EB0E019D
:104FC000CDE90032CDE9020C33464A464046059110
:104FD000FEF714FB059994F906300393B4F90430F5
:104FE0000293B4F90230019334F9083B00934A4626
:104FF000334640460136FEF7E7FA102E05F1080564
:10500000C0D107B0BDE8F0830021D9E73946E2E717
:1050100000A906087FB50546FEF7E6FC00285BD030
:105020002E490022012004B0BDE87040A0E72D2BDE
:1050300003D0A3F13002092A49D8042C04DD04B0BE
:10504000BDE87040FEF7C4BC2846F8F7B5FA04ABDB
:10505000621C03EB440424F80C0C15F8013F303BB0
:10506000092BFAD914462B78002BE0D1052CE6D178
:10507000BDF80430BDF904600F2BE0D8BDF906106F
:10508000A1F5FA7292B2B2F5FA6FD8D8BDF908203C
:10509000A2F5FA7080B2B0F5FA6FD0D8BDF90A0067
:1050A0008142CCDC8242CADB9142C8DCBDF90C50A3
:1050B00005F17D04A4B2FA2CC1D8084B23F83610B0
:1050C00003EBC6035A8098809D7104B070BD202BFD
:1050D000B5D101352246C5E70446C4E7843D00202A
:1050E0002DE9F04FDFF8B8B08FB0804617460C4678
:1050F00015460026A388ADF82C3023780893B4F920
:105100000290637820680693237994F905A00A90A9
:105110000793B9F1000F3CD0002F3FD02868BDF8AD
:1051200028100C9080B2AB88ADF8343081422A78D8
:1051300095F801C0B5F9023095F804E02CD14B4543
:105140002AD1BDF82C10BDF83400081A4142414163
:10515000CDE901C30092CDE903EA33465A46404601
:105160000991FEF74BFA0999079BCDF810A0CDE9FC
:105170000293069B0193089B00935A463346404690
:105180000136FEF721FA202E04F1060405F106058A
:10519000B0D10FB0BDE8F08F0021D9E73946E3E781
:1051A00015A9060810B5114B014603F1180253F872
:1051B000044B41F8044B9342F9D11B880B800B49F7
:1051C00000F11A0351F8044B43F8044B9142F9D112
:1051D00011881980054B343053F8041B40F8041B28
:1051E0009342F9D11B88038010BD00BF1C3706080D
:1051F0004F4B2DE9F04F1D78854203D020B985F043
:1052000001051D70BDE8F08F4A495A7CD1F8008035
:10521000CAB1A8F51C575968103F4FF0640AB9424B
:1052200016D30A2A71D044485960A8EB0101A0FBAB
:105230000101C1F347115A740029E0D098180132D6
:10524000C1715A74DBE701225A74C3F80480D6E7AF
:10525000012A01D14146E2E793F808C0961E1AFBE5
:105260000C11B146002E4DD0D01E02284FF0000088
:105270002CD96CF307006CF30F20D3F809406CF3C2
:1052800017406CF31F6084EA000E00F07F3B6FEA6A
:105290000E0E44F080340EF0803EA4EB0B048EEA38
:1052A00004049C60B408012C0CD0D3F80D4060407D
:1052B000C04344F08034A4EB0B0B00F0803080EA54
:1052C0000B00D860B40726F003001BD0461C03EB8C
:1052D000060E03EB000B9EF808404E45A4EB0C04B1
:1052E0008BF808400EDA02301E188145347AA4EBA0
:1052F0000C048EF8084005DD9BF80B00A0EB0C0CAD
:1053000086F808C0013AD2B289E7187C63288AD8A7
:1053100008480068A0F51C501038884283D893F8DC
:1053200008C04FF008091AFB0C114E469CE700BF5D
:10533000A0810020242600201F85EB5170B51F4C52
:10534000237D05460E463BB1D4E90623904271EB1E
:10535000030324BF00232375E36B1948984710F01B
:10536000010324D080F00203C3F340032375236BB1
:10537000616B5B19A36146EB0106012384F8503091
:10538000E6614307A06D48BF0123A5EB000548BFB8
:1053900084F85130002D03DD012084F8500070BDE9
:1053A00094F850000028FAD194F8510070BD82079B
:1053B000E7D5227D002AE4D02375E2E7A081002012
:1053C000C0810020F0B589B0044645F07BFB10F0A9
:1053D000FF0206D12D49012009B0BDE8F040FFF7DA
:1053E0007FBE2B4905222046F7F786FD30B92748B6
:1053F000152109B0BDE8F04044F0F4BE204625492F
:10540000244E01AA4BF04DFF4FF0FF33079302AD3E
:10541000002478B1062C02D1FEF7DAFA33E0F8F76F
:10542000CBF801AA45F8040B3146002001344BF0BB
:1054300038FFEEE7042CEFDD029E1F2EECD8039D13
:105440000F2DE9D8049C252CE6D8059800F57A7331
:10545000B3F5FA6FE0D80699FF29DDD8079A531CF7
:10546000402BD9D80C4B062707FB0633A3F8620064
:1054700083F86050094883F8614083F8641083F82A
:105480006520FFF79FFF09B0F0BD00BF008200203C
:10549000A4A70608E4A30608A08100208EBF060882
:1054A00037B505460846019145F00CFB01990446C5
:1054B00002462846F7F720FD68B92B5DA3F13002BC
:1054C000092A06D923F02003413B192B01D90134C5
:1054D000281903B030BD0020FBE72DE9F04FDFF8BD
:1054E0000CA19DB0804617460C4615460026A646E0
:1054F000BEE80F000DF1400CACE80F0023780C93D0
:105500009EE8030094F901300D93A3780E93237B5A
:1055100094F804B094F8149009928CE803000A936C
:105520000B90002F5FD0AE46BEE80F000DF1580C77
:10553000ACE80F009EE80300109B0F928CE803007C
:1055400023F07F4C169B95F804E0287B2A69297D7F
:1055500023F07F439C4544D1F34542D1099B9C46AF
:105560000F9B9C453DD10A9B83423AD10B9B9342B2
:1055700037D1A9EB0103594259410B9B06930A9B72
:105580000593099BCDF81C90CDE903B30E9B0293C4
:105590000D9B01930C9B00935246334640460F915E
:1055A000FEF72CF80F990B9B06930A9B0593099B1A
:1055B000CDF81C90CDE903B30E9B02930D9B019394
:1055C0000C9B00935246334640460136FDF7FCFFE4
:1055D000402E04F1180405F1180588D11DB0BDE86E
:1055E000F08F0021C9E73946DDE700BF2CA9060886
:1055F0002DE9F0418AB0044645F064FA10F0FF024C
:1056000005D1394901200AB0BDE8F04165E73749C5
:1056100005222046F7F770FC38B933484FF47E7105
:105620000AB0BDE8F04144F0DDBD20463049304EBF
:105630006A464BF036FE01AD002478B1092C02D148
:10564000FEF7C6F94DE0F7F7B7FF6A4645F8040BD9
:105650003146002001344BF024FEEEE7092CEFD157
:10566000DDF804E0BEF13F0FEAD8DDF808C0BCF178
:10567000010FE5D8039F7B1C402BE1D8049E2E2E02
:10568000DED8059D062DDBD8069C1A4B04F5742246
:1056900002F510729A42D3D807980628D0D80899F4
:1056A00001F5742202F510729A42C9D8099AFF2AAC
:1056B000C6D8114B4FF0180808FB0E3383F82C01A5
:1056C00083F820C10D4883F8217183F8226183F8A3
:1056D0002451C3F82841C3F8301183F83421FFF76F
:1056E00087FF0AB0BDE8F081C0820020A4A70608A9
:1056F000E4A3060880841E00A08100208EBF060857
:105700002DE9F04F164615461C4A87B007460C4651
:105710004FF0000BD4E9009AD4F8088066B3AB6868
:105720009845D5E9000125D1814523D1AAEB010394
:1057300059425941CDE9019ACDF800805B4638467F
:105740000591FDF75BFF05990C4ACDF800805B469B
:10575000CDE9019A38460BF1010BFDF735FFBBF19E
:10576000080F064A04F10C0405F10C05D2D107B06C
:10577000BDE8F08F0021DDE73146E6E74DA90608D8
:1057800070B586B0044645F09DF910F0FF0205D1D2
:105790002149012006B0BDE87040B1E71F4905224C
:1057A0002046F7F7A9FB38B91B4840F2FF3106B095
:1057B000BDE8704044F016BD20461949184E01AAB4
:1057C0004BF06FFD02AD002478B1042C02D1FEF73E
:1057D000FFF81FE0F7F7F0FE01AA45F8040B314689
:1057E000002001344BF05DFDEEE7042CEFD1029A6E
:1057F000072AECD80B4B0C480C2101FB0233039A0F
:10580000C3F82827049AC3F82027059AC3F8242749
:10581000FFF7B6FF06B070BDC0880020A4A7060839
:10582000E4A30608A08100208EBF06082DE9F04FF2
:10583000DFF804B1A1B0804617460C461546002695
:10584000A646BEE80F000DF1480CACE80F00237926
:105850000A93A3680B939EE80700A38A0D93E38A3B
:105860000E93238B0F93638B94F800A094F80C9005
:105870000C908CE807001093002F5BD0AE46BEE87A
:105880000F000DF1640CACE80F009EE807002B78C8
:1058900053458CE807004BD12B790A9A934247D1A4
:1058A000AB680B9A9A4243D12B7B4B4540D10C9A63
:1058B00082423DD1179A8A423AD118991F9BCB1A3E
:1058C00059425941109B08930F9B07930E9B0693D7
:1058D0000D9B05930C9B1191CDE903930B9B0293B8
:1058E0000A9B5A46CDE900A340463346FDF786FEA3
:1058F0001199109B08930F9B07930E9B06930D9B8A
:1059000005930C9BCDE903930B9B02930A9B5A468C
:10591000CDE900A3404633460136FDF755FE042E7F
:1059200004F11C0405F11C058AD121B0BDE8F08FFB
:105930000021C7E73946DCE75EA906082DE9F043F8
:105940008DB0044645F0BEF810F0FF0205D13E4987
:1059500001200DB0BDE8F04368E73C490522204630
:10596000F7F7CAFA38B938484FF47E710DB0BDE880
:10597000F04344F037BC20463549354E01AA4BF080
:1059800090FC02AD002478B10A2C02D1FEF720F879
:1059900057E0F7F711FE01AA45F8040B3146002045
:1059A00001344BF07EFCEEE70A2CEFD1DDF80880E5
:1059B000B8F1030FEAD8DDF80CE0BEF1010FE5D82D
:1059C000DDF810C0BCF1060FE0D8059F214B07F5AC
:1059D000742202F510729A42D8D8069E062ED5D8A7
:1059E000079D05F5742202F510729A42CED8089CE4
:1059F000B4F5004FCAD20998B0F5004FC6D20A9943
:105A0000B1F5004FC2D20B9AB2F5004FBED2124B85
:105A10004FF01C0909FB0833A3F8960783F880E7C9
:105A20000E4883F884C7C3F8887783F88C67C3F877
:105A30009057A3F89447A3F89817A3F89A27FFF76D
:105A40007DFF0DB0BDE8F08320890020A4A70608E3
:105A5000E4A3060880841E00A08100208EBF0608F3
:105A60002DE9F3473649DFF8D89001AA4BF019FC2D
:105A70004FF0000A4FF0FF3557465446D0462E46A9
:105A800068B9BAF1040F50D03ADCBAF1020F13DC56
:105A90002C492B463246012040F04AFE0EE0BAF176
:105AA000040F09D8DFE80AF0030D12171C00F7F7FE
:105AB00083FD064603281BD9FDF78AFF02B0BDE827
:105AC000F087F7F779FD05468728F4E7F7F774FDC7
:105AD00080463F28EFE7F7F76FFD04463F28EAE7E7
:105AE0000378482B03D0562BE6D1012700E000278E
:105AF00001AA494600200AF1010A4BF0D2FBBFE798
:105B0000BAF1050FD8D1882303FB0655A4010E4E28
:105B100004F47C6408F03F0844EA080406EB4505F9
:105B200044EA4734A5F8F047C8E7882303FB065248
:105B3000054B03EB4203B3F8F077C7F34037E2E7D6
:105B4000E4A3060890890020A08100201FB5094B1E
:105B50000293094B0193094B0093094A094B0A49E7
:105B60000A48FDF77BFD0A490A4805B05DF804EBD9
:105B7000FDF774BD2DA3060836A306083FA306084B
:105B800051A306084BA30608F9A2060880A9060837
:105B900098A90608B2A90608F8B50C480C4D0D4E98
:105BA0000D4FFDF75BFD00246CB93268C2F5007241
:105BB000920022B157F824100848FDF74FFD013438
:105BC000252CF1D1F8BD55F82420F2E7BBA9060831
:105BD000D4380020D030002038370608D1A9060874
:105BE0002DE9F84F054644F06DFFDFF8EC800446E0
:105BF000D8F80090C0B93048304D314FFDF76AFCFD
:105C0000012655F8041B59B10B783BB106FA04F391
:105C100013EA090F02D03846FDF706FD0134F0E71C
:105C2000BDE8F84FFDF784BC024626492846F7F741
:105C300063F978B92448214C214DFDF74BFC54F809
:105C4000041B0029ECD00B78002BF8D02846FDF778
:105C5000EBFCF4E72B78DFF864B02D2B03BF0135A4
:105C600004F1FF344FF0010A4FF0000A00265BF800
:105C7000047B1FB9BDE8F84F40F0BABC2246394654
:105C80002846F7F739F9A8B90120B040BAF1000F5A
:105C90000AD0F7F72FFD0D48FDF71CFC39460C48DC
:105CA000BDE8F84FFDF7DABC40EA0900C8F800008B
:105CB0000848F1E70136DAE7DFA90608CC3706081D
:105CC000E9F706088FB70608E9A90608F5A9060846
:105CD00024AA0608FEA90608743900202DE9F84F09
:105CE000054644F0EFFE334F0446BE68C8B932485B
:105CF000324DDFF8D880FDF7EDFB0127E3B205EB6D
:105D00008302D2F8341141B107FA03F3334202D0CF
:105D10004046FDF789FC0134F0E7BDE8F84FFDF798
:105D200007BC024626492846F7F7E6F860B9254839
:105D3000254C264DFDF7CEFB54F8041B0029ECD072
:105D40002846FDF771FCF7E72B78DFF87CB02D2BA8
:105D500003BF013504F1FF344FF0010A4FF0000A90
:105D60004FF000095BF8048BB8F1000F03D1BDE8D8
:105D7000F84F40F03DBC224641462846F7F7BCF8B4
:105D8000A8B9012303FA09F3BAF1000F0BD026EAF0
:105D900003030F48BB60FDF79DFB41460D48BDE87E
:105DA000F84FFDF75BBC33430B48BB60F3E709F1E9
:105DB0000109D7E744470020DFA906081C37060879
:105DC0008FB70608E9A9060850380608E9F706085B
:105DD000F5A9060824AA0608FEA90608F8B50C4C81
:105DE0000C4E0D4F2D252068FDF774FB616811B135
:105DF0003046FDF719FCA16811B13846FDF714FCD7
:105E0000FDF796FB013D04F11004ECD1F8BD00BF95
:105E10007838060806AA06080CAA06082DE9F047F5
:105E2000814644F04FFE4D4E0446376800BB4C4857
:105E30004C4D4D4EFDF7F8FB4FF00C0808FB04F3FA
:105E40005B5D5A1E012393403B4206D0204619F069
:105E50004DF801463046FDF7E7FB0134182CEDD133
:105E600017B94248FDF736FBBDE8F047FDF760BBC8
:105E700002463F494846F7F73FF8054678B93D489E
:105E8000FDF728FB2C46384D204619F02FF8013439
:105E900001462846FDF7C8FB1A2CF5D1E4E799F82E
:105EA00000302D2B03BF09F1010904F1FF344FF03D
:105EB000010A4FF0000A4FF00008404619F016F8AA
:105EC0002246054601464846F7F716F800283BD11A
:105ED000BAF1000F1FD0B8F1180F0BD16FF07F434C
:105EE00033602548FDF7F6FA29462448BDE8F04717
:105EF000FDF7B4BBB8F1190F01D17368F0E7204B7F
:105F00000C2202FB083898F82C345A1E01239340C7
:105F10001F433760E5E7B8F1180F03D1C6F800A0BA
:105F20001848DFE7B8F1190F01D17760F8E7144B93
:105F30000C2202FB083898F82C345A1E0123934097
:105F400027EA03073760EBE708F10108B8F11A0FF9
:105F5000B3D1BDE8F04740F04BBB00BFE43E0020AA
:105F600012AA0608483B060823AA06081CAA060827
:105F70008FB7060828AA0608F5A9060824AA060865
:105F80001C370608FEA90608F0B585B0044644F0A3
:105F900099FD04283DD1631E2546E11C13F8012F0D
:105FA000A2F16100192898BF203A8B421A70F5D1EE
:105FB0001A4F261D15F8011B019138464BF0E2F9E6
:105FC00020B1019928464BF0DDF920B105B0BDE8BC
:105FD000F040FDF7FDBCB542ECD120461FF04EF974
:105FE0000F48104CFDF776FA0C4901231A5D11F8A1
:105FF000010B04AD2A440133052B02F8080CF5D13E
:10600000002309488DF80C3002A9FDF727FB05B0E5
:10601000F0BD0028E4D0FDF7DBFCE1E7803C06089A
:1060200033AA0608D08D00200FAA06087FB5194BA9
:1060300093F8302C012A29D193F8353C0D2B05D04B
:10604000154807B05DF804EBFDF744BA11220021B2
:1060500001A84BF080F9A6238DF8003041238DF87C
:106060000130EB238DF803300C4B1B788DF8043096
:10607000B22315218DF80530684603238DF80210F0
:106080008DF806301FF0EFFA0548DAE707B05DF843
:1060900004FB00BFA081002039AA0608100A0020D6
:1060A00048AA060810B5204C2048A17AFDF7D6FA78
:1060B0001F48FDF763FAA1791E48FDF7CFFAE17991
:1060C0001D48FDF7CBFA217A1C48FDF7C7FA617A23
:1060D0001B481C4CFDF7C2FA1B48FDF74FFAB4F9F8
:1060E0001030B4F90E20B4F90C101848FDF7B6FAC8
:1060F000B4F91C30B4F91A20B4F918101448FDF79B
:10610000ADFAB4F91420B4F91210B4F916301148EC
:10611000FDF7A4FAB4F92020B4F91E100E48BDE82A
:106120001040FDF79BBA00BF0001012062AA0608DB
:106130007BAA06088FAA060897AA0608A0AA06083E
:10614000A8AA060894480020B0AA0608C3AA060810
:10615000D2AA0608E0AA0608EEAA060808B51F4B50
:106160001F4C1D68A06819F0B7FA284619F0B4FA58
:10617000A06841798B0704D4036841F002019B6950
:10618000984700210846F9F7C1FD00210120F9F7E1
:10619000BDFDA068FAF761FC70B101210020F9F79C
:1061A000B5FDA068FAF77AFC01462846FAF7EDFB40
:1061B00000210846F9F7AAFD2846FAF74EFC002808
:1061C000E7D001210846F9F7A1FD2846FAF766FC59
:1061D0000146A068FAF7D9FBD7E700BF147B00207F
:1061E000483F0020F7B50546FDF7FEFB044620B109
:1061F00003B0BDE8F040FDF7EBBB28461D491D4F3D
:1062000001AA4BF04EF82646254640B90B2D18D969
:10621000014619480B22FDF7DFFB03B0F0BD44B186
:10622000012C0AD001AA3946002001344BF039F87C
:10623000EBE7F7F7C1F90546F4E7F7F7BDF90646CE
:10624000F0E7022C0DD1A6F57A73B3F57A7F05D964
:106250000A484FF4FA624FF47A71DCE7084B23F8EE
:106260001560074B074833F915202946FDF7F6F965
:10627000D3E700BFE4A30608CAA8060838B6060894
:10628000E0010120FCAA060870B50446FDF7ACFB4E
:10629000C0B11F4B5E680136304618F027FE344609
:1062A0000546E8B901341A2CA8BF0024204618F08E
:1062B0001DFE0546A0B9B442F4D1BDE870401548B2
:1062C000FDF75CB92046F7F777F9044618F00EFEA3
:1062D000054628B921461048BDE87040FDF7BEB913
:1062E0000B4B5C6019F0BEFC0C4821462A46FDF7BA
:1062F000B5F9192C9DBF0A480C2101FB04000020B0
:10630000BDE8704098BF90F82C0419F0C7BC00BFDE
:10631000100A002009AB06081DAB060833AB0608BF
:106320001C37060838B51749052204464BF040F8DB
:1063300058B9154A13781BB901211170134A13700B
:10634000BDE838401248FDF719B91249032220462A
:106350004BF02EF880B90C4D0C4C2B7843B12378C0
:1063600033B10D48FDF787F900232B70237038BD3A
:106370000A48FDF703F9F7E7BDE838400848FDF79C
:106380007AB900BF55B00608107B0020117B0020B1
:1063900048AB0608EDB106085EAB060895AB0608EB
:1063A000A9AB06082DE9F0434C498DB0F6F7C0FDC6
:1063B000044600284BD14A4D2B78012B4BD1FCF7DA
:1063C00083FE4848162306AA55210068FAF722FEE4
:1063D0000C20FCF779FE204601AB1C18C3B29A1DB5
:1063E000D2B20CA9CE18023316F8177C16F8181C76
:1063F000DBB241EA0721934224F8021BF1D10630B7
:106400001228E9D1BDF92A60BDF92C40BDF90490EC
:10641000BDF90680BDF908E0BDF90AC0BDF90C70F0
:10642000BDF90E00BDF91010BDF91220BDF91430F0
:10643000A5F81890A5F81A80A5F81CE0A5F812C0D8
:10644000AF82E882A981EA812B82EE832C840DB091
:10645000BDE8F04326E6022BF9D101463D20FAF7CC
:10646000C5FA1920FCF749FC16215520FAF7C8FA9D
:106470003220FCF742FC1C4A204607AB1E18C3B270
:10648000991DC9B2D4186778D45C0233DBB244EAF0
:1064900007248B4226F8024BF4D106301228ECD1A7
:1064A0000C213D20B2F91260B2F91440FAF79EFABD
:1064B0001920FCF722FCBDF91C90BDF91E80BDF926
:1064C00020E0BDF922C0BDF92470BDF92600BDF958
:1064D0002810BDF92A20BDF92C30A9E7B8AB060871
:1064E00094480020B8480020295E00202DE9F0479C
:1064F0008CB0074610F8013B202BFAD00025204C29
:10650000DFF88480DFF88490DFF884A02E4601A9AC
:1065100020460EF01DFF394601A84AF0A2FFE0B167
:1065200001A94046FDF780F8494601A844F0C0FAA9
:1065300000BB20460EF0DAFF124B014600782028FF
:106540000CBF50461846FDF76FF8FCF7F1FF2046E8
:10655000FDF7E6F9FCF7ECFF0136013540F2452383
:106560009D4204F10B04D2D10EB940F041F80CB0B9
:10657000BDE8F08700212046FDF7C6F9E5E700BF3A
:10658000241E06080FAA060854A606084BF906089A
:106590005AA606082DE9F04F2DED028B8DB0067836
:1065A000202E054600F10100F9D0284644F08AFA71
:1065B000044618B1012822D12A2E20D18248834DC9
:1065C000DFF81C82FCF7DAFF002640F24527284658
:1065D00001A90EF0BDFE01A94046FDF725F80136E0
:1065E00028462146FDF790F9FCF7A2FFBE4205F1CF
:1065F0000B05ECD10DB0BDEC028BBDE8F08F3D2159
:1066000028464AF0BFFE002800F0D6800346984690
:1066100013F8012D202AFAD0A8EB05080130064610
:1066200010F8013B202BFAD0684F4FF000095FFAB9
:1066300088F840F2452B01A938460EF089FE01A8E2
:1066400044F040FA01A9024682462846F6F754FC77
:106650005E4B044610BBC24520D10B2202FB09331E
:106660009B7903F00F08B8F1060F22D1584901A811
:1066700044F01EFA0446304644F024FA0246B4B907
:106680003378222B13D1331813F8013C222B0ED16F
:10669000821E711C38460EF0F5FFABE709F10109C7
:1066A000D94507F10B07C6D13FF0A2FFA2E731465B
:1066B000F0E713F0C0030AD0402B4DD04548FCF75B
:1066C00063FF3846FDF72CF9FCF732FF92E7337889
:1066D000002BF3D0404930464AF0B3FE0446304622
:1066E00044F0F0F98442E9D13046F6F783FE3846AB
:1066F000B0EE408A0EF007FF07EE900AF8EEE77A58
:10670000F4EEC87AF1EE10FAD8D838460EF00CFF45
:1067100007EE900AF8EE677AF4EEC87AF1EE10FA16
:10672000CCDBB8F1050F0CD118EE104A38460EF04C
:10673000DDFEB8F1050F30D8DFE808F02E2E38382E
:106740003A3CB8F1040F304603D1F6F71BFF04467C
:10675000ECE7F6F731FFFAE738460EF077FF90F8EE
:1067600004B0814625462346A246AB4500D91BB15D
:10677000BAF1000FA2D0D9E7D9F80030314653F86A
:106780002500F6F7D5FB002805BF2C460123002382
:106790004FF0010A0135E8E7047001A90F48FCF742
:1067A00043FF00213846FDF7AFF823E70480F4E704
:1067B0000460F2E70460F0E728460DB0BDEC028B00
:1067C000BDE8F04F92E600BFBEAB0608241E0608E7
:1067D0004BF90608E9AB0608D0AB0608DEAB0608A5
:1067E00054A606082DE9F04FBD4BBE481968BE4EB1
:1067F000BE4CDFF83493A7B04FF47A73B1FBF3F1DA
:10680000FCF72CFF0BA8F6F793FCB6F94E2C0BA95E
:106810001BA842F097FC1BA9B548FCF71FFF20F00E
:1068200009FAB44B1B7804EB83036422D3F86C356C
:106830000093B14BB0FBF2F102FB11021B78AF48A1
:1068400092B289B2FCF70AFFAD4BAE481968AE4B65
:10685000B1FBF3F1FCF7E8FEAC4B1F68002504F236
:106860007C5804F5B36A0123AB403B420DD0590676
:106870000BD058F8253043B119F805205AF82510E7
:1068800053F82220A248FCF7CFFE0135082DEAD1AB
:10689000FCF74EFE9F489C4DFCF770FE0EA8F3F7E8
:1068A000E3FB0E999C48B1FBF5F1FCF7D7FE0F997D
:1068B0009A48B1FBF5F1FCF7D1FE10999848B1FB6D
:1068C000F5F1FCF7CBFE11999648B1FBF5F1FCF719
:1068D000C5FE954B1B78002B14BF0123022304EB4C
:1068E0008303D3F8C015099120F025FC04EB800048
:1068F000D0F8C025089220F033FC04EB8000D0F8DB
:10690000C035079320F048FC04EB8000D0F8C09518
:1069100020F054FC054620F0A1FC074620F086FC40
:10692000804618F0CDFA04EB800004EB8808D0F81C
:10693000C005049004EB8707D8F8C005039004EB6A
:106940008505D7F8C0050290D5F8C0050999DDE99D
:106950000732CDE900907548FCF780FE744B1B6848
:10696000DA031AD510F0FCFA0546B0B101467148B9
:10697000DFF81882DFF81892FCF770FE0027B8F9EC
:106980000220394648460137FCF74EFEFBB29D42D5
:1069900008F11008F3D8FCF7CBFD674B674A1D8858
:1069A000674B68491B686848DFF8E891DFF8E881C1
:1069B000664FDFF8E8B1DFF8E8A1C3F500739B008C
:1069C000FCF74CFE624A634B6348D31A634AADB28C
:1069D00029461288FCF742FE6148FCF7CFFD0025EE
:1069E00059F8041B5F48FCF71FFE5846FCF772FD80
:1069F00018F8011B002940F00E815B48FCF76AFD86
:106A00005A48FCF767FD57F8041B002940F007813E
:106A10005548FCF7B3FD0135042DE1D1544B5548E1
:106A2000198BFCF701FE01201FF05CF8054658B1F8
:106A300007EE900ADFED506AF8EEE77A86EEA77A65
:106A4000FDEEC77A17EE905A03201FF04BF803466D
:106A500058B107EE900ADFED486AF8EEE77A86EE65
:106A6000A77AFDEEC77A17EE903A002007931FF041
:106A700039F8079B58B107EE900ADFED3F6AF8EE50
:106A8000E77A86EEA77AFDEEC77A17EE900A0090B5
:106A9000B6F8541C39483A4EDFF808812A46FCF70C
:106AA000DDFD3848FCF716FD356825F0004525F07A
:106AB0007F050127002D40F0B680FCF739FD3368D3
:106AC0005B017AD512A80EF045FD002875D1129B06
:106AD000B3F5117F9EBF2C480B2505FB030063E037
:106AE00024260020F9AB0608A08100201C370608E8
:106AF00013AC06083C4800203D48002024AC0608A2
:106B0000D405002049AC060840420F00FC000120DB
:106B100059AC060861AC060876AC060888AC0608D5
:106B20009AAC0608ACAC060884400020BEAC06084F
:106B3000F80001201AAD0608182E002000000220DF
:106B4000D0300020001800004EAD060800410020A3
:106B5000008000080040000886AD0608703900205B
:106B6000C0AD0608D3AD06081EAA0608F1AD06089A
:106B7000E0010120FBAD0608002474490BAE0608B5
:106B8000F000012048AE0608241E06081C3E002026
:106B90003FAD0608EC3C0608F03E0020DBAD0608E1
:106BA000EAAD060824AA060888BF28461BA90EF0ED
:106BB000CFFB28481BA9FCF75EFD274D2748FCF7B3
:106BC00089FC2868FCF728FC00283FD012A9286817
:106BD000FCF763FC9DF85C109DF86830199A20481A
:106BE000FCF722FD169911B11E48FCF71DFD149902
:106BF00011B11D48FCF718FDFCF79AFC1B4B1B78E4
:106C000033B104EB83041A48D4F83C16FCF726FD94
:106C100027B0BDE8F08F5046FCF706FDF0E6504681
:106C2000FCF71CFDF7E695FAA5F3B3FA83F307FA30
:106C300003F2062B25EA02057FF73CAF04EB830342
:106C40004046D3F8C415FCF7EFFC33E70948FCF7DE
:106C500041FCD1E75FAE0608C447002073AE0608CA
:106C600079AE060897AE0608A0AE0608143E0020CE
:106C7000BCAE0608AFAE06082DE9F04F2DED028B35
:106C800043489FED448A95B0FCF7E8FC00252F4669
:106C9000A84608A9E8B21EF09DFE9DF82430002BFE
:106CA00054D0129C4CB107EE904AB8EEE77AC8EE89
:106CB000077AFDEEE77A17EE904ADDF830900D9BEB
:106CC0004FEAE47B09FB0BF1A9FB040604FB03116B
:106CD00041F28833C01841EB06014FF47A72002369
:106CE00044F032FDDDE910A1614306460AFB0B1BAF
:106CF00041F28833A4FB0A01C0184FF47A724FF0B6
:106D000000034BEB010144F01FFD042D4FF47A7298
:106D10000E9BB3FBF2F306934FF00A0318BF3F1824
:106D200090FBF3F203FB1200CDE9042096FBF3F293
:106D300018BFB04403FB1266CDE90226CDE9009AE4
:106D4000089A154823462946FCF788FC01351B2D77
:106D50009FD108A81EF02AFE0A9A08990F484FF4FE
:106D60007A73B2FBF3F30C9AFCF778FC0A2297FBD8
:106D7000F2F302FB137798FBF2F10948009702FB4C
:106D80001182FCF76BFC15B0BDEC028BBDE8F08FF7
:106D9000D6AE0608002474491DAF060852AF060897
:106DA00074AF06082DE9FF471B481C4C1C4E1D4FB5
:106DB000DFF87480FCF752FC0025A379E27994F89F
:106DC00008A006EB830306EB8202DB69D2F8549637
:106DD00003932046F8F73BF800F141012046029169
:106DE000F8F740F8DDE902130246BAF1000F0CD0C3
:106DF000CDE900A94046FCF731FC0135312D04F105
:106E00000C04DAD104B0BDE8F087CDF80090384624
:106E1000FCF724FCF1E700BFA2AF06087839002098
:106E20001C370608CEAF0608BEAF06082DE9F047AE
:106E3000B44E73792DED028B002B3ED096F828309E
:106E4000B14A03EB430002EB4000590090F8A6065C
:106E5000002800F0CE81012800F0AA81C81802EBBA
:106E6000400090F8A706002800F0AD81012802D16B
:106E7000A6480024C483C81802EB400090F8A80676
:106E8000002800F0B982012802D1A048002404841F
:106E90000B4402EB430292F8A936002B00F0AF82BC
:106EA000012B40F0F0809A4B1B68D80440F1B88267
:106EB00040F2DC50954B5884E5E0944C954DA36A24
:106EC000B5F95A0CD905B0EE408A03F4807A00F186
:106ED000BA81D4F8C070D5F8E88C95F8EC1C17F49A
:106EE0008079A0F2DC5314BF98F80DC098F808C060
:106EF00013F5FA7FC0F26A81B3F5FA7F00F37C8163
:106F00001AB2002AB8BF524292B2914240F3E282D2
:106F10009FED810A46F0FAFFA083BAF1000F40F01E
:106F20005E81B5F9620CB9F1000F00F0BE80A0F2ED
:106F3000DC5313F5FA7F98F80DC095F8EC1CC0F2FD
:106F4000BE80B3F5FA7F00F3AD811AB2002AB8BF54
:106F5000524292B2914240F367829FED6F0A46F02F
:106F6000D5FFE083BAF1000F40F0B280B5F96A0CAA
:106F7000B9F1000F00F0B980A0F2DC5313F5FA7FED
:106F800098F80EC095F8ED1CC0F2B980B3F5FA7F01
:106F900000F361811AB2002AB8BF524292B2914204
:106FA00040F3C1829FED5C0A46F0B0FF404200B260
:106FB0002084B9F1000F00F0B98098F8113098F8EA
:106FC0000FC0A28B554913FB00F01CFB02F2E38BB0
:106FD00098F810C01CFB03F381FB00C8C017C0EB7E
:106FE000681881FB02C0D217C2EB6012A28381FB3A
:106FF0000321DB170FFA88F8C3EB6113A4F8208094
:10700000E38303201EF05AF9B5F83E9C4FF4FA6270
:107010004946F4F74BFFA0EB090080B24FF47A72B7
:10702000C9F5FA6900FB02F292FBF9F291B2B1F5EF
:107030007A7F80F05E813948A0FB0131490904EB79
:10704000410392B2B3F9C4C0B3F9C6306FF0630E16
:10705000A3EB0C030EFB012203FB02F280FB0230C8
:10706000D317C3EB601363449BB232791BB26384C2
:1070700032B968F30F0263F31F42E3693263F362CC
:107080007A0600F13981264B1B685B0707D5BDECFA
:10709000028B2448BDE8F0470021F8F7CAB9BDECDF
:1070A000028BBDE8F0470AF051BDA0F2DC5313F5A6
:1070B000FA7F98F808C095F8EC1CBFF642AF9FED38
:1070C0001A0A46F023FFE083BAF1000F3FF44EAFF7
:1070D00094F84030B5F96A0C002B3FF449AFB4F98D
:1070E0004400B9F1000F7FF447AFA0F2DC5313F571
:1070F000FA7F98F809C095F8ED1CBFF647AF9FEDF1
:107100000A0A51E77C4300201C370608E0010120F1
:10711000F4000120A0810020000000001F85EB5139
:10712000F0000120203A0020FFFFF9C3D34FB4F94B
:107130001C003B78222B08BFD14BB0EE480A08BF99
:10714000186000210FF0FCFD3B78222B08BFCC4BD0
:1071500000B208BF5860A08306BFB4F91E00986053
:10716000B4F91E00B0EE480A01210FF0E9FD3B78AA
:10717000222B08BFC24B00B208BFD860E08306BF15
:10718000B4F920001861B4F92000B0EE480A0221D9
:107190000FF0D6FD3B78D4F8C070222B08BFB84B57
:1071A0000FFA80F8A4F8208008BFC3F8148028E7FD
:1071B000B44800248483C81802EB400090F8A70666
:1071C00000287FF453AEAF48F48D53E69FEDAE0A2E
:1071D00046F09CFEA083BAF1000F3FF4A2AE94F8F3
:1071E0003830B5F9620C002B3FF49DAEB4F93C0089
:1071F00099E6A448B48DDDE74FF4FA735B1A4FF4B7
:10720000FA72C1F5FA7102FB03F393FBF1F31BB2BF
:1072100007EE103ADFEDAC5A9FEDAC0AB8EEC77A34
:1072200007EE90CA27EE257ABBEE096AA7EE076A39
:10723000F8EE676A27EE007ADFEDA57AE6EE267AA9
:1072400027EE270A66E694F83030002B3FF441AE73
:10725000B4F934003DE64FF4FA735B1A4FF4FA7256
:10726000C1F5FA7102FB03F393FBF1F31BB207EED6
:10727000103ADFED955A9FED950AB8EEC77A07EE02
:1072800090CA27EE257ABBEE096AA7EE076AF8EEE8
:10729000676A27EE007ADFED8E7AE6EE267A27EE31
:1072A000270A81E64FF4FA735B1A4FF4FA72C1F5BC
:1072B000FA7102FB03F393FBF1F31BB207EE103AF2
:1072C000DFED815A9FED810AB8EEC77A07EE90CACA
:1072D00027EE257ABBEE096AA7EE076AF8EE676A21
:1072E00027EE007ADFED7A7AE6EE267A27EE270A95
:1072F00035E6664B1B88B8E6B4F9E0206449D3173D
:1073000081FB0212B5F8F81CC3EBA2056D1A2DB271
:1073100007EE905AB8EEE78ADFED5E7A28EE278A0C
:10732000B0EE480AF4F706FBFDEEC87A17EE903A85
:107330002033402B67D8B42D0CDDDFED576A9FED6D
:10734000577AF0EE487AF4EEC77AF1EE10FA38EE9A
:10735000668AF6DCDFED527AB4EEE78AF1EE10FAD7
:107360000CD5DFED4D6A9FED4F7AF0EE487AF4EEE2
:10737000C77AF1EE10FA38EE268AF6D4DFED4A7AB3
:10738000B4EEE78AF1EE10FA40DDDFED487A37EE31
:10739000C88A68EE087A9FED467A9FED466ADFED6F
:1073A000466AA7EE876A9FED457AE7EE866A68EE41
:1073B000275AA7EEA67AA5EE878AB4F91E3007EE03
:1073C000103AB4F91C30B8EEC77A06EE903A68EE7F
:1073D000477AF8EEE66AE6EE807A26EE888AFDEED7
:1073E000E77AA7EE008A17EE903ABDEEC88AA3832B
:1073F00018EE103AE38346E62248348E47E5214BE7
:10740000728E5A843FE69FED2E8AD6E7DFED2D7A05
:10741000B4EEE78AF1EE10FABBD5DFED217AB6E7DC
:107420000FF074FD00B245E5002B3FF73DAF3FF490
:1074300094ADA0F57A734FF4FA72C1F5FA7102FBBC
:1074400003F3B3FBF1F3A3F5FA731BB207EE103AA3
:107450009FED1D5ADFED1D5AB8EEC77A07EE90CAB0
:1074600027EE057ABBEE096AA7EE076AF8EE676AAF
:1074700027EE257ADFED167A36E700BF033C0020C1
:10748000EC7A0020E0010120FFFFF9C3083E002054
:107490006766666635FA8E3CDB0FC940E4CB164161
:1074A000DB0F49C0E4CB16C1DB0FC93FDB0F4940FE
:1074B0009A7C2E36FAAF4FB93587083CA4AA2ABE6B
:1074C00000000000DB0FC9BF0AD7233C0AD7233DC9
:1074D00000401C45002B3FF791AE3FF419ADA0F5DD
:1074E0007A734FF4FA72C1F5FA7102FB03F3B3FB3E
:1074F000F1F3A3F5FA731BB207EE103A1FED0E5A23
:107500005FED0E5AB8EEC77A07EE90CA27EE057AFD
:10751000BBEE096AA7EE076AF8EE676A27EE257ADE
:107520005FED157A8AE6002B3FF797AE3FF43AAD50
:10753000A0F57A734FF4FA72C1F5FA7102FB03F306
:10754000B3FBF1F3A3F5FA731BB207EE103A1FED8C
:10755000225A5FED225AB8EEC77A07EE90CA27EE9C
:10756000057ABBEE096AA7EE076AF8EE676A27EEAE
:10757000257A5FED297A90E62DE9F04FDFF8289221
:1075800099F9D63F012B97B002DD99F9D93FDBB9C4
:107590007B4C23685F073FD5DFF810A279480021B4
:1075A000F7F747FFDAF800305E033DD4216821F099
:1075B000004323F07F03002B59D101F00403002B7B
:1075C00070D017B0BDE8F08F99F9D81F89F8D13F76
:1075D0004FF0180E4FF492624E461EFB012E03F13F
:1075E000FF3C002701E0782F0FD006EB0E050FCDF2
:1075F00006F592640FC495E80300BC4584E80300D7
:1076000006F1180607F10107EDD15D4C0023A9F83A
:10761000D83F23685F07BFD4DFF890A10AF096FA3D
:10762000DAF800305E03C1D557482B21F3F716FF77
:107630000028BBD02168554B0B40002BB7D1544AD2
:10764000544B127803EB42035B78002BAFD011F060
:10765000040340F06082504ED6F8C020150440F17B
:10766000628221F0004222F07F02E2B101E001F0EB
:107670000403DFF83C8198F811200A2A6CD0464EAA
:10768000B26AD2079BD4002B9BD141F20242FF2366
:107690000F20A8F88C2F88F88E3F17B0BDE8F04F68
:1076A00018F0FCBA3C4E00230DF157008DF857300E
:1076B00036F0F4FB9DF85730002B46D1DAF8003055
:1076C000DFF8EC8043F40003CAF80030236843F08D
:1076D0000C032360002488F8044D08F6085308F6CC
:1076E00008721C601C7108339A42FAD11AF092FB9E
:1076F000B6F9E030294A2A4D82FB0312DB17C3EBAF
:10770000A2031BB2A8F8F83CA6F8E4300023C6F8A0
:10771000E8302B6818034DD499F80730D3B1DAF864
:107720000030D90716D5072018F0B8FA1D4B1B6892
:10773000C8F87C3F35F048FED8F8883FC8F8800F7D
:10774000C8F8843F17B0BDE8F08FDAF8003043F492
:107750008043B5E70620E7E798F81020632A8ED823
:10776000104AD8F804001268A2F51C52103A904250
:1077700085D3064A0A40002A3FF421AF7FE700BFC5
:10778000F0000120203A00209C8E00208006FF7F20
:10779000BC5D0020F01B0608E001012067666666FC
:1077A000F400012024260020284D0020F8000120AC
:1077B000A08100209B4B80201C7040F03FFB0446C2
:1077C00070B1994F3B68984200F07281D7F8DC3075
:1077D0009C4200F06481D7F8B8319C4200F0568199
:1077E000924B1B78012B97D1914C278827B1B4F885
:1077F00002B05F45C0F064811A466380237922801D
:107800000BB100232371802017F044FD07460028A8
:1078100000F06181802117F09FFEFA79854B88F88E
:10782000080F53F8223097F904000093B3F5613F35
:107830000CBF022300230293022200230192802125
:107840001A4617F0E3FE7C4BC8F80C0F5B8807461E
:107850007A4803EB4303A0FB033040094022012197
:10786000F4F724FB88F8100F002F00F03481DAF8C9
:10787000003061882F68258803F01002704B93F860
:1078800008E0A3688D422CBF00210121C3F3800CC6
:10789000002A0CBF6046002009916A49089014BF75
:1078A000604600200D7807906749684A0978109172
:1078B000AEF1010017F4006FB0FA80F04FEA5010FB
:1078C00008BF00206249069007F00200146811907A
:1078D000604AC6F8F8200020C8F8140FC1E901007A
:1078E000C1E90300B8F82A1FA8F8281F14F0080FF0
:1078F00002F5C67102F54672C6F80021C3F3C00254
:1079000008BF02460592C3F3C0120E92C3F3801261
:107910000F92C3F340120D92C3F300120C92C3F303
:107920004002C6F8FC1098F8307FC8F82C0F0B9274
:1079300003F0010203F480730493C4F3001304F012
:10794000200683460A92129304F0040401215FFA90
:107950008BF21F2A19D8DFE802F0114127272727C9
:107960002727272745872421518F8B4D491E3535E1
:107970003583106194187F5D595535B1D8F82C3F87
:1079800001FA0BF00343C8F82C3F202A00F0A7802F
:107990000BF1010BDBE7002FF0D1F6E7002EF7D05B
:1079A000ECE7002CF4D0E9E713920FF0D9FA0BF1D1
:1079B000FF338342139A4FF00101E6DC049B002B56
:1079C000DCD1E2E7139211F097FD00EBCB00139AA4
:1079D00030F89C3C0121002BD0D1D6E7049B002B32
:1079E000D6D0CBE7109B002BC8D1D1E7089B002B4A
:1079F000C4D1CDE7079B002BC0D1C9E7119B002B59
:107A0000C6D0BBE70E9B002BB8D1BEE70F9B002B67
:107A1000B4D1BAE70D9B002BB0D1B6E70A9B002B7F
:107A2000ACD1B5E7CC300020382E002050470020E4
:107A30004447002090170608EC3F0020D34D621009
:107A4000F43E0020033C0020063E0020FC00012004
:107A5000B4900020E40201200C9B002B8ED194E70F
:107A6000099B002B94D089E7059B002B86D18FE7DB
:107A7000129B002B8CD081E7069B002B7FF47EAFFE
:107A800086E70B9B002B7FF479AF7EE7204617F04B
:107A90000BFEDC220021384849F05DFCA0E62046C0
:107AA00017F002FEDC220021344849F054FC92E633
:107AB00017F0FAFDDC220021384649F04CFC85E63F
:107AC00059463846F4F7B4F997FBF0F29BFBF0F314
:107AD00092B29BB291E62A4A002313701CE698F8F2
:107AE000453F274A003B18BF012388F8313F002358
:107AF000C8F8643FA8F8683FA8F86A3F88F8783F5C
:107B000002231370D8F8702FD8F8FC3CC8F86C2FFB
:107B1000C8F8743F00E621F0004222F07F02002AFC
:107B20003FF44FADA5E5174D15232A698DF8573061
:107B30006B69A86802FB03F3834213D06B68E868A3
:107B40000DF15701184449F0CDF96B682A69A8680E
:107B5000216813446A6901326A61B3FBF0F200FBE9
:107B600012336B6041F004014FF40040216017B004
:107B7000BDE8F04F42F05AB9F02F0020142F00203A
:107B800050470020647900202DE9F047944CD4F848
:107B9000A82594F8AC35D2F8289088B033B9914B29
:107BA0001B685B0674D408B0BDE8F0878E4DD5F82D
:107BB000AC3F05F6A47098470028F0D08B4E737F39
:107BC000002B40F08E80022384F8C035D6F81E309A
:107BD000B6F92200C5F8CA3FB6F91E20B6F9203022
:107BE000A5F8CE0FB5F9C41F814FDFF81482DFF876
:107BF00014A2891AB5F9C62F0591D21AB5F9C83F52
:107C0000069205A91B1A95F8E02F079308461FF066
:107C10006BFA05A81FF018FADDED057A754BF8EE42
:107C2000E76ADDED067A93ED076AB8EEE77ADDEDF7
:107C3000077AF8EEE77A66EE866A27EE067A67EE4E
:107C4000867AC7ED026A87ED037AC7ED047A07F1F9
:107C5000080507F1740614370BE008F104083046F4
:107C6000D4F88C369847AF4206F1240605ED010A98
:107C700095D09AF80030B5EC010A012BEDD18DEDCD
:107C8000030A46F043F99DED030A48F8040BE6E7C2
:107C9000594C94F82830002B85D04FEAE9752946D5
:107CA000484643F0BBFC524BD4ED0F6A94ED107A7A
:107CB000D3ED025A93ED036AA36CE16C07EE900AD0
:107CC000E7EEA56A13EB090345EB0105A6EE277A5B
:107CD000C4E91235C4ED0F6A84ED107A08B0BDE82E
:107CE000F08794F8C035012B72D1B5F9C43F07EE87
:107CF000903AB5F9C63FF8EEE77A07EE103AB5F9D3
:107D0000C83FCDED057A07EE903AB8EEC77AF8EEA7
:107D1000E77A04F5B86705A938468DED067ACDED0A
:107D2000077AF4F719F994F8C035012B0AD100232A
:107D3000C5F8CA3FA5F8CE3F2D4B00229A60DA6005
:107D40001A612CE7022B24D000220023059306930E
:107D5000079394461346114610461746CDE900C2D4
:107D6000A5F8CC0FA5F8CE1F308471840120042122
:107D7000224AA5F8CA7FF783F4F7FAFED4F8A835AB
:107D800000200021C3E90C01C3E91001C3E90E0181
:107D9000D2E797ED065AD7ED0C5A97ED126A8DEDA2
:107DA000055AFDEEC56ABDEEE57A16EE903AFDEE97
:107DB000C67A1FB217EE103A18B217EE903A19B2FF
:107DC000CDED065A8DED076A3B4684460A46C5E767
:107DD000B5F9CA2FB5F9CC3FB5F9CE0F02E700BF10
:107DE000E0010120FC000120A0810020EC3F0020E8
:107DF0008C070120449100201043002038BF060862
:107E0000EC7A0020033C00202DE9F04F8FB01DF0EC
:107E1000FFF9DFF8F881794BA3EB0802CDE90123E4
:107E20004FF00309102200210AA849F094FA019B9F
:107E30000993029B0893724BCDF81C801A69002AA3
:107E4000BFBF704A5A6002F188325A600124F3229F
:107E5000DA604FF0000A7E23224604A907A88DF8B5
:107E60003440CDF830A08DF81030F5F71DFC5045AA
:107E700015DA0023B9F1010900F0B980002BD1D047
:107E800098F800307E2B40F0B580F5F7DCFB002839
:107E900000F0B0800FB0BDE8F04F1DF0D3B922461E
:107EA00004A95046F5F7C4FB574CDFF864B1ADF8B0
:107EB00012005C453CD30024022205A907A8ADF8B6
:107EC0001440F5F7F1FBA042D3DBBDF8120002220B
:107ED00005A9F5F7ADFB0222ADF812000DF1120174
:107EE00007A8F5F7E1FBA042C3DB0B9888B1079B1D
:107EF000089A03449342BCD80AABC0F1040221465D
:107F0000184449F028FA0AA907A8F1F750F9CDE971
:107F10000B400C9B002BACDB9DF8342022B1384980
:107F20000A6942F000420A61B3FA83F35B09A1E7F0
:107F300062888DF819A0C2F30B06B31DADF814309A
:107F40002388C3F30B011B0B8DF818301304ADF815
:107F5000161020D4062205A907A8F5F7A5FB0028CE
:107F600087DBBDF81200062205A9F5F761FB616801
:107F7000ADF81200324607A8F5F796FB0028FFF689
:107F800078AFBDF8120061683246F5F751FBADF8E5
:107F9000120014348DE700273D460135EDB206226C
:107FA00005A907A88DF81950F5F77EFB0028FFF604
:107FB00060AFBDF81200062205A9F5F739FB61682C
:107FC000ADF812003944324607A80391F5F76CFB6F
:107FD0000028FFF64EAFBDF8120003993246F5F7C0
:107FE00027FB032DADF812003744D6D1D1E7002B83
:107FF0007FF446AF0520FBF7CBF900BF00800008F7
:10800000003C024023016745ACFF06080040000821
:108010009804070870B50C4E35782D1A18BF012545
:108020000328044634BF044600242046F5F7B4FB79
:10803000064B347003F6E4701A2204FB0200C3F806
:10804000E80C284670BD00BFED3B0020A081002059
:10805000022810B50C4614D8FFF7DCFF0948FBF7DF
:10806000A7FA094B094819780131FBF7F7FA2146BD
:108070001020FBF79DFB21462020BDE81040FBF7B8
:1080800097BB10BD06B70608ED3B0020FDAF060804
:1080900038B5174C174DAC4217D30020F5F77CFBD1
:1080A00015481DF0EBF8154A136843F4800313607C
:1080B000134B2F221A7030225A70124B1878FFF788
:1080C000A9FFBDE8384026F0FFBEB4F90230002B0E
:1080D0004FF00001204607DAF5F74EFB012120465C
:1080E000F5F74AFB02212046F5F746FB1434D2E7A8
:1080F000ACFF060898040708DCAF060874390020B6
:10810000143F0020ED3B002010B5064B5C78241A8C
:1081100018BF0124032828BF002058701EF04CFD12
:10812000204610BDED3B0020022810B50C4610D8AB
:10813000FFF7EAFF0748FBF73BFA074B0748597878
:108140000131FBF78BFA21463020BDE81040FBF7E8
:108150002FBB10BDE5AF0608ED3B0020F5AF0608CC
:108160002DE9F04F0D468DB0B8490446FDF798F95A
:108170000646002840F0BF80B5492046FDF790F93B
:108180000646002840F0B980B2492046FDF788F93C
:108190000646002840F0B3802046AF49FDF780F93D
:1081A0000028064612BF1024264601240DB144F0D3
:1081B0002004AA4DAA4F95F8009095F80180DFF8A9
:1081C0001CA35745C0F09D80FFF762FF4846FFF7AC
:1081D00021FF4046FFF798FFA2493046FDF760F9BE
:1081E00008B144F0400414F01103009300F08B82B6
:1081F0009D48FBF7DDF90020FDF7A8FC9B48FBF745
:10820000D7F99B48FBF7BAF904F03003302B02D1C1
:108210009848FBF7CDF9984E9848DFF8C492FBF7E1
:10822000C7F99748FBF7C4F9D6ED007A954AF5EE01
:10823000407AF1EE10FA0CBF012100212046FBF735
:10824000C3F93146904A914E2046FCF789F8904890
:10825000FBF7AEF936F9C41C8E4AB1FA81F149092F
:108260002046FBF7B1F9A6F1C6018B4A2046FCF780
:1082700037FF8A48FBF79CF9894A8A492046FCF770
:1082800077FE8948FBF794F9884A89492046FCF72C
:1082900071FB8848FBF78CF9874B884A1E68884B2E
:1082A0001F6867EA0603CB464FF0000A01935BF8AC
:1082B000043B002B32D01978D1B1019902934FF0D1
:1082C000010808FA0AF811EA080F14BF0121002179
:1082D0002046FBF793F966EA070111EA080F774A8F
:1082E000029B14BF012100212046FBF76DF9734A60
:1082F0000AF1010ADBE7012458E7022456E70424C7
:1083000054E77B88C3F30B021B04D7E9011048BF75
:1083100002EB420248F0E6FD143752E79846694AFC
:1083200067EA0603019359F804BBBBF1000F27D09D
:108330009BF8001009B34FF0010A0AFA08FA17EA8D
:108340000A0F0BD066EA070111EA0A0F5B4614BF59
:10835000012100212046FBF751F95A4A16EA0A0F7B
:108360000BD0019B13EA0A0F18BF01215B4608BF1F
:1083700000212046FBF728F9524A08F10108D2E70C
:108380005148DFF860A1FBF713F9504AD2F800908A
:108390004F4A12685E4689EA0208DFF84CB16FEA7C
:1083A00008080127B74018EA070F14BF0121002170
:1083B00019EA070714BF52465A4630460391019204
:1083C00016F094FD019A039902900346204601910C
:1083D0000136FBF713F9002F14BF5A465246029B91
:1083E00001992046FBF7F0F8182EDAD13948DFF86A
:1083F000FCA0DFF8FC80DFF8FC90FBF7D9F8364BE7
:108400009F680026F3B20AEB8302D2F834B1BBF1C5
:10841000000F71D00121994039405B460CD04A468B
:1084200000212046FBF7D0F85B464A460021204653
:10843000FBF7E4F80136E5E7424620460191FBF7F9
:10844000C3F801995B464246F1E700BF1FB006083A
:1084500006B70608E5AF060826B00608ED3B002083
:10846000ACFF06082AB006085BBA060837B0060853
:108470004FB006085BB00608B47F00204CB7060872
:10848000ABB0060896B00608347C00209892002015
:10849000A5B00608B1B0060800820020BEB00608EC
:1084A000843D0020E0480020C4B00608047D002080
:1084B000447F0020CDB00608C44B0020D5B006088C
:1084C00074390020E1B00608A8B40608844A0020E8
:1084D000E43E0020ECB006080C4C0020980407088D
:1084E000CC3706080AB0060814B006081C37060880
:1084F00001B10608F5B006088A48FBF759F80123D0
:108500008948DFF8DCC2DFF8DCE28DF820B08DF8B6
:1085100010B08DF821B08DF811B08DF822B08DF823
:1085200012B08DF823B08DF813B01F4613F80C204D
:1085300010F8016B0CA911440DF1300801F8206C02
:1085400013F80E10884408F8106C17B1561A7742C9
:1085500077410133052BE9D1744A002608AB39462F
:1085600020468DF81460FBF749F804AB6F4A394692
:108570002046FBF729F86E48FBF71AF86D4A6E495A
:108580002046FBF7F5FC6D48FBF712F86C4A6D4985
:108590002046FCF79DFA6C48FBF70AF86B4A6C49D9
:1085A0002046FCF7ADFB6B48FBF702F8644A6549CF
:1085B0002046FCF741FC6848FAF7FAFF674A684929
:1085C0002046FBF717FC6748FAF7F2FF664A67494F
:1085D0002046FBF7D9FD6648FAF7EAFF654A664987
:1085E0002046FBF7B7FF6548FAF7E2FF644A6549A2
:1085F0002046FCF74BF86448FAF7DAFF6349204657
:108600003EF00CF86248FAF7D3FF4FF0FF331A46FA
:10861000604920463EF08CF85F48FAF7C9FF5F4A90
:108620005F492046FCF759FF5E48FAF7C1FF5E4AF2
:108630005E492046FDF764F85D48FAF7B9FF5D4AE8
:108640005D492046FDF7F2F85C48FAF7B1FF304685
:108650002146FBF7ADF8E0064BD52146304695F8AC
:1086600000806F78FFF7F4FC21460120FFF7F0FC53
:1086700021460220FFF7ECFC21463046FFF754FD6F
:1086800021460120FFF750FD21460220FFF74CFD57
:108690004046FFF7BFFC3846FFF736FD4848FAF77B
:1086A00087FF484808F10101FAF7D8FF4648791CCE
:1086B000FAF7D4FFA10703D528782146FFF7C8FCB5
:1086C000620703D568782146FFF72EFD009B13B1A2
:1086D0003E48FAF76DFF2EB13D48FAF769FF3D4875
:1086E000FAF74CFF3C4C3D4DAC420ED30DB0BDE80B
:1086F000F08F28782146FFF7ABFC68782146FFF71A
:1087000013FD0126D6E7009ED4E76388C3F30B026E
:108710001B04D4E9010148BF02EB420248F0E2FB2E
:108720001434E1E70EB10608803C060812B10608D1
:1087300011B80608BC450020A04C002002AA06087B
:10874000647D0020547E00201EB10608E47D0020D8
:10875000D47E002019B1060824B10608197B002038
:10876000EC80002028B10608B97B0020748000202E
:1087700031B10608F47C0020A47F002039B106083E
:10878000C04100207049002045B10608B092002089
:1087900048B10608F09D002053B10608C0820020B1
:1087A00030A2002059B10608C088002030A800205F
:1087B00065B106082089002090A800201FB0060897
:1087C00082B10608ADB10608A5B10608B8B1060821
:1087D000D1B10608E7B10608ACFF060898040708FF
:1087E00092920020D08D00200021B9E40121B7E44D
:1087F0002DE9F74F1CF00CFDB54CB64B9C42C0F078
:108800000C81B54C2078FFF705FC6078FFF77CFC05
:10881000B24BB3481A7C597C914224BF00221A748F
:10882000F4F768FFAF4B1A68AF4B93431FD1002199
:108830001820F0F73AFE0546C8B100211120F0F7E4
:1088400034FE002800F0188104682868231A5C426E
:108850005C4100212320F0F728FE18B102682B6844
:108860009A4200D01CB14FF48030F4F743FF00254A
:108870009E4E2C46FF2748F2BC3856F82500430888
:10888000810801F0333103F077330B44C10801F064
:108890001131C31A5B1A03EB131310F0010203F03A
:1088A0000F33B3FBF7F1C1EB012118BF0134A3EB88
:1088B000010318BFE4B2012B08D9022B0CD112B16D
:1088C00010EA080F02D140F0D7FD28B103350F2D73
:1088D000D3D1013C022C03D984480D2141F082FC04
:1088E000834A138DD18C643B8B42A8BF0B46D38443
:1088F00000BF804B9A780AB908229A7000200CF0C9
:1089000029FE7D4A1368002800F0B88023F08063B8
:1089100013607A4B7A4CD3F8E86C0EF0F7FA794B87
:1089200031781D88DFF8ECE183B22D1A64220093C0
:1089300005FB01F393FBF2F313FA80F0A4F8700542
:1089400096F80180C1F16E0301EB8107A2EB080BE1
:108950009BB24A42C1F1640C7F0092B201935FFA6C
:108960008CFC4FF00A0A4FF47A7916B2002E40F3CD
:108970008880604606FB06F308FB03F310FB00F05B
:1089800093FBF0F0584406FB00F3009893FBFAF3D6
:108990003B441BB26B4393FBF9F303442EF8023BB9
:1089A0000A32019B92B29342DFD11EF01FF93022AE
:1089B0000021554848F0CFFC0CF036FC94F8A61581
:1089C000524BC820642212FB0101996094F8A7154C
:1089D00012FB0102DA600022C3E90422C3E9062285
:1089E000C3E9082283F8292083F82A20DA624FF0AD
:1089F0007A7294F8A9151A6383F828101DF0CEFD39
:108A00001DF0F2FD0CF0F2FF10F046FB35F014FB08
:108A100003B0BDE8F04F1CF015BCB4F90230DFF82C
:108A2000F890002BADBF002703274FF00108B84690
:108A3000002608EB0601C9B28F4201D21434DCE6ED
:108A4000334A02F1060ACA453CD21588D5B35019FB
:108A5000484537D2052D35D9B4F800C0B2F802E048
:108A6000CCF30B0CE64505D192F805C00CF0030CD5
:108A70008C450AD00246E4E70446EAE643F0806308
:108A800046E714BF0846012074E73146204692F8B5
:108A900004B0F4F771FE2188BBEB113F10D1B4F89C
:108AA00002C06068CCF30B01AA1F8A42A8BF0A4625
:108AB0001CF4004F18BF01FB0600514648F012FAA3
:108AC0000136B6E731462046F4F756FEF8E700BF18
:108AD000ACFF060898040708ED3B0020684300201F
:108AE000206314067439002040000100BC450020BA
:108AF0001446002058410020F0000120A0810020F1
:108B000090A30020083E002004A900207C43002000
:108B100001400008A40201200080000808B5FFF70A
:108B200073F9FFF765FEBDE80840012017F0F4B8BF
:108B300010B50446FFF76EFA18B1FFF765F9FFF7B5
:108B400057FE601CC0B2BDE8104017F0E5B838B55C
:108B50000C4D04462046FAF747FF38B10A4B0B4844
:108B60001978BDE838400131FAF778BD2046F4F7AE
:108B700023FD0138022804D8C0B2FFF7D9FF2C46E4
:108B8000E8E738BD8EBF0608ED3B0020ADB1060812
:108B900010B50446FFF7B8FA18B1FFF735F9FFF73B
:108BA00027FE601CC0B2BDE8104017F0B5B838B55C
:108BB0000C4D04462046FAF717FF38B10A4B0B4814
:108BC0005978BDE838400131FAF748BD2046F4F73E
:108BD000F3FC0138022804D8C0B2FFF7D9FF2C46B5
:108BE000E8E738BD8EBF0608ED3B0020A5B10608BA
:108BF000174B10B51C68620705D5164B1B78022B66
:108C000001D0012010BD230703D5134B1B68D805E5
:108C1000F7D5A10603D5114B1B7E022BF1D139F0FC
:108C200077F80028EDD00E4B93F89026012A01D159
:108C3000A207E7D493F8AC050028E3D0094A507F97
:108C40000028DFD093F8C005023818BF012010BDFE
:108C5000FC00012058470020F8000120904000202F
:108C6000E0010120EC3F0020034B1B685B0700D4B0
:108C7000704709F027B900BFF00001202DE9F04F3F
:108C8000DFF89CA29FED9C7ADAF8A8359C6A9B4B92
:108C900007EE904AF8EEE77A2DED088B67EE877ABB
:108CA000C3F8544C0AF5DE63C3ED007A944B1B689D
:108CB000AFB05B07CDE90B0140F13881914B0593D3
:108CC0001B68DF0600F18A82DFF858928E4FD9F8D0
:108CD000B835D9F8BC25D7ED076AD7ED0F7A97EDEF
:108CE000117A97ED136A1B19C9F8B835D9F8C03550
:108CF00042EBE4721B19F4EEE67AC9F8C035D7ED01
:108D0000107AD9F8C435C9F8BC2543EBE473F1EE09
:108D100010FAF4EEE67AD7ED087AC8BFC7ED0F6A0D
:108D2000F1EE10FAB4EEE77A97ED127A48BFC7ED8C
:108D3000106AF1EE10FAB4EEE77AC8BFC7ED117A07
:108D4000F1EE10FA48BFC7ED127A67EEA77A97EDF9
:108D5000097AC9F8C435E6EEA67A9AF8AC35B4EECD
:108D6000C76AE7EE077A97ED146AF1EE10FAB4EEEF
:108D7000C76AC8BF87ED137AF1EE10FA48BF87EDD6
:108D8000147AB1EEE77A97ED156AB4EEC76AF1EEA0
:108D900010FA48BF87ED157A002B40F0D7805B4B67
:108DA00000935B4B1B689D0700F17E86594B0B9A25
:108DB00043F8082C0C9A43F8042C0023FB613B6217
:108DC0007B62554B93ED000AFEF730F84B4B93F85E
:108DD000467C002F40F0178699F8143D002B40F098
:108DE000B285DFF844B199F8CA3D002289F8142D04
:108DF000002B00F05985F9F741FF05460C4639F084
:108E0000E5F8284621463DF092FE2846214638F0F6
:108E10008FFFF9F733FF9BF806300022022B07463D
:108E20008846A9F8602F00F01F8426232E21CDE963
:108E300007310E232A2406932223CDE903340A2383
:108E4000029306262C244FF0240E4FF00C0C2822FF
:108E5000202308210425022001909BF80900022804
:108E60000AD1019BA9F8603FDDE907E4DDE903329F
:108E7000DDF818C0029935469BF8070002289BF8D8
:108E8000100001BFA9F8605F22467346614610B129
:108E9000A9F8601F13469BF80A200598022A08BF0C
:108EA000A9F8603F164B01681B6821F0800213F09F
:108EB0000403026000F0F5839BF80030174A03EBCF
:108EC000830302EBC30311F4C01FB3F8CA464FF08B
:108ED0000003ABF8043040F0BB81CA0641F1ED85D8
:108EE000E30601F19786260702F10D873A464346CD
:108EF000204635F049FFB0E1BD378635A08100201E
:108F0000F0000120F8000120D4080120D81201202F
:108F1000FC00012030B00020D00801201C370608DA
:108F2000E001012090A30020284D0020B84BB94A51
:108F3000059200200021C3E90001A3F5B8690AF2F7
:108F4000F4679AF8AC35002B3FF429AFB24AB34B23
:108F50000192B34A0092B34A099203F5CC72B24926
:108F6000B24C039203F5607803F55772DFEDB08AD7
:108F70009FEDB09A9FEDB08A04930A940D910291EF
:108F8000079203F50675CDF818800026049BAB48C0
:108F9000B3EC010A0493019B1B780F2B01BFFDEE7C
:108FA000C07A029A17EE903A1360A54BF1B21B6893
:108FB0009847019B03981B780F2B01BFFDEEC07AE9
:108FC000029A17EE903AD360009BD3F8843E9847FC
:108FD0009AF8C837002B40F0DC806C35099B1B7F6A
:108FE000002B42D1049B03ED010A029B0433029340
:108FF000039B24330393079B0C330793069B013693
:109000000433032E04F511740693BFD19AF8C837C0
:10901000002B3FF4C6AE99F8943C00228AF82C2F1E
:109020009BB99AF84029D8F80050D8F80440D8F8ED
:109030000810501C00F03F008AF8400908EB82003D
:109040000561C0F81041C0F81012013303F00103AC
:1090500089F8943C9AF8443C032B03F2B780DFE88C
:1090600013F0F414A815CD0E8414A38C0A9806EB03
:10907000C60206EB02121A4400EB820181ED0A0AD5
:10908000D4ED8D7AD4ED8E6A94ED8C7A70EE677A99
:10909000013367EEA77A9BB2C1ED4B7AB4F8401268
:1090A000A384F2009942324438BF002306EB021237
:1090B0000A9938BFA384134401EB830292ED0A6A34
:1090C000019B30EE077A77EEA67A37EE467AD4ED3A
:1090D0008F6A84ED8C7A92ED4B6A1B7877EEC67AB4
:1090E00027EE267AC4ED8E7A84ED8D7A27EEA67A65
:1090F000B5EEC07AF1EE10FAA8BFF1EEC77A84EDB2
:10910000087AACBF27EE887AB0EE497A152B84ED49
:10911000017A73D0D4ED046AD4ED057A76EEA66AAE
:1091200076EEE75A77EEE67AF5EE405AF1EE10FA6F
:1091300014BFD4ED074A94ED065AC4ED055A1EBF7C
:1091400084EEA56AB7EE005A35EE465AD4ED004AD1
:1091500094ED026A18BFB0EEC55AA4EE856A18BF36
:1091600084ED065A36EE077A77EE807A86EE075A55
:10917000F7EE006AE5EE275A76EEC57AB0EE650A9C
:1091800067EE867A84ED035AC4ED045AC4ED027A80
:1091900028E7069B83ED000A019B1B78122B01BF79
:1091A000FDEEC07A029A17EE903A1360079BAB4629
:1091B0006C3553F8042B089358460BF1240B904759
:1091C0005D45089BF5D1019B1B78122B01BFFDEE7D
:1091D000C07A029A17EE903AD360FFE60E200BF0A9
:1091E000D1FE002801F0FC84164B93F8D034032BF9
:1091F0003FF66AADDFF85490134FA2E6D4ED037A40
:10920000029B67EEA87AFDEEE77AC3ED007A81E76C
:1092100050A90020F8000120033C00209407012001
:10922000D8120120EC3F0020EC7A002058A9002041
:1092300000007A44000000001F852B3F1C12012013
:1092400010010120D0230120D408012090A3002088
:109250003A464346204638F09DFFC64D9BF8043001
:1092600013B100238BF802309BF8053013B10023B3
:109270008BF803309BF80B302BB1B9F8603F43F00B
:109280004003A9F8603F9BF80C302BB1B9F8603F60
:1092900043F08003A9F8603F9BF80D302BB1B9F87B
:1092A000603F43F48073A9F8603F9BEDFF0A44F0F0
:1092B0002DFEB14BC9F8880F93ED000A44F026FE4D
:1092C00095ED000AC9F88C0F44F020FE059BC9F803
:1092D000900F1A68D20640F1EB81D9F8942FD9F893
:1092E000983F134300F0BD81F9F7C8FCD9F8A03FBF
:1092F000A24DA34CA34FC31ACDE90301022008EEEF
:10930000903AF5F784FB05FB00F09F4DA5FB003577
:10931000B4F90630401B05EB500503EB8303ED0A5F
:1093200003EB830305EB850200209D00C5EB42059E
:10933000B4F9043095FBF3F5F5F769FB2188934CFC
:10934000A1FB0031D81841EB0102C01841EB020229
:10935000D20042EA5072C000C01841EB02014B013A
:10936000420143EAD063801841EB03018900884A37
:1093700041EA90710023800042F0E6F92DB286B2F6
:1093800005FB06F384FB0324DB17C3EB6413029392
:109390007C68D9F8A03FD9F8941F06932343A5EB26
:1093A000010540F07B8797ED027ADFED7A7AB9F814
:1093B000AC2FDFED795A019125EAE573B8EEE88A22
:1093C000764D28EE278AD5ED017A95ED000A85EDD8
:1093D000028A78EE277A02FB03F388EE276A07EE0B
:1093E000903AF8EEE77AF0EE406AD7EEA56A36EEEC
:1093F000877AA6EE070A85ED000A44F087FD99F802
:10940000C43F01998046002B40F07087BAF92200D2
:109410000190002900F01F811FFA88F8A0EB0808CE
:10942000B8F57A7F019AB8BF4FF47A78904580F208
:109430001281002B01F0C3830FFA88F30193029B82
:10944000D9F8985F581B069B234340F08E87544BF6
:1094500093ED007A534CB9F8AC3FD4ED017A94ED1A
:10946000000ADFED515A84ED028A78EE277A20EA6D
:10947000E07088EE276A03FB00F0B0FBF6F007EE21
:10948000900AF8EEE77AF0EE406AD7EEA56A36EE7B
:10949000877AA6EE070A84ED000A44F037FD99F8B2
:1094A000F08F0646B8F1000F40F04287BAF922006B
:1094B0000246002D00F0C780B6B2861BB6F57A7F53
:1094C000B8BF4FF47A76964280F2BD80374B029354
:1094D000B8F1000F01F0628332B2039BC9F8A03FDC
:1094E000049B7B60019B9342A8BF1346AAF82230DD
:1094F000009B93F8308FB8F1000F00F083802C4B65
:10950000D3ED008A2B4BD3ED027AD3ED016A93EDB4
:10951000046A67EEA77AF0EE005AE6EEA67AB7EE96
:10952000007AA7EEE57AB4EEC76AF1EE10FA00F31E
:109530004987059B1B680493DE0601F121869BF891
:1095400000301D4A03EB830302EBC303B3F8CA36B2
:109550001D0641F155879BF80D30002B41F0108618
:10956000BAF920300793DAF8C0300393022300F0F1
:1095700033BF00BF2C5100202851002010090500E6
:10958000F43E002030B30020010110001F85EB5194
:10959000187C3E00BD3786356F12833A44B30020F5
:1095A0006CB3002070B30020CDCCCC3D88B400203B
:1095B000D00801200C2201201C37060807EE903A43
:1095C000A74ABAF9DC3082FB0312DB17C3EBA20314
:1095D0001BB207EE103AB8EEC77AF8EEE77AB0EEB3
:1095E000C77AB4EEE77AF1EE10FA02F34B83002368
:1095F000069AB0EE680A82F87D344046D7F8C43443
:10960000022198470EF074F8964B1B78002B40F01F
:109610001881954B1B78002B40F0F380934B1B78FF
:10962000002B40F0EB80059B1A68940200F1A180AA
:10963000029B13F8D83C002B00F08D802FB0BDECBE
:10964000088BBDE8F08F00232360002389F8F03FEA
:10965000874B029341E700232B60002389F8C43F26
:10966000EDE6834B029343E701232F25A9F8603FE2
:109670002723CDE907350F234FF02B0C0693232327
:10968000CDE9033C0B23029307262D244FF0250E32
:109690004FF00D0C29222123092105250320FFF776
:1096A000DBBBD206ABF811308BF8EC3F3FF515AEC3
:1096B0009BF800306F4A03EB830302EBC303B3F85C
:1096C000CA36DB0541F16B86F7EE008A0DF01EFC11
:1096D00007EE900ABAF92240B8EEE78A0DF016FCC0
:1096E000241A07EE904A644B9FED646A93ED017A69
:1096F000F8EEE76AD3ED027A67EEA77AE7EE077A2B
:10970000F4EEC67AF1EE10FA02F3E482B7EE007AD4
:10971000F0EE005AB0EE476AA7EEE56AC7EE067AA9
:1097200077EEC77AB7EE007AA8EEA77AF0EE487A1D
:10973000E6EE877AFDEEE77A17EE904A0DF0E6FB4B
:109740004F4B84421B8803DBA342A8BF2346184625
:10975000AAF82200C1E54B4B1B6819037FF56EAFD9
:10976000F9F78CFA2FB0BDEC088BBDE8F04F1FF075
:10977000AFBC12F4003104D0434BDB79002B3FF433
:1097800057AF424B1B78232B01F0FE81404B1868EA
:1097900010F0040402F0C880029B13F8E03C002B98
:1097A00001F04482500141F1D8870FF04BF8364B5D
:1097B000DB79002B42F0848232F0CAFA10F4C06FD9
:1097C0007FF436AF03201BF079FD029D55F8DC3C99
:1097D00008EE100A1C8E0DF099FB231807EE903A44
:1097E000B8EEC88AFAEEEF7AB4EEE78AF1EE10FA34
:1097F0004CBF0123002305F8E03C19E70DF010FDF4
:1098000011E714F031FF234B5B78032B01F00C863A
:10981000214B224F1B783A789A421E46FFF4FEAE47
:109820001F4D002405EB430535F9021BE0B289B258
:10983000F7F762F83B7801369E4204F10104F3DD4C
:10984000ECE6184C94ED000A17F0B8FB0D4B1B68C2
:10985000002B81F2718194ED000A15F023F8D8E60F
:1098600067666666063E0020053E0020934800209D
:1098700088B400201C3706080C220120CCCC4C3EBA
:10988000083E0020F400012014460020033C002084
:10989000F00001200C460020617900206079002052
:1098A000643D0020D0080120744C754AD4ED0F7A35
:1098B0009FED747A517F77EE877A0022C4F8742185
:1098C000C4F87821C4F87C21C4F88021C4F81021A0
:1098D000002604F154020027C4ED597AC4ED5A7AE7
:1098E000C2E92667C2E90067C2E90A67C2E91267EE
